 SDKRIL

 Timestamp is 540049bf (Fri Aug 29 17:37:03 2014)

 Preferred load address is 10000000

 Start         Length     Name                   Class
 0001:00000000 00050538H .text                   CODE
 0001:00050538 000000bcH .text$yc                CODE
 0001:000505f4 00000074H .text$yd                CODE
 0002:00000000 0001d1a8H .rdata                  DATA
 0002:0001d1a8 00000073H .rdata$debug            DATA
 0002:0001d21c 000001bcH .rdata$r                DATA
 0002:0001d3d8 00000254H .xdata                  DATA
 0002:0001d62c 00000124H .xdata$x                DATA
 0002:0001d750 00000050H .idata$2                DATA
 0002:0001d7a0 00000014H .idata$3                DATA
 0002:0001d7b4 00000228H .idata$4                DATA
 0002:0001d9dc 00000196H .idata$6                DATA
 0002:0001db80 000059bdH .edata                  DATA
 0003:00000000 00000228H .idata$5                DATA
 0003:00000228 00000004H .CRT$XCA                DATA
 0003:0000022c 00000004H .CRT$XCAA               DATA
 0003:00000230 00000004H .CRT$XCC                DATA
 0003:00000234 00000010H .CRT$XCU                DATA
 0003:00000244 00000004H .CRT$XCZ                DATA
 0003:00000248 00000004H .CRT$XIA                DATA
 0003:0000024c 00000004H .CRT$XIZ                DATA
 0003:00000250 00000004H .CRT$XPA                DATA
 0003:00000254 00000004H .CRT$XPZ                DATA
 0003:00000258 00000004H .CRT$XTA                DATA
 0003:0000025c 00000004H .CRT$XTZ                DATA
 0003:00000260 00000c1fH .data                   DATA
 0003:00000e80 00006850H .bss                    DATA
 0004:00000000 000028e0H .pdata                  DATA
 0005:00000000 00000058H .rsrc$01                DATA
 0005:00000060 000003a0H .rsrc$02                DATA

  Address         Publics by Value              Rva+Base       Lib:Object

 0000:00000000       ___safe_se_handler_count   00000000     <absolute>
 0000:00000000       ___safe_se_handler_table   00000000     <absolute>
 0001:00000000       ??0BerTlv@@QAA@PBEI@Z      10001000 f   parse.obj
 0001:00000034       ?Parse@BerTlv@@QAAHPBEI@Z  10001034 f   parse.obj
 0001:000001d4       ?EncodedStringSizeToUnicodeStringSize@@YAHW4ENCODING_TYPE@@IAAI@Z 100011d4 f   parse.obj
 0001:000002a4       ?MatchStringBeginning@@YAHQBD0AAPBD@Z 100012a4 f   parse.obj
 0001:00000354       ?MatchStringEnd@@YAHQBD0AAPBD@Z 10001354 f   parse.obj
 0001:000004ac       ?MatchStringAnywhere@@YAHQBD0AAPBD@Z 100014ac f   parse.obj
 0001:0000052c       ?MatchBytesEnd@@YAHQBEI0IAAPBE@Z 1000152c f   parse.obj
 0001:000005d4       ?MatchBytesAnywhere@@YAHQBEI0IAAPBE@Z 100015d4 f   parse.obj
 0001:00000678       ?ParseDWord@@YAHQBDHAAKAAPBD@Z 10001678 f   parse.obj
 0001:000007bc       ?ParseHexDWord@@YAHQBDHAAKAAPBD@Z 100017bc f   parse.obj
 0001:000009c4       ?ParseUInt@@YAHQBDHAAIAAPBD@Z 100019c4 f   parse.obj
 0001:00000a00       ?ParseIntAsUInt@@YAHQBDAAIAAPBD@Z 10001a00 f   parse.obj
 0001:00000ac0       ?ParseUIntAndVerifyAbove@@YAHQBDHIAAIAAPBD@Z 10001ac0 f   parse.obj
 0001:00000b38       ?ParseUIntAndVerifyBelow@@YAHQBDHIAAIAAPBD@Z 10001b38 f   parse.obj
 0001:00000bb0       ?ParseHexUInt@@YAHQBDHAAIAAPBD@Z 10001bb0 f   parse.obj
 0001:00000bec       ?ParseFixedPoint@@YAHQBDAAKAAPBD@Z 10001bec f   parse.obj
 0001:00000d68       ?ParseString@@YAHQBDQADIAAPBD@Z 10001d68 f   parse.obj
 0001:00000eb0       ?AppendStringUCS2W@@YAHPBGAAPADQAD@Z 10001eb0 f   parse.obj
 0001:00000fd4       ?ParseStringGSMW@@YAHPBDQBDPAGQAG@Z 10001fd4 f   parse.obj
 0001:000013c8       ?ParseStringHexW@@YAHPBDQBDPAGQAG@Z 100023c8 f   parse.obj
 0001:000014e0       ?ParseStringUnicodeW@@YAHPBDQBDPAGQAG@Z 100024e0 f   parse.obj
 0001:000015c8       ?ParseStringUTF8W@@YAHPBDQBDPAGQAG@Z 100025c8 f   parse.obj
 0001:000016b0       ?ParseQuotedEncodedString@@YAHW4ENCODING_TYPE@@AAPBDPAGQAG@Z 100026b0 f   parse.obj
 0001:00001788       ?AppendStringGSMW@@YAHPBGAAPADQADHH@Z 10002788 f   parse.obj
 0001:0000189c       ?AppendStringHexW@@YAHPBGAAPADQADH@Z 1000289c f   parse.obj
 0001:00001a04       ?AppendStringUnicodeW@@YAHPBGAAPADQADH@Z 10002a04 f   parse.obj
 0001:00001adc       ?AppendStringUTF8W@@YAHPBGAAPADQADH@Z 10002adc f   parse.obj
 0001:00001bb4       ?AppendEncodedString@@YAHW4ENCODING_TYPE@@PBGAAPADQADH@Z 10002bb4 f   parse.obj
 0001:00001cb8       ?AppendQuotedEncodedString@@YAHW4ENCODING_TYPE@@PBGAAPADQAEH@Z 10002cb8 f   parse.obj
 0001:00001dc8       ?ParseEncodedString@@YAHW4ENCODING_TYPE@@PBDQBDPAGQAG@Z 10002dc8 f   parse.obj
 0001:00001eb8       ?ParseUnquotedString@@YAHQBDDQADIAAPBD@Z 10002eb8 f   parse.obj
 0001:00001fe8       ?ParseUnlimitedString@@YAHQBDAAPADAAIAAPBD@Z 10002fe8 f   parse.obj
 0001:0000217c       ?ParseUnlimitedUnquotedString@@YAHQBDDAAPADAAIAAPBD@Z 1000317c f   parse.obj
 0001:000022dc       ?FlagFromValue@@YAHIQBULISTVALUEMAP@@IAAK@Z 100032dc f   parse.obj
 0001:000023ec       ?FlagFromString@@YAHQBDQBULISTSTRINGMAP@@IAAK@Z 100033ec f   parse.obj
 0001:000024cc       ?ValueFromFlag@@YAHIQBULISTVALUEMAP@@IAAI@Z 100034cc f   parse.obj
 0001:00002570       ?StringFromFlag@@YAHIQBULISTSTRINGMAP@@IAAPBD@Z 10003570 f   parse.obj
 0001:00002614       ?ParseRangeList@@YAHQBDQBULISTVALUEMAP@@IAAKAAPBD@Z 10003614 f   parse.obj
 0001:000028dc       ?ParseStringList@@YAHQBDQBULISTSTRINGMAP@@IAAKAAPBD@Z 100038dc f   parse.obj
 0001:00002a54       ?ParseRspPrefix@@YAHQBDAAPBD@Z 10003a54 f   parse.obj
 0001:00002a8c       ?ParseRspPostfix@@YAHQBDAAPBD@Z 10003a8c f   parse.obj
 0001:00002ad0       ?FindRspPostfix@@YAHQBDAAPBD@Z 10003ad0 f   parse.obj
 0001:00002b14       ?SkipChars@@YAXQBDAAPBDPBD@Z 10003b14 f i parse.obj
 0001:00002b50       ?DeviceRemoval@@YAXK@Z     10003b50 f   SDKRIL.obj
 0001:00002c10       DllMain                    10003c10 f   SDKRIL.obj
 0001:00002c64       SwiApiStartup              10003c64 f   SDKRIL.obj
 0001:00002d0c       SwiApiShutdown             10003d0c f   SDKRIL.obj
 0001:00002e3c       ?SwiGetAudioMode@@YA?AW4SWI_RCODE@@PAGK@Z 10003e3c f   SDKRIL.obj
 0001:00002e68       ?SwiSetAudioMode@@YA?AW4SWI_RCODE@@GK@Z 10003e68 f   SDKRIL.obj
 0001:00002e9c       SwiGetAvailAirServers      10003e9c f   SDKRIL.obj
 0001:00003174       SwiSelectAirServer         10004174 f   SDKRIL.obj
 0001:00003990       SwiGetAirServerInfo        10004990 f   SDKRIL.obj
 0001:00003cdc       SwiSetNetworkPreferenceGobi 10004cdc f   SDKRIL.obj
 0001:00003dcc       SwiModemReset              10004dcc f   SDKRIL.obj
 0001:00003e34       SwiRegisterCallback        10004e34 f   SDKRIL.obj
 0001:00003f50       SwiDeRegisterCallback      10004f50 f   SDKRIL.obj
 0001:00003fd8       SwiNotify                  10004fd8 f   SDKRIL.obj
 0001:0000403c       SwiStopNotify              1000503c f   SDKRIL.obj
 0001:000040a0       SwiGetHardwareVersion      100050a0 f   SDKRIL.obj
 0001:0000443c       SwiGetFirmwareVersion      1000543c f   SDKRIL.obj
 0001:0000451c       SwiGetBootVersion          1000551c f   SDKRIL.obj
 0001:000045fc       SwiGetRadioPower           100055fc f   SDKRIL.obj
 0001:000046ec       SwiSetRadioPower           100056ec f   SDKRIL.obj
 0001:000047a8       SwiGetPriInfo              100057a8 f   SDKRIL.obj
 0001:0000485c       SwiGetPriVersion           1000585c f   SDKRIL.obj
 0001:00004924       SwiStartDataSession        10005924 f   SDKRIL.obj
 0001:00004a90       SwiStopDataSession         10005a90 f   SDKRIL.obj
 0001:00004bd8       SwiGetIPConfigurationGobi  10005bd8 f   SDKRIL.obj
 0001:00004de0       SwiGetServingNetworkGobi   10005de0 f   SDKRIL.obj
 0001:000050c8       SwiGetImagePreference      100060c8 f   SDKRIL.obj
 0001:00005134       SwiSetImagePreference      10006134 f   SDKRIL.obj
 0001:000051bc       SwiUpgradeFirmware         100061bc f   SDKRIL.obj
 0001:00005268       SwiDialCall                10006268 f   SDKRIL.obj
 0001:000052e8       SwiGetModelID              100062e8 f   SDKRIL.obj
 0001:00005354       SwiEndCall                 10006354 f   SDKRIL.obj
 0001:000053c0       SwiAnserCall               100063c0 f   SDKRIL.obj
 0001:0000542c       SwiManageCalls             1000642c f   SDKRIL.obj
 0001:000054a4       SwiATSetCLIP               100064a4 f   SDKRIL.obj
 0001:00005774       SwiATGetCLIP               10006774 f   SDKRIL.obj
 0001:00005f58       SwiATSetCLIR               10006f58 f   SDKRIL.obj
 0001:00006228       SwiATGetCLIR               10007228 f   SDKRIL.obj
 0001:00006794       SwiATSetCOLP               10007794 f   SDKRIL.obj
 0001:00006874       SwiATReleaseCall           10007874 f   SDKRIL.obj
 0001:00006a58       SwiATGetCOLP               10007a58 f   SDKRIL.obj
 0001:00007064       SwiATSetCOLR               10008064 f   SDKRIL.obj
 0001:00007144       SwiATGetCOLR               10008144 f   SDKRIL.obj
 0001:00007654       SwiATSetEnum               10008654 f   SDKRIL.obj
 0001:00007c48       SwiATSetSideToneGain       10008c48 f   SDKRIL.obj
 0001:00008090       SwiATReset                 10009090 f   SDKRIL.obj
 0001:00008474       SwiATRtnReset              10009474 f   SDKRIL.obj
 0001:000088a0       SwiATGetProvisionStatus    100098a0 f   SDKRIL.obj
 0001:00008ddc       SwiHandleSuspend           10009ddc f   SDKRIL.obj
 0001:00008ecc       ?HandlingResume@@YAXPAX@Z  10009ecc f   SDKRIL.obj
 0001:00008ee8       SwiHandleResume            10009ee8 f   SDKRIL.obj
 0001:00009038       ??0SWISYNCBLOCK@@QAA@PAVCriticalSection@@@Z 1000a038 f i SDKRIL.obj
 0001:00009074       ?Lock@CriticalSection@@QAA_NXZ 1000a074 f i SDKRIL.obj
 0001:000090a4       ??1SWISYNCBLOCK@@QAA@XZ    1000a0a4 f i SDKRIL.obj
 0001:000090c0       ?Unlock@CriticalSection@@QAA_NXZ 1000a0c0 f i SDKRIL.obj
 0001:000090f0       ?IsInitialized@CSwiGobiDll@@QAA_NXZ 1000a0f0 f i SDKRIL.obj
 0001:0000911c       ?IsInitialized@CSwiATPort@@QAAHXZ 1000a11c f i SDKRIL.obj
 0001:00009148       ??0CriticalSection@@QAA@XZ 1000a148 f i SDKRIL.obj
 0001:00009188       ??_GCriticalSection@@UAAPAXI@Z 1000a188 f i SDKRIL.obj
 0001:00009188       ??_ECriticalSection@@UAAPAXI@Z 1000a188 f i SDKRIL.obj
 0001:000091c8       ??1CriticalSection@@UAA@XZ 1000a1c8 f i SDKRIL.obj
 0001:000091f4       ?SendSMSNotify@@YAXPAX@Z   1000a1f4 f   SDKRILCdma.obj
 0001:00009418       SwiGetCDMANetworkParameters 1000a418 f   SDKRILCdma.obj
 0001:000094d4       SwiIsModemReady            1000a4d4 f   SDKRILCdma.obj
 0001:000095dc       SwiGetESN                  1000a5dc f   SDKRILCdma.obj
 0001:00009608       SwiGetESNGobi              1000a608 f   SDKRILCdma.obj
 0001:000097c4       SwiGetRssi                 1000a7c4 f   SDKRILCdma.obj
 0001:00009970       SwiGetChannelNumber        1000a970 f   SDKRILCdma.obj
 0001:00009a98       SwiGetMEIDESN              1000aa98 f   SDKRILCdma.obj
 0001:00009dcc       SwiGetServiceIndication    1000adcc f   SDKRILCdma.obj
 0001:00009fc0       SwiGetRoamingStatus        1000afc0 f   SDKRILCdma.obj
 0001:0000a1c0       SwiGetByteCounter          1000b1c0 f   SDKRILCdma.obj
 0001:0000a350       SwiGetActivationStatus     1000b350 f   SDKRILCdma.obj
 0001:0000a458       SwiSetCallOriginateCmd     1000b458 f   SDKRILCdma.obj
 0001:0000a61c       SwiGetCallConnectionState  1000b61c f   SDKRILCdma.obj
 0001:0000a76c       SwiSetCallDisconnectCmd    1000b76c f   SDKRILCdma.obj
 0001:0000a878       SwiGetCdmaSMSMessageStatus 1000b878 f   SDKRILCdma.obj
 0001:0000a994       SwiRetrieveCdmaSMSMessage  1000b994 f   SDKRILCdma.obj
 0001:0000b0f4       SwiStoreCdmaSMSMessage     1000c0f4 f   SDKRILCdma.obj
 0001:0000b494       SwiSendCdmaSMS             1000c494 f   SDKRILCdma.obj
 0001:0000b788       SwiGetEFileInfo            1000c788 f   SDKRILCdma.obj
 0001:0000ba18       SwiGetEFile                1000ca18 f   SDKRILCdma.obj
 0001:0000bbdc       SwiGetPhoneNumber          1000cbdc f   SDKRILCdma.obj
 0001:0000bd20       SwiGetPRLVersion           1000cd20 f   SDKRILCdma.obj
 0001:0000be14       SwiGetECIO                 1000ce14 f   SDKRILCdma.obj
 0001:0000bea4       SwiResetModem              1000cea4 f   SDKRILCdma.obj
 0001:0000becc       SwiResetByteCounter        1000cecc f   SDKRILCdma.obj
 0001:0000bf58       SwiSetMobileDirNum         1000cf58 f   SDKRILCdma.obj
 0001:0000c150       SwiSetIMSI                 1000d150 f   SDKRILCdma.obj
 0001:0000c418       SwiGetCdmaIMSI             1000d418 f   SDKRILCdma.obj
 0001:0000c658       SwiGetCurrentBaseStation   1000d658 f   SDKRILCdma.obj
 0001:0000c7fc       SwiGetActiveNam            1000d7fc f   SDKRILCdma.obj
 0001:0000c88c       SwiSetPowerDown            1000d88c f   SDKRILCdma.obj
 0001:0000c934       SwiGetTechSID              1000d934 f   SDKRILCdma.obj
 0001:0000ca1c       SwiGetTechNID              1000da1c f   SDKRILCdma.obj
 0001:0000cafc       SwiGetTechBandClass        1000dafc f   SDKRILCdma.obj
 0001:0000cc64       SwiGetTechPowersaveMode    1000dc64 f   SDKRILCdma.obj
 0001:0000ccfc       SwiGetCarrierID            1000dcfc f   SDKRILCdma.obj
 0001:0000d218       SwiGetSystemTime           1000e218 f   SDKRILCdma.obj
 0001:0000d2cc       SwiPstUnlock               1000e2cc f   SDKRILCdma.obj
 0001:0000d424       SwiPstLock                 1000e424 f   SDKRILCdma.obj
 0001:0000d7f8       SwiPstGetSci               1000e7f8 f   SDKRILCdma.obj
 0001:0000d8dc       SwiPstSetSci               1000e8dc f   SDKRILCdma.obj
 0001:0000d9a0       SwiPstGetPrefMode          1000e9a0 f   SDKRILCdma.obj
 0001:0000db60       SwiPstSetPrefMode          1000eb60 f   SDKRILCdma.obj
 0001:0000dc48       SwiPstGetTermHome          1000ec48 f   SDKRILCdma.obj
 0001:0000dd28       SwiPstGetTermSid           1000ed28 f   SDKRILCdma.obj
 0001:0000de0c       SwiPstGetTermNid           1000ee0c f   SDKRILCdma.obj
 0001:0000def0       SwiPstGetAccolc            1000eef0 f   SDKRILCdma.obj
 0001:0000dfe4       SwiPstSetAccolc            1000efe4 f   SDKRILCdma.obj
 0001:0000e110       SwiPstSetCurrentNam        1000f110 f   SDKRILCdma.obj
 0001:0000e1e4       SwiPstGetImsiMcc           1000f1e4 f   SDKRILCdma.obj
 0001:0000e374       SwiPstSetImsiMcc           1000f374 f   SDKRILCdma.obj
 0001:0000e440       SwiPstGetImsi1112          1000f440 f   SDKRILCdma.obj
 0001:0000e5d0       SwiPstSetImsi1112          1000f5d0 f   SDKRILCdma.obj
 0001:0000e694       SwiPstGetSystemPref        1000f694 f   SDKRILCdma.obj
 0001:0000e8f8       SwiPstGetHomeSidNid        1000f8f8 f   SDKRILCdma.obj
 0001:0000eadc       SwiPstSetHomeSidNid        1000fadc f   SDKRILCdma.obj
 0001:0000ec40       SwiGetTechHardwareVersion  1000fc40 f   SDKRILCdma.obj
 0001:0000ec78       SwiPriGetActivationMask    1000fc78 f   SDKRILCdma.obj
 0001:0000ed0c       SwiPriGetMDNLength         1000fd0c f   SDKRILCdma.obj
 0001:0000eda8       SwiPriGetMaxMosmsLen       1000fda8 f   SDKRILCdma.obj
 0001:0000ee38       SwiPstSetDsQcMip           1000fe38 f   SDKRILCdma.obj
 0001:0000eee0       SwiPstGetDsQcMip           1000fee0 f   SDKRILCdma.obj
 0001:0000ef88       SwiPstSetDsMipActiveProf   1000ff88 f   SDKRILCdma.obj
 0001:0000f07c       SwiPstGetDsMipActiveProf   1001007c f   SDKRILCdma.obj
 0001:0000f170       SwiPstSetDsMipGenUser      10010170 f   SDKRILCdma.obj
 0001:0000f338       SwiPstGetDsMipGenUser      10010338 f   SDKRILCdma.obj
 0001:0000f668       SwiPstSetDsMipSsUserProf   10010668 f   SDKRILCdma.obj
 0001:0000f87c       SwiPstGetDsMipSsUserProf   1001087c f   SDKRILCdma.obj
 0001:0000f960       SwiPstGetDsMipEnableProf   10010960 f   SDKRILCdma.obj
 0001:0000fb88       SwiGetMipErrCode           10010b88 f   SDKRILCdma.obj
 0001:0000fca0       SwiSetAKey                 10010ca0 f   SDKRILCdma.obj
 0001:0000fd2c       SwiSetDormant              10010d2c f   SDKRILCdma.obj
 0001:0000fdac       SwiGetRssiEcio             10010dac f   SDKRILCdma.obj
 0001:0000ff9c       SwiGetHdrRoamStatus        10010f9c f   SDKRILCdma.obj
 0001:000101a4       SwiGetHdrSrvState          100111a4 f   SDKRILCdma.obj
 0001:00010398       SwiGetHdrHybrPref          10011398 f   SDKRILCdma.obj
 0001:00010430       SwiSetHdrHybrPref          10011430 f   SDKRILCdma.obj
 0001:00010508       SwiSetTempModePref         10011508 f   SDKRILCdma.obj
 0001:00010900       SwiPstGetHdrUserId         10011900 f   SDKRILCdma.obj
 0001:000109d4       SwiPstSetHdrUserId         100119d4 f   SDKRILCdma.obj
 0001:00010ae0       SwiPstGetHdrPassword       10011ae0 f   SDKRILCdma.obj
 0001:00010bb4       SwiPstSetHdrPassword       10011bb4 f   SDKRILCdma.obj
 0001:00010cc0       SwiPowerSaveExit           10011cc0 f   SDKRILCdma.obj
 0001:00010d24       SwiSetPower                10011d24 f   SDKRILCdma.obj
 0001:00010dd8       SwiGetPower                10011dd8 f   SDKRILCdma.obj
 0001:00010ebc       SwiRtnReset                10011ebc f   SDKRILCdma.obj
 0001:00010fc8       SwiGetNDISMode             10011fc8 f   SDKRILCdma.obj
 0001:00011008       SwiSetNDISPrefMode         10012008 f   SDKRILCdma.obj
 0001:0001106c       SwiGetIOTADisable          1001206c f   SDKRILCdma.obj
 0001:000110fc       SwiGetOMADMConfig          100120fc f   SDKRILCdma.obj
 0001:000112b8       SwiSetOMADMConfig          100122b8 f   SDKRILCdma.obj
 0001:000115dc       SwiStartOMADMSession       100125dc f   SDKRILCdma.obj
 0001:0001175c       SwiCancelOMADMSession      1001275c f   SDKRILCdma.obj
 0001:000118c0       SwiGetOMADMSessionState    100128c0 f   SDKRILCdma.obj
 0001:00011b68       SwiGetOMADMNIAlert         10012b68 f   SDKRILCdma.obj
 0001:00011e2c       SwiSetOMADMNIAlertResponse 10012e2c f   SDKRILCdma.obj
 0001:0001219c       SwiGetGeneralFeatureSupport 1001319c f   SDKRILCdma.obj
 0001:0001222c       SwiActivateAutomatic       1001322c f   SDKRILCdma.obj
 0001:00012374       SwiSetMobileIPProfile      10013374 f   SDKRILCdma.obj
 0001:00012510       SwiGetMobileIPProfile      10013510 f   SDKRILCdma.obj
 0001:000126b0       SwiPstGetDisplayBannerName 100136b0 f   SDKRILCdma.obj
 0001:00012cdc       SwiSetOMAEXEventReport     10013cdc f   SDKRILCdma.obj
 0001:00012d84       SwiOMAEXSessionStart       10013d84 f   SDKRILCdma.obj
 0001:00012e38       SwiOMAEXSessionCancel      10013e38 f   SDKRILCdma.obj
 0001:00012ee0       SwiOMAEXSelection          10013ee0 f   SDKRILCdma.obj
 0001:00012f94       SwiOMAEXGetSettings        10013f94 f   SDKRILCdma.obj
 0001:00013068       SwiOMAEXSetSettings        10014068 f   SDKRILCdma.obj
 0001:0001313c       SwiOMAEXGetSessionInfo     1001413c f   SDKRILCdma.obj
 0001:000131f0       SwiOMAEXInit               100141f0 f   SDKRILCdma.obj
 0001:00013298       SwiOMAEXShutdown           10014298 f   SDKRILCdma.obj
 0001:00013340       ?wcsstr@@YAPAGPAGPBG@Z     10014340 f i SDKRILCdma.obj
 0001:00013374       ?GetPRLSessionID@CSwiNotify@@QAAGXZ 10014374 f i SDKRILCdma.obj
 0001:000133a0       ?GetDCSessionID@CSwiNotify@@QAAGXZ 100143a0 f i SDKRILCdma.obj
 0001:000133cc       ?SetPRLSessionID@CSwiNotify@@QAAXG@Z 100143cc f i SDKRILCdma.obj
 0001:000133ec       ?SetDCSessionID@CSwiNotify@@QAAXG@Z 100143ec f i SDKRILCdma.obj
 0001:00013414       SwiGetNetworkProviderID    10014414 f   SDKRILGsm.obj
 0001:00013624       SwiGetGsmIMSI              10014624 f   SDKRILGsm.obj
 0001:000137f4       SwiGetImei                 100147f4 f   SDKRILGsm.obj
 0001:00013940       SwiGetPLMNMode             10014940 f   SDKRILGsm.obj
 0001:000139c8       SwiSetPLMNMode             100149c8 f   SDKRILGsm.obj
 0001:0001410c       ?GobiPerformNetworkScan@@YAXPAX@Z 1001510c f   SDKRILGsm.obj
 0001:00014684       SwiStartPLMNSearch         10015684 f   SDKRILGsm.obj
 0001:00014784       SwiGetPLMNSelection        10015784 f   SDKRILGsm.obj
 0001:00014bd8       ParseGetUsimRecordStatus   10015bd8 f   SDKRILGsm.obj
 0001:000155d4       SwiSendRestrictedSIMCmd    100165d4 f   SDKRILGsm.obj
 0001:00015fdc       SwiGetSIMRecordStatus      10016fdc f   SDKRILGsm.obj
 0001:00016a68       SwiSendGenericSimCommand   10017a68 f   SDKRILGsm.obj
 0001:0001751c       SwiGetGsmProfileBasic      1001851c f   SDKRILGsm.obj
 0001:00017924       SwiSetGsmProfileBasic      10018924 f   SDKRILGsm.obj
 0001:00017e30       SwiGetProfile              10018e30 f   SDKRILGsm.obj
 0001:00017e9c       SwiSetProfile              10018e9c f   SDKRILGsm.obj
 0001:00017f08       SwiGetProfileSummary       10018f08 f   SDKRILGsm.obj
 0001:00017f74       SwiGetGsmProfileSummary    10018f74 f   SDKRILGsm.obj
 0001:0001800c       SwiActivateProfile         1001900c f   SDKRILGsm.obj
 0001:00018270       SwiGetPhonebookEntry       10019270 f   SDKRILGsm.obj
 0001:000185ac       SwiGetPktSessionStatus     100195ac f   SDKRILGsm.obj
 0001:00018618       SwiGetPktSessionStatusEx   10019618 f   SDKRILGsm.obj
 0001:00018714       SwiGetIPAddress            10019714 f   SDKRILGsm.obj
 0001:000188a8       SwiGetPinStatus            100198a8 f   SDKRILGsm.obj
 0001:00018aa8       SwiGetSimLock              10019aa8 f   SDKRILGsm.obj
 0001:00018b14       SwiGetSimLockGobi          10019b14 f   SDKRILGsm.obj
 0001:00018c98       SwiSetSimLock              10019c98 f   SDKRILGsm.obj
 0001:00018d04       SwiSetSimLockGobi          10019d04 f   SDKRILGsm.obj
 0001:00018eac       SwiSetSimPassword          10019eac f   SDKRILGsm.obj
 0001:00018f18       SwiSetSimPasswordGobi      10019f18 f   SDKRILGsm.obj
 0001:0001938c       SwiGetSimVerifyGobi        1001a38c f   SDKRILGsm.obj
 0001:000195ac       SwiSetSimVerifyGobi        1001a5ac f   SDKRILGsm.obj
 0001:00019820       SwiGetTrafficStatistics    1001a820 f   SDKRILGsm.obj
 0001:00019938       SwiGetSMSMessageStatus     1001a938 f   SDKRILGsm.obj
 0001:00019c54       SwiRetrieveSMSMessageGobi  1001ac54 f   SDKRILGsm.obj
 0001:0001a2b8       SwiRetrieveCBSMSMessageGobi 1001b2b8 f   SDKRILGsm.obj
 0001:0001a4b4       SwiStoreSMSMessageGobi     1001b4b4 f   SDKRILGsm.obj
 0001:0001a6b4       SwiSendSMS                 1001b6b4 f   SDKRILGsm.obj
 0001:0001aabc       SwiGetGsmSMSCAddr          1001babc f   SDKRILGsm.obj
 0001:0001acd8       SwiSetGsmSMSCAddr          1001bcd8 f   SDKRILGsm.obj
 0001:0001ae34       SwiGetPreferredOperatorListGobi 1001be34 f   SDKRILGsm.obj
 0001:0001c0a4       SwiRemovePreferredOperatorGobi 1001d0a4 f   SDKRILGsm.obj
 0001:0001c3a4       SwiAddPreferredOperatorGobi 1001d3a4 f   SDKRILGsm.obj
 0001:0001cbf8       SwiSetHostStartup          1001dbf8 f   SDKRILGsm.obj
 0001:0001cd80       ?SwiGetGsmSystemStatusWithPSAttachedState@@YA?AW4SWI_RCODE@@PAUSWI_STRUCT_GsmSystemStatus@@PAH@Z 1001dd80 f   SDKRILGsm.obj
 0001:0001d570       SwiGetGsmSystemStatus      1001e570 f   SDKRILGsm.obj
 0001:0001d5f4       ??0BerTlv@@QAA@XZ          1001e5f4 f i SDKRILGsm.obj
 0001:0001d654       ??1BerTlv@@QAA@XZ          1001e654 f i SDKRILGsm.obj
 0001:0001d664       ?GetTag@BerTlv@@QAAEXZ     1001e664 f i SDKRILGsm.obj
 0001:0001d68c       ?GetLength@BerTlv@@QAAIXZ  1001e68c f i SDKRILGsm.obj
 0001:0001d6b8       ?GetValue@BerTlv@@QAAPBEXZ 1001e6b8 f i SDKRILGsm.obj
 0001:0001d6e4       ?GetTotalSize@BerTlv@@QAAIXZ 1001e6e4 f i SDKRILGsm.obj
 0001:0001d710       wmemset                    1001e710 f i SDKRILGsm.obj
 0001:0001d774       ?EncodeTeleServiceHdr@@YA?AW4SWI_RCODE@@PAEPAK@Z 1001e774 f   sms.obj
 0001:0001d8e0       ?EncodePrioriyHdr@@YA?AW4SWI_RCODE@@PAEEPAK@Z 1001e8e0 f   sms.obj
 0001:0001da4c       ?EncodeDestAddrHdr@@YA?AW4SWI_RCODE@@PAEPADEPAKE@Z 1001ea4c f   sms.obj
 0001:0001dd38       ?EncodeCallbackNumber@@YA?AW4SWI_RCODE@@PAEPADEPAKE@Z 1001ed38 f   sms.obj
 0001:0001e024       ?EncodeUserDataHdr@@YA?AW4SWI_RCODE@@PAEW4SWI_TYPE_SMS_DataEncodeType@@PADEPAK@Z 1001f024 f   sms.obj
 0001:0001e438       ?EncodeMsgIdenfier@@YA?AW4SWI_RCODE@@PAEEGPAK@Z 1001f438 f   sms.obj
 0001:0001e60c       ?EncodeBearerData@@YA?AW4SWI_RCODE@@PAEEPAK@Z 1001f60c f   sms.obj
 0001:0001e6dc       ?SplitParamMTSms@@YA?AW4SWI_RCODE@@PAEKPAGPAPAE020@Z 1001f6dc f   sms.obj
 0001:0001ec04       ?DecodeBearerData@@YA?AW4SWI_RCODE@@PAEEPAG000000PAPAE002020@Z 1001fc04 f   sms.obj
 0001:0001f510       ?DecodeOriginAddr@@YA?AW4SWI_RCODE@@PAE00PAG0@Z 10020510 f   sms.obj
 0001:0001f73c       ?DecodeCallbackAddr@@YA?AW4SWI_RCODE@@PAE0PAG0@Z 1002073c f   sms.obj
 0001:0001fa0c       ?DecodeUserData@@YA?AW4SWI_RCODE@@PAEE00PAPAE@Z 10020a0c f   sms.obj
 0001:0001ff08       ?DecodeMesagePriority@@YA?AW4SWI_RCODE@@EPAE@Z 10020f08 f   sms.obj
 0001:0001ffa4       ?DecodeCompleteMTSms@@YA?AW4SWI_RCODE@@PAEKPAUSWI_STRUCT_CDMA_SMS_RetrieveSms@@@Z 10020fa4 f   sms.obj
 0001:000208ec       ?ShiftPackedBufferNBitsRight@@YAXPAEKK@Z 100218ec f   sms.obj
 0001:000209a4       ?ShiftPackedBufferNBitsLeft@@YAXPAEKK@Z 100219a4 f   sms.obj
 0001:00020a5c       ?EncodeCompleteMoSms@@YA?AW4SWI_RCODE@@PAPAEPAKPADE2EW4SWI_TYPE_SMS_DataEncodeType@@2EEGE@Z 10021a5c f   sms.obj
 0001:0002157c       ?EncodeMOPDU@@YA?AW4SWI_RCODE@@PAUSWI_STRUCT_GSM_SMS_StoreSmsGobi@@PAEPAG@Z 1002257c f   sms.obj
 0001:00022214       ?TypeofAddr@@YAEW4SWI_TYPE_SMS_Address@@W4SWI_TYPE_SMS_AddressNumbering@@@Z 10023214 f   sms.obj
 0001:00022338       ?DecodeTypeofAddr@@YA?AW4SWI_RCODE@@PAW4SWI_TYPE_SMS_Address@@PAW4SWI_TYPE_SMS_AddressNumbering@@E@Z 10023338 f   sms.obj
 0001:000224a4       ?DecodeAddr@@YA?AW4SWI_RCODE@@PAEE00@Z 100234a4 f   sms.obj
 0001:000225ec       ?CheckIsMultipartMessage@@YAHE@Z 100235ec f   sms.obj
 0001:0002262c       ?CheckIsDeliverMessage@@YA_NE@Z 1002362c f   sms.obj
 0001:0002267c       ?DecodeProtocol@@YA?AW4SWI_RCODE@@EPAW4SWI_TYPE_SMS_Protocol@@PAW4SWI_TYPE_SMS_ProtocolId@@@Z 1002367c f   sms.obj
 0001:000226e0       ?DecodeCodingScheme@@YA?AW4SWI_RCODE@@EPAW4SWI_TYPE_SMS_CodingScheme@@PAW4SWI_TYPE_SMS_CodingClass@@PAW4SWI_TYPE_SMS_CodingCompression@@@Z 100236e0 f   sms.obj
 0001:00022878       ?DecodeTimeStamp@@YA?AW4SWI_RCODE@@PAEE0E@Z 10023878 f   sms.obj
 0001:00022970       ?DecodeCompletePDU@@YA?AW4SWI_RCODE@@PAEKPAUSWI_STRUCT_GSM_SMS_RetrieveSmsGobi@@@Z 10023970 f   sms.obj
 0001:00023544       ?PackAsciiToBits@@YAKPBEKPAEPAH1@Z 10024544 f   sms.obj
 0001:0002369c       ?PackByteToBits@@YAXEQAEGG@Z 1002469c f   sms.obj
 0001:00023988       ?UnpackBitsToAByte@@YAEPAEHH@Z 10024988 f   sms.obj
 0001:00023c1c       ?Char2Num@@YAED@Z          10024c1c f   sms.obj
 0001:00023c5c       ?Num2Char@@YADE@Z          10024c5c f   sms.obj
 0001:00023ca4       ?Hex2Dec@@YAGE@Z           10024ca4 f   sms.obj
 0001:00023d14       ??4CSwiGobiDll@@QAAAAV0@ABV0@@Z 10024d14 f i stdafx.obj
 0001:00023d48       ??0CSwiATPort@@QAA@XZ      10024d48 f   SwiAtPort.obj
 0001:00023d98       ??1CSwiATPort@@QAA@XZ      10024d98 f   SwiAtPort.obj
 0001:00023e44       ?Initialize@CSwiATPort@@QAA?AW4SWI_RCODE@@PBGJDJJHHHHH@Z 10024e44 f   SwiAtPort.obj
 0001:00024700       ?Shutdown@CSwiATPort@@QAA?AW4SWI_RCODE@@XZ 10025700 f   SwiAtPort.obj
 0001:000247e4       ?WaitForResponseTimeout@CSwiATPort@@AAAHPAD0K@Z 100257e4 f   SwiAtPort.obj
 0001:00024d6c       ?WaitForResponse@CSwiATPort@@AAAHPAD0@Z 10025d6c f   SwiAtPort.obj
 0001:00025148       ?ParseNotification@CSwiATPort@@AAAXQBDAAPBDPAH@Z 10026148 f   SwiAtPort.obj
 0001:00025374       ?SendATCommand@CSwiATPort@@QAAHPAD0@Z 10026374 f   SwiAtPort.obj
 0001:00025604       ?SendATCommandTimeout@CSwiATPort@@QAAHPAD0K@Z 10026604 f   SwiAtPort.obj
 0001:00025888       ?ConvertGobiError@@YA?AW4SWI_RCODE@@K@Z 10026888 f   SwiError.obj
 0001:00025a24       ?ConvertGobiCallEndReason@@YA?AW4SWI_TYPE_EndReason@@K@Z 10026a24 f   SwiError.obj
 0001:00025a48       ?ConvertGobi2InactivityReason@@YA?AW4SWI_TYPE_InactivityReason@@K@Z 10026a48 f   SwiError.obj
 0001:00025a6c       ?ExtractOMADMSessionTypeAndInitiator@@YAXKPAW4SWI_TYPE_OMADM_SESSION_TYPE@@PAW4SWI_TYPE_OMADM_SESSION_INITIATOR@@@Z 10026a6c f   SwiError.obj
 0001:00025be0       ?ConvertGobi2OMADMError@@YA?AW4SWI_TYPE_OMADM_SESSION_RESULT@@W4SWI_TYPE_OMADM_SESSION_INITIATOR@@K@Z 10026be0 f   SwiError.obj
 0001:00025d34       ?ConvertGobi2SwiPowerMode@@YA?AW4SWI_TYPE_Power@@K@Z 10026d34 f   SwiError.obj
 0001:00025dd4       ?ConvertSwi2GobiPowerMode@@YA?AW4eGobiPowerMode@@W4SWI_TYPE_Power@@@Z 10026dd4 f   SwiError.obj
 0001:00025e84       ?ConvertGobi2SwiGSMServiceStatus@@YA?AW4SWI_TYPE_ServiceStatus@@K@Z 10026e84 f   SwiError.obj
 0001:00025fa4       ?ConvertGobi2SwiGSMServiceType@@YA?AW4SWI_TYPE_ServiceType@@KK@Z 10026fa4 f   SwiError.obj
 0001:00026020       ?ConvertGobiDataBearer2SwiSystemMode@@YA?AW4SWI_TYPE_Service@@K@Z 10027020 f   SwiError.obj
 0001:0002611c       ?ConvertGobi2SwiNvPrefOpMode@@YA?AW4SWI_TYPE_NvPrefOpMode@@KPAH@Z 1002711c f   SwiError.obj
 0001:00026310       ?ConvertSwi2GobiNvPrefOpMode@@YAKW4SWI_TYPE_NvPrefOpMode@@PAH@Z 10027310 f   SwiError.obj
 0001:00026438       ?ExtractErrorCode@@YAHPBD0PAK@Z 10027438 f   SwiError.obj
 0001:000265f4       ?SwiGetProcAddress@@YAP6AHXZPAUHINSTANCE__@@PBG@Z 100275f4 f   SwiGobiDll.obj
 0001:00026628       ?FindRIfaceIndex@@YAHW4eRadioTech@@EPAE1@Z 10027628 f   SwiGobiDll.obj
 0001:000266cc       ?FindRFInfoIndex@@YAHW4eRadioTech@@EPAURFINFO@@PAE@Z 100276cc f   SwiGobiDll.obj
 0001:00026774       ?BuildDataCapsMask@@YA?AW4eDataCaps@@EPAE@Z 10027774 f   SwiGobiDll.obj
 0001:0002681c       ??0CSwiGobiDll@@QAA@XZ     1002781c f   SwiGobiDll.obj
 0001:00026878       ??1CSwiGobiDll@@QAA@XZ     10027878 f   SwiGobiDll.obj
 0001:00026890       ?Cleanup@CSwiGobiDll@@IAAXXZ 10027890 f   SwiGobiDll.obj
 0001:00027694       ?Initialize@CSwiGobiDll@@QAA_NXZ 10028694 f   SwiGobiDll.obj
 0001:0002a7dc       ?GetDLLVersion@CSwiGobiDll@@QAAKXZ 1002b7dc f   SwiGobiDll.obj
 0001:0002a808       ?Connect@CSwiGobiDll@@QAAKXZ 1002b808 f   SwiGobiDll.obj
 0001:0002a8b0       ?Disconnect@CSwiGobiDll@@QAAKXZ 1002b8b0 f   SwiGobiDll.obj
 0001:0002a918       ?GetWirelessTech@CSwiGobiDll@@QAA?AW4SWI_TYPE_WirelessTech@@XZ 1002b918 f   SwiGobiDll.obj
 0001:0002ad60       ?GetConnectedDeviceID@CSwiGobiDll@@QAAKKPAD@Z 1002bd60 f   SwiGobiDll.obj
 0001:0002adc8       ?GetFirmwareInfo@CSwiGobiDll@@QAAKPAK0000@Z 1002bdc8 f   SwiGobiDll.obj
 0001:0002ae40       ?GetCwePkgsInfo@CSwiGobiDll@@QAAKPAGPAE010101010101@Z 1002be40 f   SwiGobiDll.obj
 0001:0002af00       ?GetSessionState@CSwiGobiDll@@QAAKPAK@Z 1002bf00 f   SwiGobiDll.obj
 0001:0002af64       ?GetDormancyState@CSwiGobiDll@@QAAKPAK@Z 1002bf64 f   SwiGobiDll.obj
 0001:0002afc8       ?GetDunCallInfo@CSwiGobiDll@@QAAKPAKPAE101111PA_KPAG221100002221@Z 1002bfc8 f   SwiGobiDll.obj
 0001:0002b0c8       ?StartDataSession@CSwiGobiDll@@QAAKPAD00PAK1@Z 1002c0c8 f   SwiGobiDll.obj
 0001:0002b178       ?StopDataSession@CSwiGobiDll@@QAAKK@Z 1002c178 f   SwiGobiDll.obj
 0001:0002b1dc       ?GetIPAddress@CSwiGobiDll@@QAAKPAK@Z 1002c1dc f   SwiGobiDll.obj
 0001:0002b240       ?GetPacketStatus@CSwiGobiDll@@QAAKPAK00000@Z 1002c240 f   SwiGobiDll.obj
 0001:0002b2c0       ?SetMobileIP@CSwiGobiDll@@QAAKK@Z 1002c2c0 f   SwiGobiDll.obj
 0001:0002b324       ?GetMobileIP@CSwiGobiDll@@QAAKPAK@Z 1002c324 f   SwiGobiDll.obj
 0001:0002b388       ?SetActiveMobileIPProfile@CSwiGobiDll@@QAAKPADE@Z 1002c388 f   SwiGobiDll.obj
 0001:0002b3f0       ?GetActiveMobileIPProfile@CSwiGobiDll@@QAAKPAE@Z 1002c3f0 f   SwiGobiDll.obj
 0001:0002b454       ?SetMobileIPProfile@CSwiGobiDll@@QAAKPADEPAEPAK22102200@Z 1002c454 f   SwiGobiDll.obj
 0001:0002b504       ?GetMobileIPProfile@CSwiGobiDll@@QAAKEPAEPAK110EPAD11@Z 1002c504 f   SwiGobiDll.obj
 0001:0002b5a4       ?SetMobileIPParameters@CSwiGobiDll@@QAAKPADPAKPAE22222@Z 1002c5a4 f   SwiGobiDll.obj
 0001:0002b634       ?GetMobileIPParameters@CSwiGobiDll@@QAAKPAKPAE11111@Z 1002c634 f   SwiGobiDll.obj
 0001:0002b6bc       ?GetLastMobileIPError@CSwiGobiDll@@QAAKPAK@Z 1002c6bc f   SwiGobiDll.obj
 0001:0002b720       ?GetAutoconnect@CSwiGobiDll@@QAAKPAK@Z 1002c720 f   SwiGobiDll.obj
 0001:0002b784       ?SetAutoconnect@CSwiGobiDll@@QAAKK@Z 1002c784 f   SwiGobiDll.obj
 0001:0002b7e8       ?SetDefaultProfile@CSwiGobiDll@@QAAKKPAK0000PAD111@Z 1002c7e8 f   SwiGobiDll.obj
 0001:0002b8d8       ?GetDefaultProfile@CSwiGobiDll@@QAAKKPAK0000EPADE1E1@Z 1002c8d8 f   SwiGobiDll.obj
 0001:0002b9d8       ?GetByteTotals@CSwiGobiDll@@QAAKPAK0@Z 1002c9d8 f   SwiGobiDll.obj
 0001:0002ba40       ?GetRFInfo@CSwiGobiDll@@QAAKPAE0@Z 1002ca40 f   SwiGobiDll.obj
 0001:0002baa8       ?PerformNetworkScan@CSwiGobiDll@@QAAKPAE0@Z 1002caa8 f   SwiGobiDll.obj
 0001:0002bb10       ?PerformNetworkRATScan@CSwiGobiDll@@QAAKPAE000@Z 1002cb10 f   SwiGobiDll.obj
 0001:0002bb80       ?InitiateNetworkRegistration@CSwiGobiDll@@QAAKKGGK@Z 1002cb80 f   SwiGobiDll.obj
 0001:0002bbf0       ?InitiateDomainAttach@CSwiGobiDll@@QAAKK@Z 1002cbf0 f   SwiGobiDll.obj
 0001:0002bc54       ?GetNetworkPreference@CSwiGobiDll@@QAAKPAK00@Z 1002cc54 f   SwiGobiDll.obj
 0001:0002bcc0       ?SetNetworkPreference@CSwiGobiDll@@QAAKKK@Z 1002ccc0 f   SwiGobiDll.obj
 0001:0002bd28       ?SetCDMANetworkParameters@CSwiGobiDll@@QAAKPADPAE1PAK222@Z 1002cd28 f   SwiGobiDll.obj
 0001:0002bdb0       ?GetCDMANetworkParameters@CSwiGobiDll@@QAAKPAE000000PAK111@Z 1002cdb0 f   SwiGobiDll.obj
 0001:0002be58       ?GetACCOLC@CSwiGobiDll@@QAAKPAE@Z 1002ce58 f   SwiGobiDll.obj
 0001:0002bebc       ?SetACCOLC@CSwiGobiDll@@QAAKPADE@Z 1002cebc f   SwiGobiDll.obj
 0001:0002bf24       ?GetANAAAAuthenticationStatus@CSwiGobiDll@@QAAKPAK@Z 1002cf24 f   SwiGobiDll.obj
 0001:0002bf88       ?GetDeviceCapabilities@CSwiGobiDll@@QAAKPAK0000PAE@Z 1002cf88 f   SwiGobiDll.obj
 0001:0002c008       ?GetFirmwareRevisions@CSwiGobiDll@@QAAKEPADE0E0@Z 1002d008 f   SwiGobiDll.obj
 0001:0002c088       ?GetPRLVersion@CSwiGobiDll@@QAAKPAG@Z 1002d088 f   SwiGobiDll.obj
 0001:0002c0ec       ?Set3Gpp2SubscriptionInfo@CSwiGobiDll@@QAAKPAEPAUMinBasedImsi@@PAUTrueImsi@@00@Z 1002d0ec f   SwiGobiDll.obj
 0001:0002c164       ?Get3Gpp2SubscriptionInfo@CSwiGobiDll@@QAAKPAEPAUMinBasedImsi@@PAUTrueImsi@@00@Z 1002d164 f   SwiGobiDll.obj
 0001:0002c1dc       ?GetERIFile@CSwiGobiDll@@QAAKPAKPAE@Z 1002d1dc f   SwiGobiDll.obj
 0001:0002c244       ?ActivateManual@CSwiGobiDll@@QAAKPADG00KPAE00@Z 1002d244 f   SwiGobiDll.obj
 0001:0002c2d4       ?GetPower@CSwiGobiDll@@QAAKPAK@Z 1002d2d4 f   SwiGobiDll.obj
 0001:0002c338       ?GetOfflineReason@CSwiGobiDll@@QAAKPAK0@Z 1002d338 f   SwiGobiDll.obj
 0001:0002c3a0       ?GetNetworkTime@CSwiGobiDll@@QAAKPA_KPAK@Z 1002d3a0 f   SwiGobiDll.obj
 0001:0002c408       ?ValidateSPC@CSwiGobiDll@@QAAKPAD@Z 1002d408 f   SwiGobiDll.obj
 0001:0002c46c       ?DeleteSMS@CSwiGobiDll@@QAAKKPAK0@Z 1002d46c f   SwiGobiDll.obj
 0001:0002c518       ?GetSMSList@CSwiGobiDll@@QAAKKPAK0PAE@Z 1002d518 f   SwiGobiDll.obj
 0001:0002c5c8       ?GetSMS@CSwiGobiDll@@QAAKKKPAK00PAE@Z 1002d5c8 f   SwiGobiDll.obj
 0001:0002c688       ?ModifySMSStatus@CSwiGobiDll@@QAAKKKK@Z 1002d688 f   SwiGobiDll.obj
 0001:0002c734       ?SaveSMS@CSwiGobiDll@@QAAKKKKPAEPAK@Z 1002d734 f   SwiGobiDll.obj
 0001:0002c7ec       ?SendSMS@CSwiGobiDll@@QAAKKKPAEEPAK@Z 1002d7ec f   SwiGobiDll.obj
 0001:0002c8a4       ?GetSMSCAddress@CSwiGobiDll@@QAAKEPADE0@Z 1002d8a4 f   SwiGobiDll.obj
 0001:0002c954       ?SetSMSCAddress@CSwiGobiDll@@QAAKPAD0@Z 1002d954 f   SwiGobiDll.obj
 0001:0002c9fc       ?SetSMSProtocol@CSwiGobiDll@@QAAKE@Z 1002d9fc f   SwiGobiDll.obj
 0001:0002caa0       ?SetSMSRoute@CSwiGobiDll@@QAAKKPAE@Z 1002daa0 f   SwiGobiDll.obj
 0001:0002cb48       ?SetSMSBroadcastActivation@CSwiGobiDll@@QAAKEE@Z 1002db48 f   SwiGobiDll.obj
 0001:0002cbf0       ?DMSUIMSetPINProtection@CSwiGobiDll@@QAAKKKPADPAK1@Z 1002dbf0 f   SwiGobiDll.obj
 0001:0002cc68       ?UIMGetCardStatus@CSwiGobiDll@@QAAKPAHPAUQMI_UIM_GET_CARD_STATUS_RESP@@@Z 1002dc68 f   SwiGobiDll.obj
 0001:0002ccd0       ?UIMVerifyPIN@CSwiGobiDll@@QAAKPAUQMI_UIM_VERIFY_PIN_REQ_SESSION_INFORMATION@@PAUQMI_UIM_VERIFY_PIN_REQ_VERIFY_PIN@@PAUQMI_UIM_VERIFY_PIN_RESP_RETRIES_REMAINING@@@Z 1002dcd0 f   SwiGobiDll.obj
 0001:0002cd3c       ?UIMUnblockPIN@CSwiGobiDll@@QAAKPAUQMI_UIM_UNBLOCK_PIN_REQ_SESSION_INFORMATION@@PAUQMI_UIM_UNBLOCK_PIN_REQ_UNBLOCK_PIN@@PAUQMI_UIM_UNBLOCK_PIN_RESP_RETRIES_REMAINING@@@Z 1002dd3c f   SwiGobiDll.obj
 0001:0002cda8       ?UIMSetPINProtection@CSwiGobiDll@@QAAKPAUQMI_UIM_SET_PIN_PROTECTION_REQ_SESSION_INFORMATION@@PAUQMI_UIM_SET_PIN_PROTECTION_REQ_SET_PIN_PROTECTION@@PAUQMI_UIM_SET_PIN_PROTECTION_RESP_RETRIES_REMAINING@@@Z 1002dda8 f   SwiGobiDll.obj
 0001:0002ce14       ?UIMChangePIN@CSwiGobiDll@@QAAKPAUQMI_UIM_CHANGE_PIN_REQ_SESSION_INFORMATION@@PAUQMI_UIM_CHANGE_PIN_REQ_CHANGE_PIN@@PAUQMI_UIM_CHANGE_PIN_RESP_RETRIES_REMAINING@@@Z 1002de14 f   SwiGobiDll.obj
 0001:0002ce80       ?DMSUIMVerifyPIN@CSwiGobiDll@@QAAKKPADPAK1@Z 1002de80 f   SwiGobiDll.obj
 0001:0002cef0       ?DMSUIMUnblockPIN@CSwiGobiDll@@QAAKKPAD0PAK1@Z 1002def0 f   SwiGobiDll.obj
 0001:0002cf68       ?DMSUIMChangePIN@CSwiGobiDll@@QAAKKPAD0PAK1@Z 1002df68 f   SwiGobiDll.obj
 0001:0002cfe0       ?DMSUIMGetPINStatus@CSwiGobiDll@@QAAKKPAK00@Z 1002dfe0 f   SwiGobiDll.obj
 0001:0002d050       ?DMSUIMGetICCID@CSwiGobiDll@@QAAKEPAD@Z 1002e050 f   SwiGobiDll.obj
 0001:0002d0b8       ?DMSUIMGetControlKeyStatus@CSwiGobiDll@@QAAKKPAK00@Z 1002e0b8 f   SwiGobiDll.obj
 0001:0002d128       ?DMSUIMSetControlKeyProtection@CSwiGobiDll@@QAAKKKPADPAK@Z 1002e128 f   SwiGobiDll.obj
 0001:0002d198       ?DMSUIMUnblockControlKey@CSwiGobiDll@@QAAKKPADPAK@Z 1002e198 f   SwiGobiDll.obj
 0001:0002d204       ?ResetToFactoryDefaults@CSwiGobiDll@@QAAKPAD@Z 1002e204 f   SwiGobiDll.obj
 0001:0002d268       ?GetPDSState@CSwiGobiDll@@QAAKPAK0@Z 1002e268 f   SwiGobiDll.obj
 0001:0002d2d0       ?SetPDSState@CSwiGobiDll@@QAAKK@Z 1002e2d0 f   SwiGobiDll.obj
 0001:0002d334       ?PDSInjectTimeReference@CSwiGobiDll@@QAAK_KG@Z 1002e334 f   SwiGobiDll.obj
 0001:0002d3a0       ?GetPDSDefaults@CSwiGobiDll@@QAAKPAKPAE00@Z 1002e3a0 f   SwiGobiDll.obj
 0001:0002d410       ?SetPDSDefaults@CSwiGobiDll@@QAAKKEKK@Z 1002e410 f   SwiGobiDll.obj
 0001:0002d480       ?GetXTRAAutomaticDownload@CSwiGobiDll@@QAAKPAKPAG@Z 1002e480 f   SwiGobiDll.obj
 0001:0002d4e8       ?SetXTRAAutomaticDownload@CSwiGobiDll@@QAAKKG@Z 1002e4e8 f   SwiGobiDll.obj
 0001:0002d550       ?GetXTRANetwork@CSwiGobiDll@@QAAKPAK@Z 1002e550 f   SwiGobiDll.obj
 0001:0002d5b4       ?SetXTRANetwork@CSwiGobiDll@@QAAKK@Z 1002e5b4 f   SwiGobiDll.obj
 0001:0002d618       ?GetXTRAValidity@CSwiGobiDll@@QAAKPAG00@Z 1002e618 f   SwiGobiDll.obj
 0001:0002d684       ?SetXTRAValidity@CSwiGobiDll@@QAAKGGG@Z 1002e684 f   SwiGobiDll.obj
 0001:0002d6f0       ?SetXTRAEmbeddedClient@CSwiGobiDll@@QAAKEE@Z 1002e6f0 f   SwiGobiDll.obj
 0001:0002d758       ?SetNMEAConfig@CSwiGobiDll@@QAAKEEEPAG@Z 1002e758 f   SwiGobiDll.obj
 0001:0002d7c8       ?GetNMEAConfig@CSwiGobiDll@@QAAKPAE00PAG@Z 1002e7c8 f   SwiGobiDll.obj
 0001:0002d838       ?ForceXTRADownload@CSwiGobiDll@@QAAKXZ 1002e838 f   SwiGobiDll.obj
 0001:0002d898       ?GetAGPSConfig@CSwiGobiDll@@QAAKPAK0@Z 1002e898 f   SwiGobiDll.obj
 0001:0002d900       ?SetAGPSConfig@CSwiGobiDll@@QAAKKK@Z 1002e900 f   SwiGobiDll.obj
 0001:0002d968       ?GetServiceAutomaticTracking@CSwiGobiDll@@QAAKPAK@Z 1002e968 f   SwiGobiDll.obj
 0001:0002d9cc       ?SetServiceAutomaticTracking@CSwiGobiDll@@QAAKK@Z 1002e9cc f   SwiGobiDll.obj
 0001:0002da30       ?GetPortAutomaticTracking@CSwiGobiDll@@QAAKPAK@Z 1002ea30 f   SwiGobiDll.obj
 0001:0002da94       ?SetPortAutomaticTracking@CSwiGobiDll@@QAAKK@Z 1002ea94 f   SwiGobiDll.obj
 0001:0002daf8       ?ResetPDSData@CSwiGobiDll@@QAAKPAK0@Z 1002eaf8 f   SwiGobiDll.obj
 0001:0002db60       ?GetDataBearerTechnology@CSwiGobiDll@@QAAKPAK@Z 1002eb60 f   SwiGobiDll.obj
 0001:0002dbc4       ?GetSessionDuration@CSwiGobiDll@@QAAKPA_K@Z 1002ebc4 f   SwiGobiDll.obj
 0001:0002dc28       ?GetSignalStrengths@CSwiGobiDll@@QAAKPAKPAC0@Z 1002ec28 f   SwiGobiDll.obj
 0001:0002dce4       ?GetServingNetworkCaps@CSwiGobiDll@@QAAKPAE0@Z 1002ece4 f   SwiGobiDll.obj
 0001:0002dd4c       ?GetConnectionRate@CSwiGobiDll@@QAAKPAK000@Z 1002ed4c f   SwiGobiDll.obj
 0001:0002ddbc       ?GetServingNetwork@CSwiGobiDll@@QAAKPAK000PAE10PAG2EPAD@Z 1002edbc f   SwiGobiDll.obj
 0001:0002de64       ?GetHomeNetwork@CSwiGobiDll@@QAAKPAG0EPAD00@Z 1002ee64 f   SwiGobiDll.obj
 0001:0002dee4       ?GetManufacturer@CSwiGobiDll@@QAAKEPAD@Z 1002eee4 f   SwiGobiDll.obj
 0001:0002df4c       ?GetModelID@CSwiGobiDll@@QAAKEPAD@Z 1002ef4c f   SwiGobiDll.obj
 0001:0002dfb4       ?GetFirmwareRevision@CSwiGobiDll@@QAAKEPAD@Z 1002efb4 f   SwiGobiDll.obj
 0001:0002e01c       ?GetHardwareRevision@CSwiGobiDll@@QAAKEPAD@Z 1002f01c f   SwiGobiDll.obj
 0001:0002e084       ?GetVoiceNumber@CSwiGobiDll@@QAAKEPADE0@Z 1002f084 f   SwiGobiDll.obj
 0001:0002e0f4       ?GetSerialNumbers@CSwiGobiDll@@QAAKEPADE0E0@Z 1002f0f4 f   SwiGobiDll.obj
 0001:0002e174       ?GetIMSI@CSwiGobiDll@@QAAKEPAD@Z 1002f174 f   SwiGobiDll.obj
 0001:0002e1dc       ?UpgradeFirmwareW@CSwiGobiDll@@QAAKPAG@Z 1002f1dc f   SwiGobiDll.obj
 0001:0002e284       ?GetImageStoreW@CSwiGobiDll@@QAAKGPAG@Z 1002f284 f   SwiGobiDll.obj
 0001:0002e2ec       ?GetImageInfoW@CSwiGobiDll@@QAAKPBGPAK1111@Z 1002f2ec f   SwiGobiDll.obj
 0001:0002e36c       ?DisableCallbacks@CSwiGobiDll@@QAAXXZ 1002f36c f   SwiGobiDll.obj
 0001:0002e770       ?SetSessionStateCB@CSwiGobiDll@@SAKP6AXKK@Z@Z 1002f770 f   SwiGobiDll.obj
 0001:0002e828       ?SetDataCapsCB@CSwiGobiDll@@SAKP6AXEPAE@Z@Z 1002f828 f   SwiGobiDll.obj
 0001:0002e888       ?SetByteTotalsCB@CSwiGobiDll@@SAKP6AX_K0@ZE@Z 1002f888 f   SwiGobiDll.obj
 0001:0002e8ec       ?SetDataBearerCB@CSwiGobiDll@@SAKP6AXK@Z@Z 1002f8ec f   SwiGobiDll.obj
 0001:0002e94c       ?SetDormancyStatusCB@CSwiGobiDll@@SAKP6AXK@Z@Z 1002f94c f   SwiGobiDll.obj
 0001:0002e9ac       ?SetMobileIPStatusCB@CSwiGobiDll@@SAKP6AXK@Z@Z 1002f9ac f   SwiGobiDll.obj
 0001:0002ea0c       ?SetActivationStatusCB@CSwiGobiDll@@SAKP6AXK@Z@Z 1002fa0c f   SwiGobiDll.obj
 0001:0002ea6c       ?SetPowerCB@CSwiGobiDll@@SAKP6AXK@Z@Z 1002fa6c f   SwiGobiDll.obj
 0001:0002eacc       ?SetRoamingIndicatorCB@CSwiGobiDll@@SAKP6AXK@Z@Z 1002facc f   SwiGobiDll.obj
 0001:0002eb2c       ?SetSignalStrengthCB@CSwiGobiDll@@SAKP6AXCK@ZEPAC@Z 1002fb2c f   SwiGobiDll.obj
 0001:0002eb94       ?SetRFInfoCB@CSwiGobiDll@@SAKP6AXKKK@Z@Z 1002fb94 f   SwiGobiDll.obj
 0001:0002ebf4       ?SetNewSMSCB@CSwiGobiDll@@SAKP6AXKK@Z@Z 1002fbf4 f   SwiGobiDll.obj
 0001:0002ec54       ?SetNewSMSCBCB@CSwiGobiDll@@SAKP6AXEKEGPAE@Z@Z 1002fc54 f   SwiGobiDll.obj
 0001:0002ecb4       ?SetVoiceMessageCB@CSwiGobiDll@@SAKP6AXEPAE00@Z@Z 1002fcb4 f   SwiGobiDll.obj
 0001:0002ed58       ?SetPhonebookRecordReadCB@CSwiGobiDll@@SAKP6AXEGPAUarrPBInfo@@@Z@Z 1002fd58 f   SwiGobiDll.obj
 0001:0002edb8       ?SetNITZCB@CSwiGobiDll@@SAKP6AXGEEEEEEEE@Z@Z 1002fdb8 f   SwiGobiDll.obj
 0001:0002ee18       ?SetEmergencyModeCB@CSwiGobiDll@@SAKP6AXPAE@Z@Z 1002fe18 f   SwiGobiDll.obj
 0001:0002ee78       ?SetOMADMStateCB@CSwiGobiDll@@SAKP6AXKK@Z@Z 1002fe78 f   SwiGobiDll.obj
 0001:0002eed8       ?SetOMADMAlertCB@CSwiGobiDll@@SAKP6AXKG@Z@Z 1002fed8 f   SwiGobiDll.obj
 0001:0002ef38       ?SetDeviceRemovalCallback@CSwiGobiDll@@QAAKP6AXK@Z@Z 1002ff38 f   SwiGobiDll.obj
 0001:0002efec       ?SetPower@CSwiGobiDll@@QAAKK@Z 1002ffec f   SwiGobiDll.obj
 0001:0002f0ac       ?ActivateAutomatic@CSwiGobiDll@@QAAKPAD@Z 100300ac f   SwiGobiDll.obj
 0001:0002f1ac       ?GetActivationState@CSwiGobiDll@@QAAKPAK@Z 100301ac f   SwiGobiDll.obj
 0001:0002f260       ?OMADMGetFeatureSettings@CSwiGobiDll@@QAAKPAK0@Z 10030260 f   SwiGobiDll.obj
 0001:0002f318       ?OMADMGetSessionInfo@CSwiGobiDll@@QAAKPAK00PAEPAG2@Z 10030318 f   SwiGobiDll.obj
 0001:0002f3e8       ?OMADMSetProvisioningFeature@CSwiGobiDll@@QAAKK@Z 100303e8 f   SwiGobiDll.obj
 0001:0002f49c       ?OMADMSetPRLUpdateFeature@CSwiGobiDll@@QAAKK@Z 1003049c f   SwiGobiDll.obj
 0001:0002f550       ?OMADMStartSession@CSwiGobiDll@@QAAKK@Z 10030550 f   SwiGobiDll.obj
 0001:0002f604       ?OMADMCancelSession@CSwiGobiDll@@QAAKXZ 10030604 f   SwiGobiDll.obj
 0001:0002f6b4       ?OMADMGetPendingNIA@CSwiGobiDll@@QAAKPAKPAG@Z 100306b4 f   SwiGobiDll.obj
 0001:0002f76c       ?OMADMSendSelection@CSwiGobiDll@@QAAKKG@Z 1003076c f   SwiGobiDll.obj
 0001:0002f824       ?GetIPConfiguration@CSwiGobiDll@@QAAKPAK0000@Z 10030824 f   SwiGobiDll.obj
 0001:0002f8ec       ?OMAEXSetEventReport@CSwiGobiDll@@QAAKXZ 100308ec f   SwiGobiDll.obj
 0001:0002f99c       ?OMAEXSessionStart@CSwiGobiDll@@QAAKPAE@Z 1003099c f   SwiGobiDll.obj
 0001:0002fa50       ?OMAEXSessionCancel@CSwiGobiDll@@QAAKXZ 10030a50 f   SwiGobiDll.obj
 0001:0002fb00       ?OMAEXSelection@CSwiGobiDll@@QAAKPAE@Z 10030b00 f   SwiGobiDll.obj
 0001:0002fbb4       ?OMAEXGetSettings@CSwiGobiDll@@QAAKPAE00000@Z 10030bb4 f   SwiGobiDll.obj
 0001:0002fc84       ?OMAEXSetSettings@CSwiGobiDll@@QAAKPAE00000@Z 10030c84 f   SwiGobiDll.obj
 0001:0002fd54       ?OMAEXSessionGetInfo@CSwiGobiDll@@QAAKPAUomaSessionInfo@@@Z 10030d54 f   SwiGobiDll.obj
 0001:0002fe08       ?OMAEXInit@CSwiGobiDll@@QAAKXZ 10030e08 f   SwiGobiDll.obj
 0001:0002feb8       ?OMAEXShutdown@CSwiGobiDll@@QAAKXZ 10030eb8 f   SwiGobiDll.obj
 0001:0002ff68       ?GetImagePreference@CSwiGobiDll@@QAAKPAKPAE@Z 10030f68 f   SwiGobiDll.obj
 0001:0002ffd0       ?SetImagePreference@CSwiGobiDll@@QAAKKPAEKEPAK0@Z 10030fd0 f   SwiGobiDll.obj
 0001:00030050       ?GetAudioProfile@CSwiGobiDll@@QAAKPAE@Z 10031050 f   SwiGobiDll.obj
 0001:0003012c       ?SetAudioProfile@CSwiGobiDll@@QAAKPAE@Z 1003112c f   SwiGobiDll.obj
 0001:00030260       ?SetMICMuteStatus@CSwiGobiDll@@QAAKPAE@Z 10031260 f   SwiGobiDll.obj
 0001:000303a0       ?SetSpeakerMuteStatus@CSwiGobiDll@@QAAKPAE@Z 100313a0 f   SwiGobiDll.obj
 0001:000304d4       ?SetReceiverVolume@CSwiGobiDll@@QAAKPAE@Z 100314d4 f   SwiGobiDll.obj
 0001:00030608       ?SetMicVolume@CSwiGobiDll@@QAAKPAG@Z 10031608 f   SwiGobiDll.obj
 0001:00030774       ?GetMicVolume@CSwiGobiDll@@QAAKPAG@Z 10031774 f   SwiGobiDll.obj
 0001:0003088c       ?SetEchoCancelMode@CSwiGobiDll@@QAAKPAE@Z 1003188c f   SwiGobiDll.obj
 0001:000309f8       ?GetEchoCancelMode@CSwiGobiDll@@QAAKPAE@Z 100319f8 f   SwiGobiDll.obj
 0001:00030b10       ?SetNoiseSuppression@CSwiGobiDll@@QAAKPAE@Z 10031b10 f   SwiGobiDll.obj
 0001:00030c7c       ?GetNoiseSuppression@CSwiGobiDll@@QAAKPAE@Z 10031c7c f   SwiGobiDll.obj
 0001:00030d94       ?SetAutoOutputGain@CSwiGobiDll@@QAAKPAE@Z 10031d94 f   SwiGobiDll.obj
 0001:00030f00       ?GetAutoOutputGain@CSwiGobiDll@@QAAKPAE@Z 10031f00 f   SwiGobiDll.obj
 0001:00031018       ?SetAutoInputGain@CSwiGobiDll@@QAAKPAE@Z 10032018 f   SwiGobiDll.obj
 0001:00031184       ?GetAutoInputGain@CSwiGobiDll@@QAAKPAE@Z 10032184 f   SwiGobiDll.obj
 0001:0003129c       ?SetTXPCMFilter@CSwiGobiDll@@QAAKPAG0PAK0@Z 1003229c f   SwiGobiDll.obj
 0001:00031408       ?GetTXPCMFilter@CSwiGobiDll@@QAAKPAG0PAK0@Z 10032408 f   SwiGobiDll.obj
 0001:00031534       ?SetRXPCMFilter@CSwiGobiDll@@QAAKPAG0PAK0@Z 10032534 f   SwiGobiDll.obj
 0001:000316a0       ?GetRXPCMFilter@CSwiGobiDll@@QAAKPAG0PAK0@Z 100326a0 f   SwiGobiDll.obj
 0001:000317cc       ?SetRXGainLevel@CSwiGobiDll@@QAAKPAEPAG1@Z 100327cc f   SwiGobiDll.obj
 0001:00031918       ?SetSideToneGain@CSwiGobiDll@@QAAKPAG@Z 10032918 f   SwiGobiDll.obj
 0001:00031a84       ?GetSideToneGain@CSwiGobiDll@@QAAKPAG@Z 10032a84 f   SwiGobiDll.obj
 0001:00031b9c       ?PlayAudioTone@CSwiGobiDll@@QAAKPAE@Z 10032b9c f   SwiGobiDll.obj
 0001:00031cb4       ?OrigUSSD@CSwiGobiDll@@QAAKPAUUSSInfo@@PAGPAUalphaIDInfo@@0PAE3PAUccSUPSType@@@Z 10032cb4 f   SwiGobiDll.obj
 0001:00031d3c       ?AnswerUSSD@CSwiGobiDll@@QAAKPAUUSSInfo@@@Z 10032d3c f   SwiGobiDll.obj
 0001:00031da0       ?CancelUSSD@CSwiGobiDll@@QAAKXZ 10032da0 f   SwiGobiDll.obj
 0001:00031e00       ?ChangeBarringPwd@CSwiGobiDll@@QAAKPAUcallBarringPwd@@PAGPAUalphaIDInfo@@PAE3PAUccSUPSType@@@Z 10032e00 f   SwiGobiDll.obj
 0001:00031e80       ?DialCall@CSwiGobiDll@@QAAKPAUtDialReqParam@@PAEPAUalphaIDInfo@@1PAUccSUPSType@@@Z 10032e80 f   SwiGobiDll.obj
 0001:00031ef8       ?EndCall@CSwiGobiDll@@QAAKPAE0@Z 10032ef8 f   SwiGobiDll.obj
 0001:00031f60       ?AnserCall@CSwiGobiDll@@QAAKPAE0@Z 10032f60 f   SwiGobiDll.obj
 0001:00031fc8       ?SetCallInfoCB@CSwiGobiDll@@SAKP6AXPAUarrCallInfo@@PAUarrRemotePartyNum@@PAUarrRemotePartyName@@PAUarrAlertingType@@PAUarrSvcOption@@PAUarrCallEndReason@@PAUarrAlphaIDInfo@@PAUarrPeerNumInfo@@PAUarrDiagInfo@@77PAUarrAlertingPattern@@@Z@Z 10032fc8 f   SwiGobiDll.obj
 0001:00032028       ?SetInfoRecCB@CSwiGobiDll@@SAKP6AXPAEPAUsignalInfo@@PAUcallerIDInfo@@PAD330PAUpeerNumInfo@@44PAUredirectNumInfo@@0000PAUlineCtlInfo@@PAUextDisplayInfo@@@Z@Z 10033028 f   SwiGobiDll.obj
 0001:00032088       ?SetUSSDInfoCB@CSwiGobiDll@@SAKP6AXPAEPAUUSSInfo@@@Z@Z 10033088 f   SwiGobiDll.obj
 0001:000320e8       ?SetAllPbInitDoneCB@CSwiGobiDll@@SAKP6AXEPAEPAG@Z@Z 100330e8 f   SwiGobiDll.obj
 0001:0003218c       ?SetEmergencyListCB@CSwiGobiDll@@SAKP6AXEPAUemergencyNumberEntry@@@Z@Z 1003318c f   SwiGobiDll.obj
 0001:00032230       ?SetOMAEXEventCB@CSwiGobiDll@@SAKP6AXPAUFUMOInfo@@PAUOMAInfo@@@Z@Z 10033230 f   SwiGobiDll.obj
 0001:000322d4       ?ManageCalls@CSwiGobiDll@@QAAKPAE0PAG@Z 100332d4 f   SwiGobiDll.obj
 0001:00032340       ?GetCLIR@CSwiGobiDll@@QAAKPAUstatusResp@@PAGPAUalphaIDInfo@@PAE3PAUccSUPSType@@@Z 10033340 f   SwiGobiDll.obj
 0001:000323c0       ?GetCallWaiting@CSwiGobiDll@@QAAKPAE0PAGPAUalphaIDInfo@@00PAUccSUPSType@@@Z 100333c0 f   SwiGobiDll.obj
 0001:00032448       ?SetSUPS@CSwiGobiDll@@QAAKPAUvoiceSetSUPSServiceReq@@PAGPAUalphaIDInfo@@PAE3PAUccSUPSType@@@Z 10033448 f   SwiGobiDll.obj
 0001:000324c8       ?GetCallBarring@CSwiGobiDll@@QAAKPAE00PAGPAUalphaIDInfo@@00PAUccSUPSType@@@Z 100334c8 f   SwiGobiDll.obj
 0001:00032558       ?GetCallForwarding@CSwiGobiDll@@QAAKPAE0PAUgetCallFWInfo@@0PAUalphaIDInfo@@00PAUccSUPSType@@PAUgetExtCallFWInfo@@@Z 10033558 f   SwiGobiDll.obj
 0001:000325f0       ?GetAllCallInfo@CSwiGobiDll@@QAAKPAUarrCallInfo@@PAUarrRemotePartyNum@@PAUarrRemotePartyName@@PAUarrAlertingType@@PAUarrUUSInfo@@PAUarrSvcOption@@PAE6PAUarrCallEndReason@@PAUarrAlphaIDInfo@@PAUarrPeerNumInfo@@PAUarrDiagInfo@@99PAUarrAlertingPattern@@@Z 100335f0 f   SwiGobiDll.obj
 0001:000326b8       ?SendFlash@CSwiGobiDll@@QAAKPAEPAD00@Z 100336b8 f   SwiGobiDll.obj
 0001:00032728       ?StartDTMF@CSwiGobiDll@@QAAKPAE00@Z 10033728 f   SwiGobiDll.obj
 0001:00032794       ?StopDTMF@CSwiGobiDll@@QAAKPAE0@Z 10033794 f   SwiGobiDll.obj
 0001:000327fc       ?GetPhonebookCapabilities@CSwiGobiDll@@QAAKPAEPAG1100@Z 100337fc f   SwiGobiDll.obj
 0001:0003287c       ?ReadPhonebookRecords@CSwiGobiDll@@QAAKPAEPAG111@Z 1003387c f   SwiGobiDll.obj
 0001:000328f4       ?WritePhonebookRecord@CSwiGobiDll@@QAAKPAEPAG1000000@Z 100338f4 f   SwiGobiDll.obj
 0001:0003298c       ?DeletePhonebookRecord@CSwiGobiDll@@QAAKPAEPAG1@Z 1003398c f   SwiGobiDll.obj
 0001:000329f8       ?GetCellLocationInfo@CSwiGobiDll@@QAAKPAUgeranCellInfo@@PAUumtsCellInfo@@PAUcdmaCellInfo@@PAK@Z 100339f8 f   SwiGobiDll.obj
 0001:00032aac       ?GetWaitingMessage@CSwiGobiDll@@QAAKPAUwaitingMsgInfo@@@Z 10033aac f   SwiGobiDll.obj
 0001:00032b54       ?GetRTREConfig@CSwiGobiDll@@QAAKPAE0@Z 10033b54 f   SwiGobiDll.obj
 0001:00032c00       ?SwiM2MAV_AudioGetProfile@CSwiGobiDll@@QAAKPAE000000@Z 10033c00 f   SwiGobiDll.obj
 0001:00032c88       ?SwiM2MAV_AudioSetProfile@CSwiGobiDll@@QAAKPAE00000@Z 10033c88 f   SwiGobiDll.obj
 0001:00032d08       ?SwiM2MAV_AudioGetVolume@CSwiGobiDll@@QAAKPAE00@Z 10033d08 f   SwiGobiDll.obj
 0001:00032d74       ?SwiM2MAV_AudioSetVolume@CSwiGobiDll@@QAAKPAE00@Z 10033d74 f   SwiGobiDll.obj
 0001:00032de0       ?SwiM2MAV_AudioGetAVMute@CSwiGobiDll@@QAAKPAE000@Z 10033de0 f   SwiGobiDll.obj
 0001:00032e50       ?SwiM2MAV_AudioSetAVMute@CSwiGobiDll@@QAAKPAE000@Z 10033e50 f   SwiGobiDll.obj
 0001:00032ec0       ?SwiM2MAV_AudioGetAVCFG@CSwiGobiDll@@QAAKPAUAudioConfig@@PAE@Z 10033ec0 f   SwiGobiDll.obj
 0001:00032f28       ?SwiM2MAV_AudioSetAVCFG@CSwiGobiDll@@QAAKPAE00PAUPIFACETable@@@Z 10033f28 f   SwiGobiDll.obj
 0001:00032f98       ?SwiM2MAV_AudioNVDef@CSwiGobiDll@@QAAKXZ 10033f98 f   SwiGobiDll.obj
 0001:00032ff8       ?SwiM2MAV_AudioSetLPBK@CSwiGobiDll@@QAAKPAE@Z 10033ff8 f   SwiGobiDll.obj
 0001:0003305c       ?SwiM2MAV_AudioGetSpeakerGain@CSwiGobiDll@@QAAKPAEPAG@Z 1003405c f   SwiGobiDll.obj
 0001:000330c4       ?SwiM2MAV_AudioSetSpeakerGain@CSwiGobiDll@@QAAKPAEPAG@Z 100340c4 f   SwiGobiDll.obj
 0001:0003312c       ?SwiM2MAV_AudioGetSTG@CSwiGobiDll@@QAAKPAEPAG@Z 1003412c f   SwiGobiDll.obj
 0001:00033194       ?SwiM2MAV_AudioSetSTG@CSwiGobiDll@@QAAKPAEPAG@Z 10034194 f   SwiGobiDll.obj
 0001:000331fc       ?SwiM2MAV_AudioGetTxVolume@CSwiGobiDll@@QAAKPAEPAG@Z 100341fc f   SwiGobiDll.obj
 0001:00033264       ?SwiM2MAV_AudioSetTxVolume@CSwiGobiDll@@QAAKPAEPAG@Z 10034264 f   SwiGobiDll.obj
 0001:000332cc       ?SwiM2MAV_AudioGetMicGain@CSwiGobiDll@@QAAKPAEPAG@Z 100342cc f   SwiGobiDll.obj
 0001:00033334       ?SwiM2MAV_AudioSetMicGain@CSwiGobiDll@@QAAKPAEPAG@Z 10034334 f   SwiGobiDll.obj
 0001:0003339c       ?SwiM2MAV_AudioGetVolDB@CSwiGobiDll@@QAAKPAE00PAG@Z 1003439c f   SwiGobiDll.obj
 0001:0003340c       ?SwiM2MAV_AudioSetVolDB@CSwiGobiDll@@QAAKPAE00PAG@Z 1003440c f   SwiGobiDll.obj
 0001:0003347c       ?SwiM2MAV_AudioGetAVTXG@CSwiGobiDll@@QAAKPAEPAG@Z 1003447c f   SwiGobiDll.obj
 0001:000334e4       ?SwiM2MAV_AudioSetAVTXG@CSwiGobiDll@@QAAKPAEPAG@Z 100344e4 f   SwiGobiDll.obj
 0001:0003354c       ?SwiM2MAV_AudioGetAVRXG@CSwiGobiDll@@QAAKPAEPAG@Z 1003454c f   SwiGobiDll.obj
 0001:000335b4       ?SwiM2MAV_AudioSetAVRXG@CSwiGobiDll@@QAAKPAEPAG@Z 100345b4 f   SwiGobiDll.obj
 0001:0003361c       ?SwiM2MAV_AudioGetAVEC@CSwiGobiDll@@QAAKPAE0@Z 1003461c f   SwiGobiDll.obj
 0001:00033684       ?SwiM2MAV_AudioSetAVEC@CSwiGobiDll@@QAAKPAE0@Z 10034684 f   SwiGobiDll.obj
 0001:000336ec       ?SwiM2MAV_AudioGetAVNS@CSwiGobiDll@@QAAKPAE0@Z 100346ec f   SwiGobiDll.obj
 0001:00033754       ?SwiM2MAV_AudioSetAVNS@CSwiGobiDll@@QAAKPAE0@Z 10034754 f   SwiGobiDll.obj
 0001:000337bc       ?SwiM2MAV_AudioPlayTone@CSwiGobiDll@@QAAKPAE0PAG@Z 100347bc f   SwiGobiDll.obj
 0001:00033828       ?GenericCallStateChanged@@YAXXZ 10034828 f   SwiNotify.obj
 0001:0003382c       ?GenericSmsSendStatusChanged@@YAXXZ 1003482c f   SwiNotify.obj
 0001:00033830       ?GenericPlmnModeChanged@@YAXXZ 10034830 f   SwiNotify.obj
 0001:00033834       ?GenericPlmnAvailableChanged@@YAXXZ 10034834 f   SwiNotify.obj
 0001:00033838       ?GenericPlmnReadyChanged@@YAXXZ 10034838 f   SwiNotify.obj
 0001:0003383c       ?GenericPhonebookReadyChanged@@YAXXZ 1003483c f   SwiNotify.obj
 0001:00033840       ?OMAEXEventCallback@CSwiNotify@@SAXPAUFUMOInfo@@PAUOMAInfo@@@Z 10034840 f   SwiNotify.obj
 0001:00033968       ?CallInfoCallback@CSwiNotify@@SAXPAUarrCallInfo@@PAUarrRemotePartyNum@@PAUarrRemotePartyName@@PAUarrAlertingType@@PAUarrSvcOption@@PAUarrCallEndReason@@PAUarrAlphaIDInfo@@PAUarrPeerNumInfo@@PAUarrDiagInfo@@77PAUarrAlertingPattern@@@Z 10034968 f   SwiNotify.obj
 0001:000342e0       ?InfoRecCallback@CSwiNotify@@SAXPAEPAUsignalInfo@@PAUcallerIDInfo@@PAD330PAUpeerNumInfo@@44PAUredirectNumInfo@@0000PAUlineCtlInfo@@PAUextDisplayInfo@@@Z 100352e0 f   SwiNotify.obj
 0001:00034698       ?USSDCallback@CSwiNotify@@SAXPAEPAUUSSInfo@@@Z 10035698 f   SwiNotify.obj
 0001:00034894       ?ReadSIMPhoneBookCallback@CSwiNotify@@SAXEGPAUarrPBInfo@@@Z 10035894 f   SwiNotify.obj
 0001:00034d60       ?AllSIMPhonebookInitDoneCallback@CSwiNotify@@SAXEPAEPAG@Z 10035d60 f   SwiNotify.obj
 0001:00034e20       ?EmergencyListCallback@CSwiNotify@@SAXEPAUemergencyNumberEntry@@@Z 10035e20 f   SwiNotify.obj
 0001:00035234       ?NetworkIdentityAndTimeZoneCallback@@YAXGEEEEEEEE@Z 10036234 f   SwiNotify.obj
 0001:00035314       ?EmergencyModeCallback@@YAXPAE@Z 10036314 f   SwiNotify.obj
 0001:000353f4       ?SessionStateCallback@CSwiNotify@@SAXKK@Z 100363f4 f   SwiNotify.obj
 0001:000354e0       ?DataBearerCallback@@YAXK@Z 100364e0 f   SwiNotify.obj
 0001:000354f0       ?DormancyStatusCallback@@YAXK@Z 100364f0 f   SwiNotify.obj
 0001:00035544       ?SetMobileIPStatusCallback@@YAXK@Z 10036544 f   SwiNotify.obj
 0001:0003555c       ?ActivationStatusCallback@CSwiNotify@@SAXK@Z 1003655c f   SwiNotify.obj
 0001:000355fc       ?GobiAPIPowerCallback@@YAXK@Z 100365fc f   SwiNotify.obj
 0001:000356a8       ?PowerCallback@CSwiNotify@@SAXPAX@Z 100366a8 f   SwiNotify.obj
 0001:00035750       ?GobiAPIRoamingIndicatorCallback@@YAXK@Z 10036750 f   SwiNotify.obj
 0001:000357fc       ?RoamingIndicatorCallback@CSwiNotify@@SAXPAX@Z 100367fc f   SwiNotify.obj
 0001:000358a4       ?GobiAPISignalStrengthCallback@@YAXCK@Z 100368a4 f   SwiNotify.obj
 0001:00035974       ?SignalStrengthCallback@CSwiNotify@@SAXPAX@Z 10036974 f   SwiNotify.obj
 0001:00035a28       ?GobiAPIRFinfoCallback@@YAXKKK@Z 10036a28 f   SwiNotify.obj
 0001:00035a90       ?RFinfoCallback@CSwiNotify@@SAXK@Z 10036a90 f   SwiNotify.obj
 0001:00035b74       ?NewSMSCallback@@YAXKK@Z   10036b74 f   SwiNotify.obj
 0001:00035d0c       ?NewSMSCBCallback@@YAXEKEGPAE@Z 10036d0c f   SwiNotify.obj
 0001:00035db4       ?VoiceMessageCallback@@YAXEPAE00@Z 10036db4 f   SwiNotify.obj
 0001:00036018       ?GobiAPIDataCapabilities@@YAXEPAE@Z 10037018 f   SwiNotify.obj
 0001:00036158       ?ByteTotalsCallback@CSwiNotify@@SAX_K0@Z 10037158 f   SwiNotify.obj
 0001:00036268       ?GobiAPIOMADMStateCallback@@YAXKK@Z 10037268 f   SwiNotify.obj
 0001:000362c8       ?GobiAPIOMADMAlertCallback@@YAXKG@Z 100372c8 f   SwiNotify.obj
 0001:000363d8       ?OMADMStateCallback@CSwiNotify@@SAXK@Z 100373d8 f   SwiNotify.obj
 0001:000364c4       ?OMADMAlertCallback@CSwiNotify@@SAXPAX@Z 100374c4 f   SwiNotify.obj
 0001:000365bc       ??0CSwiNotify@@QAA@XZ      100375bc f   SwiNotify.obj
 0001:00036634       ?RemoveAll@CSwiNotify@@QAAXXZ 10037634 f   SwiNotify.obj
 0001:00036828       ??1CSwiNotify@@QAA@XZ      10037828 f   SwiNotify.obj
 0001:00036868       ?RegisterCallback@CSwiNotify@@QAAXP6AXPAUSwiNotifyVariant@@@ZPAVCSwiGobiDll@@@Z 10037868 f   SwiNotify.obj
 0001:000368bc       ?DeregisterCallback@CSwiNotify@@QAAXP6AXPAUSwiNotifyVariant@@@Z@Z 100378bc f   SwiNotify.obj
 0001:00036918       ?LocateCallbackFn@CSwiNotify@@QAAHW4SWI_TYPE_Notify@@W4eCBAdminOperation@@PAHPAK@Z 10037918 f   SwiNotify.obj
 0001:00037254       ?Add@CSwiNotify@@QAA?AW4SWI_RCODE@@W4SWI_TYPE_Notify@@K@Z 10038254 f   SwiNotify.obj
 0001:00037b74       ?Remove@CSwiNotify@@QAA?AW4SWI_RCODE@@W4SWI_TYPE_Notify@@K@Z 10038b74 f   SwiNotify.obj
 0001:00038150       ?HandleSignalStrengthCallback@CSwiNotify@@QAAHPAXCK@Z 10039150 f   SwiNotify.obj
 0001:000392d0       ?HandleSessionStateCallback@CSwiNotify@@QAAHPAXKK@Z 1003a2d0 f   SwiNotify.obj
 0001:00039a60       ?HandleRoamingIndicatorCallback@CSwiNotify@@QAAHPAXK@Z 1003aa60 f   SwiNotify.obj
 0001:0003a470       ?HandlePowerCallback@CSwiNotify@@QAAHPAXK@Z 1003b470 f   SwiNotify.obj
 0001:0003a9f8       ?HandleActivationStatusCallback@CSwiNotify@@QAAHPAXK@Z 1003b9f8 f   SwiNotify.obj
 0001:0003aec4       ?HandleOMADMStateCallback@CSwiNotify@@QAAHPAXK@Z 1003bec4 f   SwiNotify.obj
 0001:0003b37c       ?HandleOMADMAlertCallback@CSwiNotify@@QAAHPAX@Z 1003c37c f   SwiNotify.obj
 0001:0003b884       ?HandleByteTotalsCallback@CSwiNotify@@QAAHPAX_K1@Z 1003c884 f   SwiNotify.obj
 0001:0003bd40       ?HandleRFinfoCallback@CSwiNotify@@QAAHPAXK@Z 1003cd40 f   SwiNotify.obj
 0001:0003c194       ?HandleSuspend@CSwiNotify@@QAAXXZ 1003d194 f   SwiNotify.obj
 0001:0003c450       ?HandleResume@CSwiNotify@@QAAXXZ 1003d450 f   SwiNotify.obj
 0001:0003c700       ?GetMySelf@CSwiNotify@@SAPAV1@XZ 1003d700 f i SwiNotify.obj
 0001:0003c720       ?GetGobi@CSwiNotify@@SAPAVCSwiGobiDll@@XZ 1003d720 f i SwiNotify.obj
 0001:0003c740       ??1?$_Iterator@$00@?$list@UszCallbackItem@@V?$allocator@UszCallbackItem@@@std@@@std@@QAA@XZ 1003d740 f i SwiNotify.obj
 0001:0003c758       ??4?$_Iterator@$00@?$list@UszCallbackItem@@V?$allocator@UszCallbackItem@@@std@@@std@@QAAAAV012@ABV012@@Z 1003d758 f i SwiNotify.obj
 0001:0003c788       ??1?$_Const_iterator@$00@?$list@UszCallbackItem@@V?$allocator@UszCallbackItem@@@std@@@std@@QAA@XZ 1003d788 f i SwiNotify.obj
 0001:0003c7a0       ??4?$_Const_iterator@$00@?$list@UszCallbackItem@@V?$allocator@UszCallbackItem@@@std@@@std@@QAAAAV012@ABV012@@Z 1003d7a0 f i SwiNotify.obj
 0001:0003c7e8       ??1?$_Bidit@UszCallbackItem@@HPBU1@ABU1@@std@@QAA@XZ 1003d7e8 f i SwiNotify.obj
 0001:0003c808       ??1_Iterator_base@std@@QAA@XZ 1003d808 f i SwiNotify.obj
 0001:0003c85c       ?_Orphan_me@_Iterator_base@std@@QAAXXZ 1003d85c f i SwiNotify.obj
 0001:0003c924       ??4?$_Bidit@UszCallbackItem@@HPBU1@ABU1@@std@@QAAAAU01@ABU01@@Z 1003d924 f i SwiNotify.obj
 0001:0003c95c       ??4_Iterator_base@std@@QAAAAV01@ABV01@@Z 1003d95c f i SwiNotify.obj
 0001:0003c9ec       ?_Adopt@_Iterator_base@std@@QAAXPBV_Container_base@2@@Z 1003d9ec f i SwiNotify.obj
 0001:0003ca9c       ??0szCallbackItem@@QAA@XZ  1003da9c f i SwiNotify.obj
 0001:0003cad0       ??1szCallbackItem@@QAA@XZ  1003dad0 f i SwiNotify.obj
 0001:0003caec       ??1?$_Iterator@$00@?$list@UszNotifyItem@@V?$allocator@UszNotifyItem@@@std@@@std@@QAA@XZ 1003daec f i SwiNotify.obj
 0001:0003cb04       ??4?$_Iterator@$00@?$list@UszNotifyItem@@V?$allocator@UszNotifyItem@@@std@@@std@@QAAAAV012@ABV012@@Z 1003db04 f i SwiNotify.obj
 0001:0003cb34       ??0?$_Iterator@$00@?$list@UszNotifyItem@@V?$allocator@UszNotifyItem@@@std@@@std@@QAA@ABV012@@Z 1003db34 f i SwiNotify.obj
 0001:0003cb68       ??0?$_Iterator@$00@?$list@UszCallbackItem@@V?$allocator@UszCallbackItem@@@std@@@std@@QAA@ABV012@@Z 1003db68 f i SwiNotify.obj
 0001:0003cb9c       ??1?$_Const_iterator@$00@?$list@UszNotifyItem@@V?$allocator@UszNotifyItem@@@std@@@std@@QAA@XZ 1003db9c f i SwiNotify.obj
 0001:0003cbb4       ??4?$_Const_iterator@$00@?$list@UszNotifyItem@@V?$allocator@UszNotifyItem@@@std@@@std@@QAAAAV012@ABV012@@Z 1003dbb4 f i SwiNotify.obj
 0001:0003cbfc       ??0?$_Const_iterator@$00@?$list@UszNotifyItem@@V?$allocator@UszNotifyItem@@@std@@@std@@QAA@ABV012@@Z 1003dbfc f i SwiNotify.obj
 0001:0003cc48       ??0?$_Const_iterator@$00@?$list@UszCallbackItem@@V?$allocator@UszCallbackItem@@@std@@@std@@QAA@ABV012@@Z 1003dc48 f i SwiNotify.obj
 0001:0003cc94       ??1?$_Bidit@UszNotifyItem@@HPBU1@ABU1@@std@@QAA@XZ 1003dc94 f i SwiNotify.obj
 0001:0003ccac       ??4?$_Bidit@UszNotifyItem@@HPBU1@ABU1@@std@@QAAAAU01@ABU01@@Z 1003dcac f i SwiNotify.obj
 0001:0003ccdc       ??0?$_Bidit@UszNotifyItem@@HPBU1@ABU1@@std@@QAA@ABU01@@Z 1003dcdc f i SwiNotify.obj
 0001:0003cd10       ??0_Iterator_base@std@@QAA@ABV01@@Z 1003dd10 f i SwiNotify.obj
 0001:0003cd5c       ??0?$_Bidit@UszCallbackItem@@HPBU1@ABU1@@std@@QAA@ABU01@@Z 1003dd5c f i SwiNotify.obj
 0001:0003cd98       ??0?$list@UszNotifyItem@@V?$allocator@UszNotifyItem@@@std@@@std@@QAA@XZ 1003dd98 f i SwiNotify.obj
 0001:0003ce30       ??1?$list@UszNotifyItem@@V?$allocator@UszNotifyItem@@@std@@@std@@QAA@XZ 1003de30 f i SwiNotify.obj
 0001:0003ce70       ?begin@?$list@UszNotifyItem@@V?$allocator@UszNotifyItem@@@std@@@std@@QAA?AV?$_Iterator@$00@12@XZ 1003de70 f i SwiNotify.obj
 0001:0003ced4       ?end@?$list@UszNotifyItem@@V?$allocator@UszNotifyItem@@@std@@@std@@QAA?AV?$_Iterator@$00@12@XZ 1003ded4 f i SwiNotify.obj
 0001:0003cf28       ?size@?$list@UszNotifyItem@@V?$allocator@UszNotifyItem@@@std@@@std@@QBAIXZ 1003df28 f i SwiNotify.obj
 0001:0003cf54       ?push_back@?$list@UszNotifyItem@@V?$allocator@UszNotifyItem@@@std@@@std@@QAAXABUszNotifyItem@@@Z 1003df54 f i SwiNotify.obj
 0001:0003cfa4       ?erase@?$list@UszNotifyItem@@V?$allocator@UszNotifyItem@@@std@@@std@@QAA?AV?$_Iterator@$00@12@V312@@Z 1003dfa4 f i SwiNotify.obj
 0001:0003d1b8       ?clear@?$list@UszNotifyItem@@V?$allocator@UszNotifyItem@@@std@@@std@@QAAXXZ 1003e1b8 f i SwiNotify.obj
 0001:0003d2cc       ??0?$list@UszCallbackItem@@V?$allocator@UszCallbackItem@@@std@@@std@@QAA@XZ 1003e2cc f i SwiNotify.obj
 0001:0003d364       ??1?$list@UszCallbackItem@@V?$allocator@UszCallbackItem@@@std@@@std@@QAA@XZ 1003e364 f i SwiNotify.obj
 0001:0003d3a4       ?begin@?$list@UszCallbackItem@@V?$allocator@UszCallbackItem@@@std@@@std@@QAA?AV?$_Iterator@$00@12@XZ 1003e3a4 f i SwiNotify.obj
 0001:0003d408       ?end@?$list@UszCallbackItem@@V?$allocator@UszCallbackItem@@@std@@@std@@QAA?AV?$_Iterator@$00@12@XZ 1003e408 f i SwiNotify.obj
 0001:0003d45c       ?size@?$list@UszCallbackItem@@V?$allocator@UszCallbackItem@@@std@@@std@@QBAIXZ 1003e45c f i SwiNotify.obj
 0001:0003d488       ?empty@?$list@UszCallbackItem@@V?$allocator@UszCallbackItem@@@std@@@std@@QBA_NXZ 1003e488 f i SwiNotify.obj
 0001:0003d4d8       ?pop_front@?$list@UszCallbackItem@@V?$allocator@UszCallbackItem@@@std@@@std@@QAAXXZ 1003e4d8 f i SwiNotify.obj
 0001:0003d52c       ?push_back@?$list@UszCallbackItem@@V?$allocator@UszCallbackItem@@@std@@@std@@QAAXABUszCallbackItem@@@Z 1003e52c f i SwiNotify.obj
 0001:0003d57c       ?erase@?$list@UszCallbackItem@@V?$allocator@UszCallbackItem@@@std@@@std@@QAA?AV?$_Iterator@$00@12@V312@@Z 1003e57c f i SwiNotify.obj
 0001:0003d790       ??0?$_Iterator@$00@?$list@UszCallbackItem@@V?$allocator@UszCallbackItem@@@std@@@std@@QAA@XZ 1003e790 f i SwiNotify.obj
 0001:0003d7c0       ??D?$_Iterator@$00@?$list@UszCallbackItem@@V?$allocator@UszCallbackItem@@@std@@@std@@QBAAAUszCallbackItem@@XZ 1003e7c0 f i SwiNotify.obj
 0001:0003d7f8       ??E?$_Iterator@$00@?$list@UszCallbackItem@@V?$allocator@UszCallbackItem@@@std@@@std@@QAA?AV012@H@Z 1003e7f8 f i SwiNotify.obj
 0001:0003d8b0       ??9?$_Const_iterator@$00@?$list@UszCallbackItem@@V?$allocator@UszCallbackItem@@@std@@@std@@QBA_NABV012@@Z 1003e8b0 f i SwiNotify.obj
 0001:0003d908       ??0?$_Iterator@$00@?$list@UszNotifyItem@@V?$allocator@UszNotifyItem@@@std@@@std@@QAA@XZ 1003e908 f i SwiNotify.obj
 0001:0003d938       ??D?$_Iterator@$00@?$list@UszNotifyItem@@V?$allocator@UszNotifyItem@@@std@@@std@@QBAAAUszNotifyItem@@XZ 1003e938 f i SwiNotify.obj
 0001:0003d970       ??E?$_Iterator@$00@?$list@UszNotifyItem@@V?$allocator@UszNotifyItem@@@std@@@std@@QAA?AV012@H@Z 1003e970 f i SwiNotify.obj
 0001:0003da28       ??9?$_Const_iterator@$00@?$list@UszNotifyItem@@V?$allocator@UszNotifyItem@@@std@@@std@@QBA_NABV012@@Z 1003ea28 f i SwiNotify.obj
 0001:0003da80       ??1?$_List_val@UszNotifyItem@@V?$allocator@UszNotifyItem@@@std@@@std@@QAA@XZ 1003ea80 f i SwiNotify.obj
 0001:0003da98       ??1?$_List_val@UszCallbackItem@@V?$allocator@UszCallbackItem@@@std@@@std@@QAA@XZ 1003ea98 f i SwiNotify.obj
 0001:0003dab0       ??1?$_List_ptr@UszNotifyItem@@V?$allocator@UszNotifyItem@@@std@@@std@@QAA@XZ 1003eab0 f i SwiNotify.obj
 0001:0003dac8       ??1?$_List_ptr@UszCallbackItem@@V?$allocator@UszCallbackItem@@@std@@@std@@QAA@XZ 1003eac8 f i SwiNotify.obj
 0001:0003dae0       ??1?$_List_nod@UszNotifyItem@@V?$allocator@UszNotifyItem@@@std@@@std@@QAA@XZ 1003eae0 f i SwiNotify.obj
 0001:0003daf8       ??1_Container_base@std@@QAA@XZ 1003eaf8 f i SwiNotify.obj
 0001:0003db10       ?_Orphan_all@_Container_base@std@@QBAXXZ 1003eb10 f i SwiNotify.obj
 0001:0003dba4       ??1?$_List_nod@UszCallbackItem@@V?$allocator@UszCallbackItem@@@std@@@std@@QAA@XZ 1003eba4 f i SwiNotify.obj
 0001:0003dbbc       ?_Nextnode@?$list@UszNotifyItem@@V?$allocator@UszNotifyItem@@@std@@@std@@KAAAPAU_Node@?$_List_nod@UszNotifyItem@@V?$allocator@UszNotifyItem@@@std@@@2@PAU342@@Z 1003ebbc f i SwiNotify.obj
 0001:0003dbe0       ?_Prevnode@?$list@UszNotifyItem@@V?$allocator@UszNotifyItem@@@std@@@std@@KAAAPAU_Node@?$_List_nod@UszNotifyItem@@V?$allocator@UszNotifyItem@@@std@@@2@PAU342@@Z 1003ebe0 f i SwiNotify.obj
 0001:0003dc10       ?_Insert@?$list@UszNotifyItem@@V?$allocator@UszNotifyItem@@@std@@@std@@QAAXV?$_Iterator@$00@12@ABUszNotifyItem@@@Z 1003ec10 f i SwiNotify.obj
 0001:0003dd14       ?_Buynode@?$list@UszNotifyItem@@V?$allocator@UszNotifyItem@@@std@@@std@@IAAPAU_Node@?$_List_nod@UszNotifyItem@@V?$allocator@UszNotifyItem@@@std@@@2@XZ 1003ed14 f i SwiNotify.obj
 0001:0003de18       ?_Tidy@?$list@UszNotifyItem@@V?$allocator@UszNotifyItem@@@std@@@std@@IAAXXZ 1003ee18 f i SwiNotify.obj
 0001:0003deac       ?_Orphan_ptr@?$list@UszNotifyItem@@V?$allocator@UszNotifyItem@@@std@@@std@@IBAXAAV12@PAU_Node@?$_List_nod@UszNotifyItem@@V?$allocator@UszNotifyItem@@@std@@@2@@Z 1003eeac f i SwiNotify.obj
 0001:0003df80       ??0?$_List_val@UszNotifyItem@@V?$allocator@UszNotifyItem@@@std@@@std@@QAA@V?$allocator@UszNotifyItem@@@1@@Z 1003ef80 f i SwiNotify.obj
 0001:0003dfdc       ??0?$allocator@UszNotifyItem@@@std@@QAA@XZ 1003efdc f i SwiNotify.obj
 0001:0003e000       ?deallocate@?$allocator@U_Node@?$_List_nod@UszNotifyItem@@V?$allocator@UszNotifyItem@@@std@@@std@@@std@@QAAXPAU_Node@?$_List_nod@UszNotifyItem@@V?$allocator@UszNotifyItem@@@std@@@2@I@Z 1003f000 f i SwiNotify.obj
 0001:0003e018       ?destroy@?$allocator@U_Node@?$_List_nod@UszNotifyItem@@V?$allocator@UszNotifyItem@@@std@@@std@@@std@@QAAXPAU_Node@?$_List_nod@UszNotifyItem@@V?$allocator@UszNotifyItem@@@std@@@2@@Z 1003f018 f i SwiNotify.obj
 0001:0003e030       ?_Nextnode@?$list@UszCallbackItem@@V?$allocator@UszCallbackItem@@@std@@@std@@KAAAPAU_Node@?$_List_nod@UszCallbackItem@@V?$allocator@UszCallbackItem@@@std@@@2@PAU342@@Z 1003f030 f i SwiNotify.obj
 0001:0003e054       ?_Prevnode@?$list@UszCallbackItem@@V?$allocator@UszCallbackItem@@@std@@@std@@KAAAPAU_Node@?$_List_nod@UszCallbackItem@@V?$allocator@UszCallbackItem@@@std@@@2@PAU342@@Z 1003f054 f i SwiNotify.obj
 0001:0003e084       ?_Insert@?$list@UszCallbackItem@@V?$allocator@UszCallbackItem@@@std@@@std@@QAAXV?$_Iterator@$00@12@ABUszCallbackItem@@@Z 1003f084 f i SwiNotify.obj
 0001:0003e188       ?_Buynode@?$list@UszCallbackItem@@V?$allocator@UszCallbackItem@@@std@@@std@@IAAPAU_Node@?$_List_nod@UszCallbackItem@@V?$allocator@UszCallbackItem@@@std@@@2@XZ 1003f188 f i SwiNotify.obj
 0001:0003e28c       ?_Tidy@?$list@UszCallbackItem@@V?$allocator@UszCallbackItem@@@std@@@std@@IAAXXZ 1003f28c f i SwiNotify.obj
 0001:0003e320       ?_Orphan_ptr@?$list@UszCallbackItem@@V?$allocator@UszCallbackItem@@@std@@@std@@IBAXAAV12@PAU_Node@?$_List_nod@UszCallbackItem@@V?$allocator@UszCallbackItem@@@std@@@2@@Z 1003f320 f i SwiNotify.obj
 0001:0003e3f4       ??0?$_List_val@UszCallbackItem@@V?$allocator@UszCallbackItem@@@std@@@std@@QAA@V?$allocator@UszCallbackItem@@@1@@Z 1003f3f4 f i SwiNotify.obj
 0001:0003e450       ??0?$allocator@UszCallbackItem@@@std@@QAA@XZ 1003f450 f i SwiNotify.obj
 0001:0003e474       ?deallocate@?$allocator@U_Node@?$_List_nod@UszCallbackItem@@V?$allocator@UszCallbackItem@@@std@@@std@@@std@@QAAXPAU_Node@?$_List_nod@UszCallbackItem@@V?$allocator@UszCallbackItem@@@std@@@2@I@Z 1003f474 f i SwiNotify.obj
 0001:0003e48c       ?destroy@?$allocator@U_Node@?$_List_nod@UszCallbackItem@@V?$allocator@UszCallbackItem@@@std@@@std@@@std@@QAAXPAU_Node@?$_List_nod@UszCallbackItem@@V?$allocator@UszCallbackItem@@@std@@@2@@Z 1003f48c f i SwiNotify.obj
 0001:0003e4a4       ??0?$_Iterator@$00@?$list@UszCallbackItem@@V?$allocator@UszCallbackItem@@@std@@@std@@QAA@PAU_Node@?$_List_nod@UszCallbackItem@@V?$allocator@UszCallbackItem@@@std@@@2@PBV12@@Z 1003f4a4 f i SwiNotify.obj
 0001:0003e4dc       ??E?$_Iterator@$00@?$list@UszCallbackItem@@V?$allocator@UszCallbackItem@@@std@@@std@@QAAAAV012@XZ 1003f4dc f i SwiNotify.obj
 0001:0003e508       ??0?$_Const_iterator@$00@?$list@UszCallbackItem@@V?$allocator@UszCallbackItem@@@std@@@std@@QAA@XZ 1003f508 f i SwiNotify.obj
 0001:0003e548       ??D?$_Const_iterator@$00@?$list@UszCallbackItem@@V?$allocator@UszCallbackItem@@@std@@@std@@QBAABUszCallbackItem@@XZ 1003f548 f i SwiNotify.obj
 0001:0003e624       ??8?$_Const_iterator@$00@?$list@UszCallbackItem@@V?$allocator@UszCallbackItem@@@std@@@std@@QBA_NABV012@@Z 1003f624 f i SwiNotify.obj
 0001:0003e68c       ?_Mynode@?$_Const_iterator@$00@?$list@UszCallbackItem@@V?$allocator@UszCallbackItem@@@std@@@std@@QBAPAU_Node@?$_List_nod@UszCallbackItem@@V?$allocator@UszCallbackItem@@@std@@@3@XZ 1003f68c f i SwiNotify.obj
 0001:0003e6b8       ??0?$_Iterator@$00@?$list@UszNotifyItem@@V?$allocator@UszNotifyItem@@@std@@@std@@QAA@PAU_Node@?$_List_nod@UszNotifyItem@@V?$allocator@UszNotifyItem@@@std@@@2@PBV12@@Z 1003f6b8 f i SwiNotify.obj
 0001:0003e6f0       ??E?$_Iterator@$00@?$list@UszNotifyItem@@V?$allocator@UszNotifyItem@@@std@@@std@@QAAAAV012@XZ 1003f6f0 f i SwiNotify.obj
 0001:0003e71c       ??0?$_Const_iterator@$00@?$list@UszNotifyItem@@V?$allocator@UszNotifyItem@@@std@@@std@@QAA@XZ 1003f71c f i SwiNotify.obj
 0001:0003e75c       ??D?$_Const_iterator@$00@?$list@UszNotifyItem@@V?$allocator@UszNotifyItem@@@std@@@std@@QBAABUszNotifyItem@@XZ 1003f75c f i SwiNotify.obj
 0001:0003e838       ??8?$_Const_iterator@$00@?$list@UszNotifyItem@@V?$allocator@UszNotifyItem@@@std@@@std@@QBA_NABV012@@Z 1003f838 f i SwiNotify.obj
 0001:0003e8a0       ?_Mynode@?$_Const_iterator@$00@?$list@UszNotifyItem@@V?$allocator@UszNotifyItem@@@std@@@std@@QBAPAU_Node@?$_List_nod@UszNotifyItem@@V?$allocator@UszNotifyItem@@@std@@@3@XZ 1003f8a0 f i SwiNotify.obj
 0001:0003e8cc       ??0?$_Bidit@UszCallbackItem@@HPBU1@ABU1@@std@@QAA@XZ 1003f8cc f i SwiNotify.obj
 0001:0003e8fc       ??0_Iterator_base@std@@QAA@XZ 1003f8fc f i SwiNotify.obj
 0001:0003e93c       ??0?$_Bidit@UszNotifyItem@@HPBU1@ABU1@@std@@QAA@XZ 1003f93c f i SwiNotify.obj
 0001:0003e96c       ?_Myval@?$list@UszNotifyItem@@V?$allocator@UszNotifyItem@@@std@@@std@@KAAAUszNotifyItem@@PAU_Node@?$_List_nod@UszNotifyItem@@V?$allocator@UszNotifyItem@@@std@@@2@@Z 1003f96c f i SwiNotify.obj
 0001:0003e99c       ?_Buynode@?$list@UszNotifyItem@@V?$allocator@UszNotifyItem@@@std@@@std@@IAAPAU_Node@?$_List_nod@UszNotifyItem@@V?$allocator@UszNotifyItem@@@std@@@2@PAU342@0ABUszNotifyItem@@@Z 1003f99c f i SwiNotify.obj
 0001:0003eafc       ?_Incsize@?$list@UszNotifyItem@@V?$allocator@UszNotifyItem@@@std@@@std@@IAAXI@Z 1003fafc f i SwiNotify.obj
 0001:0003ebcc       ??0length_error@std@@QAA@ABV?$basic_string@DU?$char_traits@D@std@@V?$allocator@D@2@@1@@Z 1003fbcc f i SwiNotify.obj
 0001:0003ec18       ??0logic_error@std@@QAA@ABV?$basic_string@DU?$char_traits@D@std@@V?$allocator@D@2@@1@@Z 1003fc18 f i SwiNotify.obj
 0001:0003ec88       ?what@logic_error@std@@UBAPBDXZ 1003fc88 f i SwiNotify.obj
 0001:0003ecbc       ??_Elogic_error@std@@UAAPAXI@Z 1003fcbc f i SwiNotify.obj
 0001:0003ecbc       ??_Glogic_error@std@@UAAPAXI@Z 1003fcbc f i SwiNotify.obj
 0001:0003ecfc       ??1logic_error@std@@UAA@XZ 1003fcfc f i SwiNotify.obj
 0001:0003ed30       ??1length_error@std@@UAA@XZ 1003fd30 f i SwiNotify.obj
 0001:0003ed58       ??_Glength_error@std@@UAAPAXI@Z 1003fd58 f i SwiNotify.obj
 0001:0003ed58       ??_Elength_error@std@@UAAPAXI@Z 1003fd58 f i SwiNotify.obj
 0001:0003eda0       ??0?$basic_string@DU?$char_traits@D@std@@V?$allocator@D@2@@std@@QAA@ABV01@@Z 1003fda0 f i SwiNotify.obj
 0001:0003ee40       ??1?$basic_string@DU?$char_traits@D@std@@V?$allocator@D@2@@std@@QAA@XZ 1003fe40 f i SwiNotify.obj
 0001:0003ee88       ?c_str@?$basic_string@DU?$char_traits@D@std@@V?$allocator@D@2@@std@@QBAPBDXZ 1003fe88 f i SwiNotify.obj
 0001:0003eeb8       ??1?$_String_val@DV?$allocator@D@std@@@std@@QAA@XZ 1003feb8 f i SwiNotify.obj
 0001:0003eed0       ??1_String_base@std@@QAA@XZ 1003fed0 f i SwiNotify.obj
 0001:0003eee8       ?assign@?$basic_string@DU?$char_traits@D@std@@V?$allocator@D@2@@std@@QAAAAV12@ABV12@II@Z 1003fee8 f i SwiNotify.obj
 0001:0003f00c       ?_Tidy@?$basic_string@DU?$char_traits@D@std@@V?$allocator@D@2@@std@@IAAX_NI@Z 1004000c f i SwiNotify.obj
 0001:0003f0b8       ?_Myptr@?$basic_string@DU?$char_traits@D@std@@V?$allocator@D@2@@std@@IBAPBDXZ 100400b8 f i SwiNotify.obj
 0001:0003f110       ??0?$_String_val@DV?$allocator@D@std@@@std@@IAA@V?$allocator@D@1@@Z 10040110 f i SwiNotify.obj
 0001:0003f150       ??0?$allocator@D@std@@QAA@ABV01@@Z 10040150 f i SwiNotify.obj
 0001:0003f174       ??0_String_base@std@@QAA@XZ 10040174 f i SwiNotify.obj
 0001:0003f1a4       ??0_Container_base@std@@QAA@XZ 100401a4 f i SwiNotify.obj
 0001:0003f1d4       ?erase@?$basic_string@DU?$char_traits@D@std@@V?$allocator@D@2@@std@@QAAAAV12@II@Z 100401d4 f i SwiNotify.obj
 0001:0003f2e8       ?size@?$basic_string@DU?$char_traits@D@std@@V?$allocator@D@2@@std@@QBAIXZ 100402e8 f i SwiNotify.obj
 0001:0003f314       ?_Eos@?$basic_string@DU?$char_traits@D@std@@V?$allocator@D@2@@std@@IAAXI@Z 10040314 f i SwiNotify.obj
 0001:0003f364       ?assign@?$char_traits@D@std@@SAXAADABD@Z 10040364 f i SwiNotify.obj
 0001:0003f384       ?_Grow@?$basic_string@DU?$char_traits@D@std@@V?$allocator@D@2@@std@@IAA_NI_N@Z 10040384 f i SwiNotify.obj
 0001:0003f498       ?_Myptr@?$basic_string@DU?$char_traits@D@std@@V?$allocator@D@2@@std@@IAAPADXZ 10040498 f i SwiNotify.obj
 0001:0003f4f0       ?deallocate@?$allocator@D@std@@QAAXPADI@Z 100404f0 f i SwiNotify.obj
 0001:0003f508       ??0?$_List_ptr@UszNotifyItem@@V?$allocator@UszNotifyItem@@@std@@@std@@IAA@V?$allocator@UszNotifyItem@@@1@@Z 10040508 f i SwiNotify.obj
 0001:0003f564       ??0?$allocator@UszNotifyItem@@@std@@QAA@ABV01@@Z 10040564 f i SwiNotify.obj
 0001:0003f588       ?allocate@?$allocator@U_Node@?$_List_nod@UszNotifyItem@@V?$allocator@UszNotifyItem@@@std@@@std@@@std@@QAAPAU_Node@?$_List_nod@UszNotifyItem@@V?$allocator@UszNotifyItem@@@std@@@2@I@Z 10040588 f i SwiNotify.obj
 0001:0003f5bc       ?construct@?$allocator@PAU_Node@?$_List_nod@UszNotifyItem@@V?$allocator@UszNotifyItem@@@std@@@std@@@std@@QAAXPAPAU_Node@?$_List_nod@UszNotifyItem@@V?$allocator@UszNotifyItem@@@std@@@2@ABQAU342@@Z 100405bc f i SwiNotify.obj
 0001:0003f5d8       ?destroy@?$allocator@PAU_Node@?$_List_nod@UszNotifyItem@@V?$allocator@UszNotifyItem@@@std@@@std@@@std@@QAAXPAPAU_Node@?$_List_nod@UszNotifyItem@@V?$allocator@UszNotifyItem@@@std@@@2@@Z 100405d8 f i SwiNotify.obj
 0001:0003f5f0       ?_Myval@?$list@UszCallbackItem@@V?$allocator@UszCallbackItem@@@std@@@std@@KAAAUszCallbackItem@@PAU_Node@?$_List_nod@UszCallbackItem@@V?$allocator@UszCallbackItem@@@std@@@2@@Z 100405f0 f i SwiNotify.obj
 0001:0003f618       ?clear@?$list@UszCallbackItem@@V?$allocator@UszCallbackItem@@@std@@@std@@QAAXXZ 10040618 f i SwiNotify.obj
 0001:0003f72c       ?_Buynode@?$list@UszCallbackItem@@V?$allocator@UszCallbackItem@@@std@@@std@@IAAPAU_Node@?$_List_nod@UszCallbackItem@@V?$allocator@UszCallbackItem@@@std@@@2@PAU342@0ABUszCallbackItem@@@Z 1004072c f i SwiNotify.obj
 0001:0003f88c       ?_Incsize@?$list@UszCallbackItem@@V?$allocator@UszCallbackItem@@@std@@@std@@IAAXI@Z 1004088c f i SwiNotify.obj
 0001:0003f95c       ??0?$_List_ptr@UszCallbackItem@@V?$allocator@UszCallbackItem@@@std@@@std@@IAA@V?$allocator@UszCallbackItem@@@1@@Z 1004095c f i SwiNotify.obj
 0001:0003f9b8       ??0?$allocator@UszCallbackItem@@@std@@QAA@ABV01@@Z 100409b8 f i SwiNotify.obj
 0001:0003f9dc       ?allocate@?$allocator@U_Node@?$_List_nod@UszCallbackItem@@V?$allocator@UszCallbackItem@@@std@@@std@@@std@@QAAPAU_Node@?$_List_nod@UszCallbackItem@@V?$allocator@UszCallbackItem@@@std@@@2@I@Z 100409dc f i SwiNotify.obj
 0001:0003fa10       ?construct@?$allocator@PAU_Node@?$_List_nod@UszCallbackItem@@V?$allocator@UszCallbackItem@@@std@@@std@@@std@@QAAXPAPAU_Node@?$_List_nod@UszCallbackItem@@V?$allocator@UszCallbackItem@@@std@@@2@ABQAU342@@Z 10040a10 f i SwiNotify.obj
 0001:0003fa2c       ?destroy@?$allocator@PAU_Node@?$_List_nod@UszCallbackItem@@V?$allocator@UszCallbackItem@@@std@@@std@@@std@@QAAXPAPAU_Node@?$_List_nod@UszCallbackItem@@V?$allocator@UszCallbackItem@@@std@@@2@@Z 10040a2c f i SwiNotify.obj
 0001:0003fa4c       ??0?$_Const_iterator@$00@?$list@UszCallbackItem@@V?$allocator@UszCallbackItem@@@std@@@std@@QAA@PAU_Node@?$_List_nod@UszCallbackItem@@V?$allocator@UszCallbackItem@@@std@@@2@PBV12@@Z 10040a4c f i SwiNotify.obj
 0001:0003fab4       ??E?$_Const_iterator@$00@?$list@UszCallbackItem@@V?$allocator@UszCallbackItem@@@std@@@std@@QAAAAV012@XZ 10040ab4 f i SwiNotify.obj
 0001:0003fba4       ?_Compat@?$_Const_iterator@$00@?$list@UszCallbackItem@@V?$allocator@UszCallbackItem@@@std@@@std@@QBAXABV123@@Z 10040ba4 f i SwiNotify.obj
 0001:0003fc68       ??0?$_Const_iterator@$00@?$list@UszNotifyItem@@V?$allocator@UszNotifyItem@@@std@@@std@@QAA@PAU_Node@?$_List_nod@UszNotifyItem@@V?$allocator@UszNotifyItem@@@std@@@2@PBV12@@Z 10040c68 f i SwiNotify.obj
 0001:0003fcd0       ??E?$_Const_iterator@$00@?$list@UszNotifyItem@@V?$allocator@UszNotifyItem@@@std@@@std@@QAAAAV012@XZ 10040cd0 f i SwiNotify.obj
 0001:0003fdc0       ?_Compat@?$_Const_iterator@$00@?$list@UszNotifyItem@@V?$allocator@UszNotifyItem@@@std@@@std@@QBAXABV123@@Z 10040dc0 f i SwiNotify.obj
 0001:0003fe7c       ??0length_error@std@@QAA@ABV01@@Z 10040e7c f i SwiNotify.obj
 0001:0003fec8       ??0logic_error@std@@QAA@ABV01@@Z 10040ec8 f i SwiNotify.obj
 0001:0003ff48       ??0?$basic_string@DU?$char_traits@D@std@@V?$allocator@D@2@@std@@QAA@PBD@Z 10040f48 f i SwiNotify.obj
 0001:0003ffc8       ?max_size@?$basic_string@DU?$char_traits@D@std@@V?$allocator@D@2@@std@@QBAIXZ 10040fc8 f i SwiNotify.obj
 0001:00040030       ?_Copy@?$basic_string@DU?$char_traits@D@std@@V?$allocator@D@2@@std@@IAAXII@Z 10041030 f i SwiNotify.obj
 0001:00040264       ?max_size@?$list@UszNotifyItem@@V?$allocator@UszNotifyItem@@@std@@@std@@QBAIXZ 10041264 f i SwiNotify.obj
 0001:00040298       ??0?$_List_nod@UszNotifyItem@@V?$allocator@UszNotifyItem@@@std@@@std@@IAA@V?$allocator@UszNotifyItem@@@1@@Z 10041298 f i SwiNotify.obj
 0001:000402d8       ?construct@?$allocator@UszNotifyItem@@@std@@QAAXPAUszNotifyItem@@ABU3@@Z 100412d8 f i SwiNotify.obj
 0001:000402f4       ?max_size@?$list@UszCallbackItem@@V?$allocator@UszCallbackItem@@@std@@@std@@QBAIXZ 100412f4 f i SwiNotify.obj
 0001:00040328       ??0?$_List_nod@UszCallbackItem@@V?$allocator@UszCallbackItem@@@std@@@std@@IAA@V?$allocator@UszCallbackItem@@@1@@Z 10041328 f i SwiNotify.obj
 0001:00040368       ?construct@?$allocator@UszCallbackItem@@@std@@QAAXPAUszCallbackItem@@ABU3@@Z 10041368 f i SwiNotify.obj
 0001:00040384       ?assign@?$basic_string@DU?$char_traits@D@std@@V?$allocator@D@2@@std@@QAAAAV12@PBD@Z 10041384 f i SwiNotify.obj
 0001:000403c8       ?length@?$char_traits@D@std@@SAIPBD@Z 100413c8 f i SwiNotify.obj
 0001:000403f8       ??0?$allocator@D@std@@QAA@XZ 100413f8 f i SwiNotify.obj
 0001:0004041c       ?allocate@?$allocator@D@std@@QAAPADI@Z 1004141c f i SwiNotify.obj
 0001:00040450       ?max_size@?$allocator@D@std@@QBAIXZ 10041450 f i SwiNotify.obj
 0001:0004049c       ?max_size@?$allocator@UszNotifyItem@@@std@@QBAIXZ 1004149c f i SwiNotify.obj
 0001:000404e8       ?max_size@?$allocator@UszCallbackItem@@@std@@QBAIXZ 100414e8 f i SwiNotify.obj
 0001:00040538       ?assign@?$basic_string@DU?$char_traits@D@std@@V?$allocator@D@2@@std@@QAAAAV12@PBDI@Z 10041538 f i SwiNotify.obj
 0001:00040604       ?_Inside@?$basic_string@DU?$char_traits@D@std@@V?$allocator@D@2@@std@@IAA_NPBD@Z 10041604 f i SwiNotify.obj
 0001:00040698       ??$_Debug_pointer@D@std@@YAXPBDPBGI@Z 10041698 f i SwiNotify.obj
 0001:000406c8       ??$copy_s@U?$char_traits@D@std@@@_Traits_helper@std@@YAPADPADIPBDI@Z 100416c8 f i SwiNotify.obj
 0001:00040730       ??$_Destroy@U_Node@?$_List_nod@UszNotifyItem@@V?$allocator@UszNotifyItem@@@std@@@std@@@std@@YAXPAU_Node@?$_List_nod@UszNotifyItem@@V?$allocator@UszNotifyItem@@@std@@@0@@Z 10041730 f i SwiNotify.obj
 0001:00040740       ??$_Destroy@U_Node@?$_List_nod@UszCallbackItem@@V?$allocator@UszCallbackItem@@@std@@@std@@@std@@YAXPAU_Node@?$_List_nod@UszCallbackItem@@V?$allocator@UszCallbackItem@@@std@@@0@@Z 10041740 f i SwiNotify.obj
 0001:0004075c       ??$move_s@U?$char_traits@D@std@@@_Traits_helper@std@@YAPADPADIPBDI@Z 1004175c f i SwiNotify.obj
 0001:000407c4       ??$?0UszNotifyItem@@@?$allocator@PAU_Node@?$_List_nod@UszNotifyItem@@V?$allocator@UszNotifyItem@@@std@@@std@@@std@@QAA@ABV?$allocator@UszNotifyItem@@@1@@Z 100417c4 f i SwiNotify.obj
 0001:000407e8       ??$_Allocate@U_Node@?$_List_nod@UszNotifyItem@@V?$allocator@UszNotifyItem@@@std@@@std@@@std@@YAPAU_Node@?$_List_nod@UszNotifyItem@@V?$allocator@UszNotifyItem@@@std@@@0@IPAU120@@Z 100417e8 f i SwiNotify.obj
 0001:00040878       ??0bad_alloc@std@@QAA@PBD@Z 10041878 f i SwiNotify.obj
 0001:000408bc       ??1bad_alloc@std@@UAA@XZ   100418bc f i SwiNotify.obj
 0001:000408e4       ??_Ebad_alloc@std@@UAAPAXI@Z 100418e4 f i SwiNotify.obj
 0001:000408e4       ??_Gbad_alloc@std@@UAAPAXI@Z 100418e4 f i SwiNotify.obj
 0001:00040924       ??$_Construct@PAU_Node@?$_List_nod@UszNotifyItem@@V?$allocator@UszNotifyItem@@@std@@@std@@PAU123@@std@@YAXPAPAU_Node@?$_List_nod@UszNotifyItem@@V?$allocator@UszNotifyItem@@@std@@@0@ABQAU120@@Z 10041924 f i SwiNotify.obj
 0001:0004098c       ??2@YAPAXIPAX@Z            1004198c f i SwiNotify.obj
 0001:000409b0       ??$_Destroy@PAU_Node@?$_List_nod@UszNotifyItem@@V?$allocator@UszNotifyItem@@@std@@@std@@@std@@YAXPAPAU_Node@?$_List_nod@UszNotifyItem@@V?$allocator@UszNotifyItem@@@std@@@0@@Z 100419b0 f i SwiNotify.obj
 0001:000409c0       ??$?0UszCallbackItem@@@?$allocator@PAU_Node@?$_List_nod@UszCallbackItem@@V?$allocator@UszCallbackItem@@@std@@@std@@@std@@QAA@ABV?$allocator@UszCallbackItem@@@1@@Z 100419c0 f i SwiNotify.obj
 0001:000409e4       ??$_Allocate@U_Node@?$_List_nod@UszCallbackItem@@V?$allocator@UszCallbackItem@@@std@@@std@@@std@@YAPAU_Node@?$_List_nod@UszCallbackItem@@V?$allocator@UszCallbackItem@@@std@@@0@IPAU120@@Z 100419e4 f i SwiNotify.obj
 0001:00040a74       ??$_Construct@PAU_Node@?$_List_nod@UszCallbackItem@@V?$allocator@UszCallbackItem@@@std@@@std@@PAU123@@std@@YAXPAPAU_Node@?$_List_nod@UszCallbackItem@@V?$allocator@UszCallbackItem@@@std@@@0@ABQAU120@@Z 10041a74 f i SwiNotify.obj
 0001:00040adc       ??$_Destroy@PAU_Node@?$_List_nod@UszCallbackItem@@V?$allocator@UszCallbackItem@@@std@@@std@@@std@@YAXPAPAU_Node@?$_List_nod@UszCallbackItem@@V?$allocator@UszCallbackItem@@@std@@@0@@Z 10041adc f i SwiNotify.obj
 0001:00040aec       ??$?0UszNotifyItem@@@?$allocator@U_Node@?$_List_nod@UszNotifyItem@@V?$allocator@UszNotifyItem@@@std@@@std@@@std@@QAA@ABV?$allocator@UszNotifyItem@@@1@@Z 10041aec f i SwiNotify.obj
 0001:00040b10       ??$_Construct@UszNotifyItem@@U1@@std@@YAXPAUszNotifyItem@@ABU1@@Z 10041b10 f i SwiNotify.obj
 0001:00040b78       ??$?0UszCallbackItem@@@?$allocator@U_Node@?$_List_nod@UszCallbackItem@@V?$allocator@UszCallbackItem@@@std@@@std@@@std@@QAA@ABV?$allocator@UszCallbackItem@@@1@@Z 10041b78 f i SwiNotify.obj
 0001:00040ba4       ??$_Construct@UszCallbackItem@@U1@@std@@YAXPAUszCallbackItem@@ABU1@@Z 10041ba4 f i SwiNotify.obj
 0001:00040c34       ??3@YAXPAX0@Z              10041c34 f i SwiNotify.obj
 0001:00040c44       ??$_Allocate@D@std@@YAPADIPAD@Z 10041c44 f i SwiNotify.obj
 0001:00040ccc       ??_G_Node@?$_List_nod@UszCallbackItem@@V?$allocator@UszCallbackItem@@@std@@@std@@QAAPAXI@Z 10041ccc f i SwiNotify.obj
 0001:00040d0c       ??0bad_alloc@std@@QAA@ABV01@@Z 10041d0c f i SwiNotify.obj
 0001:00040d50       ??0szCallbackItem@@QAA@ABU0@@Z 10041d50 f i SwiNotify.obj
 0001:00040d9c       ??1_Node@?$_List_nod@UszCallbackItem@@V?$allocator@UszCallbackItem@@@std@@@std@@QAA@XZ 10041d9c f i SwiNotify.obj
 0001:00040dc0       ??0?$list@UszNotifyItem@@V?$allocator@UszNotifyItem@@@std@@@std@@QAA@ABV01@@Z 10041dc0 f i SwiNotify.obj
 0001:00040f34       ?begin@?$list@UszNotifyItem@@V?$allocator@UszNotifyItem@@@std@@@std@@QBA?AV?$_Const_iterator@$00@12@XZ 10041f34 f i SwiNotify.obj
 0001:00040f98       ?end@?$list@UszNotifyItem@@V?$allocator@UszNotifyItem@@@std@@@std@@QBA?AV?$_Const_iterator@$00@12@XZ 10041f98 f i SwiNotify.obj
 0001:00040fec       ??$_Char_traits_cat@U?$char_traits@D@std@@@std@@YA?AU_Secure_char_traits_tag@0@XZ 10041fec f i SwiNotify.obj
 0001:00041020       ??$copy_s@U?$char_traits@D@std@@@_Traits_helper@std@@YAPADPADIPBDIU_Secure_char_traits_tag@1@@Z 10042020 f i SwiNotify.obj
 0001:0004105c       ?_Copy_s@?$char_traits@D@std@@SAPADPADIPBDI@Z 1004205c f i SwiNotify.obj
 0001:00041094       ??$move_s@U?$char_traits@D@std@@@_Traits_helper@std@@YAPADPADIPBDIU_Secure_char_traits_tag@1@@Z 10042094 f i SwiNotify.obj
 0001:000410d0       ?_Move_s@?$char_traits@D@std@@SAPADPADIPBDI@Z 100420d0 f i SwiNotify.obj
 0001:00041110       ??$insert@V?$_Const_iterator@$00@?$list@UszNotifyItem@@V?$allocator@UszNotifyItem@@@std@@@std@@@?$list@UszNotifyItem@@V?$allocator@UszNotifyItem@@@std@@@std@@QAAXV?$_Iterator@$00@01@V?$_Const_iterator@$00@01@1@Z 10042110 f i SwiNotify.obj
 0001:00041274       ??$_Iter_cat@V?$_Const_iterator@$00@?$list@UszNotifyItem@@V?$allocator@UszNotifyItem@@@std@@@std@@@std@@YA?AUbidirectional_iterator_tag@0@ABV?$_Const_iterator@$00@?$list@UszNotifyItem@@V?$allocator@UszNotifyItem@@@std@@@0@@Z 10042274 f i SwiNotify.obj
 0001:000412a0       ??$_Insert@V?$_Const_iterator@$00@?$list@UszNotifyItem@@V?$allocator@UszNotifyItem@@@std@@@std@@@?$list@UszNotifyItem@@V?$allocator@UszNotifyItem@@@std@@@std@@QAAXV?$_Iterator@$00@01@V?$_Const_iterator@$00@01@1Uforward_iterator_tag@1@@Z 100422a0 f i SwiNotify.obj
 0001:00041530       ??F?$_Iterator@$00@?$list@UszNotifyItem@@V?$allocator@UszNotifyItem@@@std@@@std@@QAAAAV012@XZ 10042530 f i SwiNotify.obj
 0001:0004155c       ??F?$_Const_iterator@$00@?$list@UszNotifyItem@@V?$allocator@UszNotifyItem@@@std@@@std@@QAAAAV012@XZ 1004255c f i SwiNotify.obj
 0001:00041660       ??$_Debug_range@V?$_Const_iterator@$00@?$list@UszNotifyItem@@V?$allocator@UszNotifyItem@@@std@@@std@@@std@@YAXV?$_Const_iterator@$00@?$list@UszNotifyItem@@V?$allocator@UszNotifyItem@@@std@@@0@0PBGI@Z 10042660 f i SwiNotify.obj
 0001:0004175c       ??$_Debug_get_cont@V?$_Const_iterator@$00@?$list@UszNotifyItem@@V?$allocator@UszNotifyItem@@@std@@@std@@@std@@YAPBV_Container_base@0@ABV?$_Const_iterator@$00@?$list@UszNotifyItem@@V?$allocator@UszNotifyItem@@@std@@@0@@Z 1004275c f i SwiNotify.obj
 0001:00041788       ??$_Debug_range2@V?$_Const_iterator@$00@?$list@UszNotifyItem@@V?$allocator@UszNotifyItem@@@std@@@std@@@std@@YAXV?$_Const_iterator@$00@?$list@UszNotifyItem@@V?$allocator@UszNotifyItem@@@std@@@0@0PBGIUinput_iterator_tag@0@@Z 10042788 f i SwiNotify.obj
 0001:000417c8       ?SemiByteToChar@@YADEH@Z   100427c8 f   util.obj
 0001:000418b4       ?SemiByteCharsToByte@@YAEDD@Z 100428b4 f   util.obj
 0001:00041970       ?UnicodeCharToGSM@@YAHGPAD@Z 10042970 f   util.obj
 0001:00041b28       ?GSMCharToUnicode@@YAHDPAG@Z 10042b28 f   util.obj
 0001:00041b70       ?GSMHexToGSM@@YAHQBDIQADIAAI@Z 10042b70 f   util.obj
 0001:00041c58       ?GSMToGSMHex@@YAHQBDIQADIAAI@Z 10042c58 f   util.obj
 0001:00041d64       ?ConvertFromUnicode@@YAHW4ENCODING_TYPE@@QBGIQADIAAI@Z 10042d64 f   util.obj
 0001:000426dc       ?ConvertToUnicode@@YAHW4ENCODING_TYPE@@QBDIQAGIAAI@Z 100436dc f   util.obj
 0001:00042e3c       ?DetermineSimResponseError@@YAJKK@Z 10043e3c f   util.obj
 0001:00042f30       ?IsElementarySimFile@@YAHK@Z 10043f30 f   util.obj
 0001:00042fbc       ?StringFilterW@@YAJPAGI00@Z 10043fbc f   util.obj
 0001:00043114       ?ComposeCmdWithByteArray@@YAHQBDQBEI0AAPAD@Z 10044114 f   util.obj
 0001:00043548       ?BeginLineSpecificCommand@@YAPADPADIK@Z 10044548 f   util.obj
 0001:00043590       ?AllocateOrReallocateStorage@@YAHQAPAEIIQAII@Z 10044590 f   util.obj
 0001:00043740       ?DumpMem@@YAXPAXH@Z        10044740 f   util.obj
 0001:00044460       __security_check_cookie    10045460     corelibc:armsecgs.obj
 0001:00044474       __gsfailure                10045474     corelibc:armsecgs.obj
 0001:000444b8       _onexit                    100454b8 f   corelibc:onexit.obj
 0001:00044564       atexit                     10045564 f   corelibc:onexit.obj
 0001:00044584       _DllMainCRTStartup         10045584 f   corelibc:pegdmain.obj
 0001:0004461c       __security_init_cookie     1004561c f   corelibc:seccinit.obj
 0001:0004466c       GetCurrentProcess          1004566c f i corelibc:crt0dat.obj
 0001:000446a8       _cinit                     100456a8 f   corelibc:crt0dat.obj
 0001:00044818       exit                       10045818 f   corelibc:crt0dat.obj
 0001:00044830       _exit                      10045830 f   corelibc:crt0dat.obj
 0001:00044848       _cexit                     10045848 f   corelibc:crt0dat.obj
 0001:00044864       _c_exit                    10045864 f   corelibc:crt0dat.obj
 0001:000448b0       ?ConvertGSMMixedToUnicode@@YA_NIQBDIQAGIAAI@Z 100458b0 f   ccoreutl:ccoreutl.dll
 0001:000448c0       ntohl                      100458c0 f   ws2:WS2.dll
 0001:000448d0       inet_ntoa                  100458d0 f   ws2:WS2.dll
 0001:000448e0       SetEvent                   100458e0 f i toolbox:toolbox_i.obj
 0001:000448f4       ??0SYNCBLOCK_Implementation@@QAA@AAUCRITICAL_SECTION@@@Z 100458f4 f i toolbox:toolbox_i.obj
 0001:00044914       ??1SYNCBLOCK_Implementation@@QAA@XZ 10045914 f i toolbox:toolbox_i.obj
 0001:00044928       ??0UNSYNCBLOCK_Implementation@@QAA@AAUCRITICAL_SECTION@@@Z 10045928 f i toolbox:toolbox_i.obj
 0001:00044948       ??1UNSYNCBLOCK_Implementation@@QAA@XZ 10045948 f i toolbox:toolbox_i.obj
 0001:0004495c       ?_tcsncpyz@@YAPAGQAGQBGI@Z 1004595c f   toolbox:toolbox_i.obj
 0001:000449b4       ?_tcsncatz@@YAPAGQAGQBGI@Z 100459b4 f   toolbox:toolbox_i.obj
 0001:00044a1c       ?strncpyz@@YAPADQADQBDI@Z  10045a1c f   toolbox:toolbox_i.obj
 0001:00044a74       ?strncatz@@YAPADQADQBDI@Z  10045a74 f   toolbox:toolbox_i.obj
 0001:00044adc       ?wcsncpyz@@YAPAGQAGQBGI@Z  10045adc f   toolbox:toolbox_i.obj
 0001:00044b34       ?wcsncatz@@YAPAGQAGQBGI@Z  10045b34 f   toolbox:toolbox_i.obj
 0001:00044b9c       ?_sntprintfz@@YAHQAGIQBGZZ 10045b9c f   toolbox:toolbox_i.obj
 0001:00044c08       ?_snprintfz@@YAHQADIQBDZZ  10045c08 f   toolbox:toolbox_i.obj
 0001:00044c74       ?_snwprintfz@@YAHQAGIQBGZZ 10045c74 f   toolbox:toolbox_i.obj
 0001:00044ce0       ?GetRegistryDWORD@@YA_NQAUHKEY__@@QBG1QAK@Z 10045ce0 f   toolbox:toolbox_i.obj
 0001:00044da0       ?SetRegistryDWORD@@YA_NQAUHKEY__@@QBG1K@Z 10045da0 f   toolbox:toolbox_i.obj
 0001:00044e44       ?GetRegistryBoolean@@YA_NQAUHKEY__@@QBG1QA_N@Z 10045e44 f   toolbox:toolbox_i.obj
 0001:00044e90       ?SetRegistryBoolean@@YA_NQAUHKEY__@@QBG1_N@Z 10045e90 f   toolbox:toolbox_i.obj
 0001:00044eac       ?GetRegistryBINARY@@YA_NQAUHKEY__@@QBG1QAEK@Z 10045eac f   toolbox:toolbox_i.obj
 0001:00044f5c       ?SetRegistryBINARY@@YA_NQAUHKEY__@@QBG1QBEK@Z 10045f5c f   toolbox:toolbox_i.obj
 0001:00044ffc       ?GetRegistrySZ@@YA_NQAUHKEY__@@QBG1QAGK@Z 10045ffc f   toolbox:toolbox_i.obj
 0001:000450b0       ?SetRegistrySZ@@YA_NQAUHKEY__@@QBG11@Z 100460b0 f   toolbox:toolbox_i.obj
 0001:0004515c       ?BoundedRandom@@YAHHH@Z    1004615c f   toolbox:toolbox_i.obj
 0001:000451ec       ??0ResourceString@@QAA@XZ  100461ec f   toolbox:toolbox_i.obj
 0001:000451f8       ??BResourceString@@QAAPBGXZ 100461f8 f   toolbox:toolbox_i.obj
 0001:00045210       ??1ResourceString@@QAA@XZ  10046210 f   toolbox:toolbox_i.obj
 0001:00045224       ??0CommandLineTokenizer@@QAA@XZ 10046224 f   toolbox:toolbox_i.obj
 0001:00045234       ??1CommandLineTokenizer@@QAA@XZ 10046234 f   toolbox:toolbox_i.obj
 0001:00045250       ?SetCommandLine@CommandLineTokenizer@@QAA_NPBG@Z 10046250 f   toolbox:toolbox_i.obj
 0001:000452d0       ?NextParameter@CommandLineTokenizer@@QAAPAGXZ 100462d0 f   toolbox:toolbox_i.obj
 0001:00045428       ??0CommandLineParameterHandler@@QAA@QBGQAPBGQAP6A_N0@ZQ6A_N0@Z@Z 10046428 f   toolbox:toolbox_i.obj
 0001:00045464       ?ProcessParameters@CommandLineParameterHandler@@QAA_NXZ 10046464 f   toolbox:toolbox_i.obj
 0001:00045560       ??0AnsiString@@QAA@QBGG@Z  10046560 f   toolbox:toolbox_i.obj
 0001:0004565c       ??0AnsiString@@QAA@QBDD@Z  1004665c f   toolbox:toolbox_i.obj
 0001:000456dc       ??1AnsiString@@QAA@XZ      100466dc f   toolbox:toolbox_i.obj
 0001:000456f8       ??0WideString@@QAA@QBDD@Z  100466f8 f   toolbox:toolbox_i.obj
 0001:000457e0       ??0WideString@@QAA@QBGG@Z  100467e0 f   toolbox:toolbox_i.obj
 0001:00045864       ??1WideString@@QAA@XZ      10046864 f   toolbox:toolbox_i.obj
 0001:00045880       ??0USAsciiString@@QAA@PBG@Z 10046880 f   toolbox:toolbox_i.obj
 0001:00045908       ??0USAsciiString@@QAA@QBD@Z 10046908 f   toolbox:toolbox_i.obj
 0001:00045958       ??1USAsciiString@@QAA@XZ   10046958 f   toolbox:toolbox_i.obj
 0001:00045974       ??0VerboseString@@QAA@QBGGG@Z 10046974 f   toolbox:toolbox_i.obj
 0001:00045b0c       ??1VerboseString@@QAA@XZ   10046b0c f   toolbox:toolbox_i.obj
 0001:00045b28       ??0PrintableString@@QAA@QBDI_NDD@Z 10046b28 f   toolbox:toolbox_i.obj
 0001:00045cf0       ??1PrintableString@@QAA@XZ 10046cf0 f   toolbox:toolbox_i.obj
 0001:00045d0c       ??0HexString@@QAA@QBDI@Z   10046d0c f   toolbox:toolbox_i.obj
 0001:00045d80       ??1HexString@@QAA@XZ       10046d80 f   toolbox:toolbox_i.obj
 0001:00045d9c       ?GetSize@StringCollection@@UAAHXZ 10046d9c f   toolbox:toolbox_i.obj
 0001:00045dbc       ??0CCheckPoint@@QAA@XZ     10046dbc f   toolbox:toolbox_i.obj
 0001:00045de8       ??1CCheckPoint@@QAA@XZ     10046de8 f   toolbox:toolbox_i.obj
 0001:00045e38       ?Init@CCheckPoint@@QAA_NI@Z 10046e38 f   toolbox:toolbox_i.obj
 0001:00045ea4       ?Reached@CCheckPoint@@QAAXXZ 10046ea4 f   toolbox:toolbox_i.obj
 0001:00045ef0       ?Wait@CCheckPoint@@QAA_NK@Z 10046ef0 f   toolbox:toolbox_i.obj
 0001:00045f54       ?bsearch@@YAPAXPBX0IIP6AH00@Z@Z 10046f54 f   toolbox:toolbox_i.obj
 0001:00046008       ?MemoryReadable@@YA_NPBXI@Z 10047008 f   toolbox:toolbox_i.obj
 0001:00046038       ?MemoryWriteable@@YA_NPAXI@Z 10047038 f   toolbox:toolbox_i.obj
 0001:00046070       ?_tcsReadable@@YA_NPBG@Z   10047070 f   toolbox:toolbox_i.obj
 0001:000460bc       ?_tcsWriteable@@YA_NPAG@Z  100470bc f   toolbox:toolbox_i.obj
 0001:00046114       ?strReadable@@YA_NPBD@Z    10047114 f   toolbox:toolbox_i.obj
 0001:00046160       ?strWriteable@@YA_NPAD@Z   10047160 f   toolbox:toolbox_i.obj
 0001:000461b4       ?wcsReadable@@YA_NPBG@Z    100471b4 f   toolbox:toolbox_i.obj
 0001:00046200       ?wcsWriteable@@YA_NPAG@Z   10047200 f   toolbox:toolbox_i.obj
 0001:00046250       ?RemoveTask@TaskList@@QAA_NI@Z 10047250 f   toolbox:toolbox_i.obj
 0001:000463e8       ?TasksRemaining@TaskList@@QAAIXZ 100473e8 f   toolbox:toolbox_i.obj
 0001:00046468       ?TaskListThreadProc@@YAKPAX@Z 10047468 f   toolbox:toolbox_i.obj
 0001:00046630       ??0WorkerThread@@QAA@Q6AKPAX0@ZQAXK@Z 10047630 f   toolbox:toolbox_i.obj
 0001:00046648       ?StopWorkerThread@WorkerThread@@QAA_NXZ 10047648 f   toolbox:toolbox_i.obj
 0001:000466cc       ?RunWorkerThreadProc@WorkerThread@@CAKPAX@Z 100476cc f   toolbox:toolbox_i.obj
 0001:00046700       ??0MemoryMappedFileData@@QAA@XZ 10047700 f   toolbox:toolbox_i.obj
 0001:00046720       ??1MemoryMappedFileData@@QAA@XZ 10047720 f   toolbox:toolbox_i.obj
 0001:0004675c       ?Initialize@MemoryMappedFileData@@QAA_NQBG@Z 1004775c f   toolbox:toolbox_i.obj
 0001:00046834       ??0StringBuffer@@QAA@I@Z   10047834 f   toolbox:toolbox_i.obj
 0001:00046848       ?Empty@StringBuffer@@QAAXXZ 10047848 f   toolbox:toolbox_i.obj
 0001:00046860       ?FreeMemory@StringBuffer@@QAAXXZ 10047860 f   toolbox:toolbox_i.obj
 0001:00046894       ?EnsureSpaceToAddStringLength@StringBuffer@@AAA_NI@Z 10047894 f   toolbox:toolbox_i.obj
 0001:0004695c       ?GetSystemTimeAsFileTime@@YAXPAU_FILETIME@@@Z 1004795c f   toolbox:toolbox_i.obj
 0001:00046988       ?GetPointerAtIndex@?$GrowablePointerCollection@G@@QAAPAGH@Z 10047988 f i toolbox:toolbox_i.obj
 0001:000469cc       ?GetPointerIndex@?$GrowablePointerCollection@G@@QAAHPBG@Z 100479cc f i toolbox:toolbox_i.obj
 0001:00046a30       ??1?$GrowableThingCollection@PAG@@UAA@XZ 10047a30 f i toolbox:toolbox_i.obj
 0001:00046a6c       ?AddThing@?$GrowableThingCollection@PAG@@UAA_NQAG@Z 10047a6c f i toolbox:toolbox_i.obj
 0001:00046ae4       ?InsertThing@?$GrowableThingCollection@PAG@@UAA_NQAGH@Z 10047ae4 f i toolbox:toolbox_i.obj
 0001:00046b94       ?RemoveThingAtIndex@?$GrowableThingCollection@PAG@@UAA_NH@Z 10047b94 f i toolbox:toolbox_i.obj
 0001:00046c1c       ?RemoveThing@?$GrowableThingCollection@PAG@@UAA_NQAG@Z 10047c1c f i toolbox:toolbox_i.obj
 0001:00046cb4       ?RemoveAllThings@?$GrowableThingCollection@PAG@@UAA_NXZ 10047cb4 f i toolbox:toolbox_i.obj
 0001:00046d00       ?SwapThingsAtIndices@?$GrowableThingCollection@PAG@@UAA_NHH@Z 10047d00 f i toolbox:toolbox_i.obj
 0001:00046d8c       ?GetSize@?$GrowableThingCollection@PAG@@UAAHXZ 10047d8c f i toolbox:toolbox_i.obj
 0001:00046db4       ?Lock@?$GrowableThingCollection@PAG@@UAA_NXZ 10047db4 f i toolbox:toolbox_i.obj
 0001:00046de4       ?Unlock@?$GrowableThingCollection@PAG@@UAA_NXZ 10047de4 f i toolbox:toolbox_i.obj
 0001:00046e28       ?BlockModificationByOtherThreads@?$GrowableThingCollection@PAG@@UAA_NXZ 10047e28 f i toolbox:toolbox_i.obj
 0001:00046e40       ?AllowModificationByOtherThreads@?$GrowableThingCollection@PAG@@UAA_NXZ 10047e40 f i toolbox:toolbox_i.obj
 0001:00046e58       ?GetThingAtIndex@?$GrowableThingCollection@PAG@@UAAPAGH@Z 10047e58 f i toolbox:toolbox_i.obj
 0001:00046eb0       ?SetThingAtIndex@?$GrowableThingCollection@PAG@@UAA_NQAGH@Z 10047eb0 f i toolbox:toolbox_i.obj
 0001:00046efc       ?GetThingIndex@?$GrowableThingCollection@PAG@@UAAHQAG@Z 10047efc f i toolbox:toolbox_i.obj
 0001:00046f70       ?GetFilteredThingIndex@?$GrowableThingCollection@PAG@@UAAHP6A_NABQAGPAX@ZQAX@Z 10047f70 f i toolbox:toolbox_i.obj
 0001:00046fe0       ?GetPointerToThingAtIndex@?$GrowableThingCollection@PAG@@UAAPAPAGH@Z 10047fe0 f i toolbox:toolbox_i.obj
 0001:00047030       ?GetPointerToThing@?$GrowableThingCollection@PAG@@UAAPAPAGQAG@Z 10048030 f i toolbox:toolbox_i.obj
 0001:000470a4       ?MakeRoomForAnotherThing@?$GrowableThingCollection@PAG@@MAA_NXZ 100480a4 f i toolbox:toolbox_i.obj
 0001:00047108       ??0?$GrowableThingCollection@PAX@@QAA@H@Z 10048108 f i toolbox:toolbox_i.obj
 0001:00047158       ??1?$GrowableThingCollection@PAX@@UAA@XZ 10048158 f i toolbox:toolbox_i.obj
 0001:00047194       ?AddThing@?$GrowableThingCollection@PAX@@UAA_NQAX@Z 10048194 f i toolbox:toolbox_i.obj
 0001:0004720c       ?InsertThing@?$GrowableThingCollection@PAX@@UAA_NQAXH@Z 1004820c f i toolbox:toolbox_i.obj
 0001:000472bc       ?RemoveThingAtIndex@?$GrowableThingCollection@PAX@@UAA_NH@Z 100482bc f i toolbox:toolbox_i.obj
 0001:00047344       ?RemoveThing@?$GrowableThingCollection@PAX@@UAA_NQAX@Z 10048344 f i toolbox:toolbox_i.obj
 0001:000473dc       ?RemoveAllThings@?$GrowableThingCollection@PAX@@UAA_NXZ 100483dc f i toolbox:toolbox_i.obj
 0001:00047428       ?SwapThingsAtIndices@?$GrowableThingCollection@PAX@@UAA_NHH@Z 10048428 f i toolbox:toolbox_i.obj
 0001:000474b4       ?GetSize@?$GrowableThingCollection@PAX@@UAAHXZ 100484b4 f i toolbox:toolbox_i.obj
 0001:000474dc       ?Lock@?$GrowableThingCollection@PAX@@UAA_NXZ 100484dc f i toolbox:toolbox_i.obj
 0001:0004750c       ?Unlock@?$GrowableThingCollection@PAX@@UAA_NXZ 1004850c f i toolbox:toolbox_i.obj
 0001:00047550       ?BlockModificationByOtherThreads@?$GrowableThingCollection@PAX@@UAA_NXZ 10048550 f i toolbox:toolbox_i.obj
 0001:00047568       ?AllowModificationByOtherThreads@?$GrowableThingCollection@PAX@@UAA_NXZ 10048568 f i toolbox:toolbox_i.obj
 0001:00047580       ?GetThingAtIndex@?$GrowableThingCollection@PAX@@UAAPAXH@Z 10048580 f i toolbox:toolbox_i.obj
 0001:000475d8       ?SetThingAtIndex@?$GrowableThingCollection@PAX@@UAA_NQAXH@Z 100485d8 f i toolbox:toolbox_i.obj
 0001:00047624       ?GetThingIndex@?$GrowableThingCollection@PAX@@UAAHQAX@Z 10048624 f i toolbox:toolbox_i.obj
 0001:00047698       ?GetFilteredThingIndex@?$GrowableThingCollection@PAX@@UAAHP6A_NABQAXPAX@ZQAX@Z 10048698 f i toolbox:toolbox_i.obj
 0001:00047708       ?GetPointerToThingAtIndex@?$GrowableThingCollection@PAX@@UAAPAPAXH@Z 10048708 f i toolbox:toolbox_i.obj
 0001:00047758       ?GetPointerToThing@?$GrowableThingCollection@PAX@@UAAPAPAXQAX@Z 10048758 f i toolbox:toolbox_i.obj
 0001:000477cc       ?MakeRoomForAnotherThing@?$GrowableThingCollection@PAX@@MAA_NXZ 100487cc f i toolbox:toolbox_i.obj
 0001:00047830       ??0?$GrowableThingCollection@UTaskListTaskData@TaskList@@@@QAA@H@Z 10048830 f i toolbox:toolbox_i.obj
 0001:00047880       ??1?$GrowableThingCollection@UTaskListTaskData@TaskList@@@@UAA@XZ 10048880 f i toolbox:toolbox_i.obj
 0001:000478bc       ?AddThing@?$GrowableThingCollection@UTaskListTaskData@TaskList@@@@UAA_NUTaskListTaskData@TaskList@@@Z 100488bc f i toolbox:toolbox_i.obj
 0001:00047954       ?InsertThing@?$GrowableThingCollection@UTaskListTaskData@TaskList@@@@UAA_NUTaskListTaskData@TaskList@@H@Z 10048954 f i toolbox:toolbox_i.obj
 0001:00047a24       ?RemoveThingAtIndex@?$GrowableThingCollection@UTaskListTaskData@TaskList@@@@UAA_NH@Z 10048a24 f i toolbox:toolbox_i.obj
 0001:00047ab4       ?RemoveThing@?$GrowableThingCollection@UTaskListTaskData@TaskList@@@@UAA_NUTaskListTaskData@TaskList@@@Z 10048ab4 f i toolbox:toolbox_i.obj
 0001:00047b6c       ?RemoveAllThings@?$GrowableThingCollection@UTaskListTaskData@TaskList@@@@UAA_NXZ 10048b6c f i toolbox:toolbox_i.obj
 0001:00047bb8       ?SwapThingsAtIndices@?$GrowableThingCollection@UTaskListTaskData@TaskList@@@@UAA_NHH@Z 10048bb8 f i toolbox:toolbox_i.obj
 0001:00047c74       ?GetSize@?$GrowableThingCollection@UTaskListTaskData@TaskList@@@@UAAHXZ 10048c74 f i toolbox:toolbox_i.obj
 0001:00047c9c       ?Lock@?$GrowableThingCollection@UTaskListTaskData@TaskList@@@@UAA_NXZ 10048c9c f i toolbox:toolbox_i.obj
 0001:00047ccc       ?Unlock@?$GrowableThingCollection@UTaskListTaskData@TaskList@@@@UAA_NXZ 10048ccc f i toolbox:toolbox_i.obj
 0001:00047d10       ?BlockModificationByOtherThreads@?$GrowableThingCollection@UTaskListTaskData@TaskList@@@@UAA_NXZ 10048d10 f i toolbox:toolbox_i.obj
 0001:00047d28       ?AllowModificationByOtherThreads@?$GrowableThingCollection@UTaskListTaskData@TaskList@@@@UAA_NXZ 10048d28 f i toolbox:toolbox_i.obj
 0001:00047d40       ?GetThingAtIndex@?$GrowableThingCollection@UTaskListTaskData@TaskList@@@@UAA?AUTaskListTaskData@TaskList@@H@Z 10048d40 f i toolbox:toolbox_i.obj
 0001:00047dbc       ?SetThingAtIndex@?$GrowableThingCollection@UTaskListTaskData@TaskList@@@@UAA_NUTaskListTaskData@TaskList@@H@Z 10048dbc f i toolbox:toolbox_i.obj
 0001:00047e24       ?GetThingIndex@?$GrowableThingCollection@UTaskListTaskData@TaskList@@@@UAAHUTaskListTaskData@TaskList@@@Z 10048e24 f i toolbox:toolbox_i.obj
 0001:00047e98       ?GetFilteredThingIndex@?$GrowableThingCollection@UTaskListTaskData@TaskList@@@@UAAHP6A_NABUTaskListTaskData@TaskList@@PAX@ZQAX@Z 10048e98 f i toolbox:toolbox_i.obj
 0001:00047f10       ?GetPointerToThingAtIndex@?$GrowableThingCollection@UTaskListTaskData@TaskList@@@@UAAPAUTaskListTaskData@TaskList@@H@Z 10048f10 f i toolbox:toolbox_i.obj
 0001:00047f64       ?GetPointerToThing@?$GrowableThingCollection@UTaskListTaskData@TaskList@@@@UAAPAUTaskListTaskData@TaskList@@U23@@Z 10048f64 f i toolbox:toolbox_i.obj
 0001:00047fe4       ?MakeRoomForAnotherThing@?$GrowableThingCollection@UTaskListTaskData@TaskList@@@@MAA_NXZ 10048fe4 f i toolbox:toolbox_i.obj
 0001:0004804c       ??_G?$GrowableThingCollection@PAG@@UAAPAXI@Z 1004904c f i toolbox:toolbox_i.obj
 0001:0004804c       ??_E?$GrowableThingCollection@PAG@@UAAPAXI@Z 1004904c f i toolbox:toolbox_i.obj
 0001:00048074       ??_G?$GrowableThingCollection@PAX@@UAAPAXI@Z 10049074 f i toolbox:toolbox_i.obj
 0001:00048074       ??_E?$GrowableThingCollection@PAX@@UAAPAXI@Z 10049074 f i toolbox:toolbox_i.obj
 0001:0004809c       ??_G?$GrowableThingCollection@UTaskListTaskData@TaskList@@@@UAAPAXI@Z 1004909c f i toolbox:toolbox_i.obj
 0001:0004809c       ??_E?$GrowableThingCollection@UTaskListTaskData@TaskList@@@@UAAPAXI@Z 1004909c f i toolbox:toolbox_i.obj
 0001:000480c4       ??0?$GrowableThingCollection@PAG@@QAA@H@Z 100490c4 f i toolbox:toolbox_i.obj
 0001:00048114       ?LoadResourceString@ResourceString@@QAAPBGPAUHINSTANCE__@@I@Z 10049114 f   toolbox:toolbox_i.obj
 0001:00048180       ??0CommandLineTokenizer@@QAA@PBG@Z 10049180 f   toolbox:toolbox_i.obj
 0001:000481a0       ?GetString@StringCollection@@UAAPAGH@Z 100491a0 f   toolbox:toolbox_i.obj
 0001:000481b4       ?FindStringIndex@SortedStringCollection@@QAAHQBG@Z 100491b4 f   toolbox:toolbox_i.obj
 0001:00048248       ??0TaskList@@QAA@I@Z       10049248 f   toolbox:toolbox_i.obj
 0001:000482f0       ??1TaskList@@QAA@XZ        100492f0 f   toolbox:toolbox_i.obj
 0001:000483a8       ?AddWorkerThread@TaskList@@AAA_NXZ 100493a8 f   toolbox:toolbox_i.obj
 0001:00048440       ??1WorkerThread@@QAA@XZ    10049440 f   toolbox:toolbox_i.obj
 0001:00048450       ?StartWorkerThread@WorkerThread@@QAA_NXZ 10049450 f   toolbox:toolbox_i.obj
 0001:0004851c       ??1StringBuffer@@QAA@XZ    1004951c f   toolbox:toolbox_i.obj
 0001:0004852c       ?Set@StringBuffer@@QAA_NQBG@Z 1004952c f   toolbox:toolbox_i.obj
 0001:00048584       ?Append@StringBuffer@@QAA_NQBG@Z 10049584 f   toolbox:toolbox_i.obj
 0001:000485ec       ?Append@StringBuffer@@QAA_NQBGI@Z 100495ec f   toolbox:toolbox_i.obj
 0001:00048660       ??0?$GrowablePointerCollection@G@@QAA@H@Z 10049660 f i toolbox:toolbox_i.obj
 0001:000486a4       ?RemoveThingAtIndex@?$GrowablePointerCollection@G@@UAA_NH@Z 100496a4 f i toolbox:toolbox_i.obj
 0001:000486ac       ?RemoveAllThings@?$GrowablePointerCollection@G@@UAA_NXZ 100496ac f i toolbox:toolbox_i.obj
 0001:000486b4       ?SwapThingsAtIndices@?$GrowablePointerCollection@G@@UAA_NHH@Z 100496b4 f i toolbox:toolbox_i.obj
 0001:000486bc       ?GetThingAtIndex@?$GrowablePointerCollection@G@@UAAPAGH@Z 100496bc f i toolbox:toolbox_i.obj
 0001:000486c4       ?GetFilteredThingIndex@?$GrowablePointerCollection@G@@UAAHP6A_NABQAGPAX@ZQAX@Z 100496c4 f i toolbox:toolbox_i.obj
 0001:000486cc       ?GetPointerToThingAtIndex@?$GrowablePointerCollection@G@@UAAPAPAGH@Z 100496cc f i toolbox:toolbox_i.obj
 0001:000486d4       ??1?$GrowablePointerCollection@G@@UAA@XZ 100496d4 f i toolbox:toolbox_i.obj
 0001:00048708       ?AddPointer@?$GrowablePointerCollection@G@@QAA_NQBG@Z 10049708 f i toolbox:toolbox_i.obj
 0001:00048718       ?InsertPointer@?$GrowablePointerCollection@G@@QAA_NQBGH@Z 10049718 f i toolbox:toolbox_i.obj
 0001:00048728       ??_G?$GrowablePointerCollection@G@@UAAPAXI@Z 10049728 f i toolbox:toolbox_i.obj
 0001:00048728       ??_E?$GrowablePointerCollection@G@@UAAPAXI@Z 10049728 f i toolbox:toolbox_i.obj
 0001:00048770       ??0ResourceString@@QAA@PAUHINSTANCE__@@I@Z 10049770 f   toolbox:toolbox_i.obj
 0001:00048790       ??0StringCollection@@QAA@XZ 10049790 f   toolbox:toolbox_i.obj
 0001:000487b8       ??1StringCollection@@UAA@XZ 100497b8 f   toolbox:toolbox_i.obj
 0001:000487f8       ?AddString@StringCollection@@UAA_NQBGQAH@Z 100497f8 f   toolbox:toolbox_i.obj
 0001:00048850       ??0SortedStringCollection@@QAA@_N@Z 10049850 f   toolbox:toolbox_i.obj
 0001:000488a0       ??1SortedStringCollection@@UAA@XZ 100498a0 f   toolbox:toolbox_i.obj
 0001:000488c0       ?AddString@SortedStringCollection@@UAA_NQBG_N@Z 100498c0 f   toolbox:toolbox_i.obj
 0001:00048990       ?AddTask@TaskList@@QAA_NPAIP6A_NPAX@Z1W4TaskListUrgency@1@@Z 10049990 f   toolbox:toolbox_i.obj
 0001:00048ad8       ??_GStringCollection@@UAAPAXI@Z 10049ad8 f i toolbox:toolbox_i.obj
 0001:00048ad8       ??_EStringCollection@@UAAPAXI@Z 10049ad8 f i toolbox:toolbox_i.obj
 0001:00048b00       ??_GSortedStringCollection@@UAAPAXI@Z 10049b00 f i toolbox:toolbox_i.obj
 0001:00048b00       ??_ESortedStringCollection@@UAAPAXI@Z 10049b00 f i toolbox:toolbox_i.obj
 0001:00048b34       ?TBD_Assert@@YA_N_NQBG1H@Z 10049b34 f   sw_utilityG:sw_utilityG.dll
 0001:00048b44       ?LogC@@YAXPBGZZ            10049b44 f   sw_utilityG:sw_utilityG.dll
 0001:00048b54       ?LogStoreFileLine@@YAXPAGH@Z 10049b54 f   sw_utilityG:sw_utilityG.dll
 0001:00048b64       ?WriteLog@@YAXKPBGZZ       10049b64 f   sw_utilityG:sw_utilityG.dll
 0001:00048b74       ?GetRegValue@@YAJPAUHKEY__@@PBG1PAGPAK@Z 10049b74 f   sw_utilityG:sw_utilityG.dll
 0001:00048b84       ?LogW@@YAXPBGZZ            10049b84 f   sw_utilityG:sw_utilityG.dll
 0001:00048b94       ?SW_AtoT@@YAPAGPAGPADK@Z   10049b94 f   sw_utilityG:sw_utilityG.dll
 0001:00048ba4       ?TBD_Output@@YAXW4TBD_CLASS_TYPE@@W4TBD_OUTPUT_LEVEL@@QBGZZ 10049ba4 f   sw_utilityG:sw_utilityG.dll
 0001:00048bb4       ?SW_TtoA@@YAPADPADPAGK@Z   10049bb4 f   sw_utilityG:sw_utilityG.dll
 0001:00048bc4       ?DisplayRawData@@YAXIPAEHPBG@Z 10049bc4 f   sw_utilityG:sw_utilityG.dll
 0001:00048bd4       __rt_udiv                  10049bd4 f   coredll:COREDLL.dll
 0001:00048be4       strlen                     10049be4 f   coredll:COREDLL.dll
 0001:00048bf4       strstr                     10049bf4 f   coredll:COREDLL.dll
 0001:00048c04       strcmp                     10049c04 f   coredll:COREDLL.dll
 0001:00048c14       memcmp                     10049c14 f   coredll:COREDLL.dll
 0001:00048c24       strspn                     10049c24 f   coredll:COREDLL.dll
 0001:00048c34       LocalFree                  10049c34 f   coredll:COREDLL.dll
 0001:00048c44       LocalAllocTrace            10049c44 f   coredll:COREDLL.dll
 0001:00048c54       strchr                     10049c54 f   coredll:COREDLL.dll
 0001:00048c64       wcslen                     10049c64 f   coredll:COREDLL.dll
 0001:00048c74       ??3@YAXPAX@Z               10049c74 f   coredll:COREDLL.dll
 0001:00048c84       ??2@YAPAXI@Z               10049c84 f   coredll:COREDLL.dll
 0001:00048c94       memset                     10049c94 f   coredll:COREDLL.dll
 0001:00048ca4       NKDbgPrintfW               10049ca4 f   coredll:COREDLL.dll
 0001:00048cb4       EnterCriticalSection       10049cb4 f   coredll:COREDLL.dll
 0001:00048cc4       LeaveCriticalSection       10049cc4 f   coredll:COREDLL.dll
 0001:00048cd4       GetLastError               10049cd4 f   coredll:COREDLL.dll
 0001:00048ce4       swscanf                    10049ce4 f   coredll:COREDLL.dll
 0001:00048cf4       _snprintf                  10049cf4 f   coredll:COREDLL.dll
 0001:00048d04       ??_V@YAXPAX@Z              10049d04 f   coredll:COREDLL.dll
 0001:00048d14       ??_U@YAPAXI@Z              10049d14 f   coredll:COREDLL.dll
 0001:00048d24       sscanf                     10049d24 f   coredll:COREDLL.dll
 0001:00048d34       free                       10049d34 f   coredll:COREDLL.dll
 0001:00048d44       malloc                     10049d44 f   coredll:COREDLL.dll
 0001:00048d54       CloseHandle                10049d54 f   coredll:COREDLL.dll
 0001:00048d64       CreateThread               10049d64 f   coredll:COREDLL.dll
 0001:00048d74       InitializeCriticalSection  10049d74 f   coredll:COREDLL.dll
 0001:00048d84       DeleteCriticalSection      10049d84 f   coredll:COREDLL.dll
 0001:00048d94       Sleep                      10049d94 f   coredll:COREDLL.dll
 0001:00048da4       strtoul                    10049da4 f   coredll:COREDLL.dll
 0001:00048db4       abs                        10049db4 f   coredll:COREDLL.dll
 0001:00048dc4       strncpy                    10049dc4 f   coredll:COREDLL.dll
 0001:00048dd4       __rt_udiv64by64            10049dd4 f   coredll:COREDLL.dll
 0001:00048de4       memcpy                     10049de4 f   coredll:COREDLL.dll
 0001:00048df4       wcscmp                     10049df4 f   coredll:COREDLL.dll
 0001:00048e04       wcsncpy                    10049e04 f   coredll:COREDLL.dll
 0001:00048e14       MultiByteToWideChar        10049e14 f   coredll:COREDLL.dll
 0001:00048e24       wcsstr                     10049e24 f   coredll:COREDLL.dll
 0001:00048e34       sprintf                    10049e34 f   coredll:COREDLL.dll
 0001:00048e44       wcscpy                     10049e44 f   coredll:COREDLL.dll
 0001:00048e54       atol                       10049e54 f   coredll:COREDLL.dll
 0001:00048e64       strcat                     10049e64 f   coredll:COREDLL.dll
 0001:00048e74       strcpy                     10049e74 f   coredll:COREDLL.dll
 0001:00048e84       __rt_sdiv                  10049e84 f   coredll:COREDLL.dll
 0001:00048e94       _wtol                      10049e94 f   coredll:COREDLL.dll
 0001:00048ea4       swprintf                   10049ea4 f   coredll:COREDLL.dll
 0001:00048eb4       PurgeComm                  10049eb4 f   coredll:COREDLL.dll
 0001:00048ec4       SetCommState               10049ec4 f   coredll:COREDLL.dll
 0001:00048ed4       toupper                    10049ed4 f   coredll:COREDLL.dll
 0001:00048ee4       SetupComm                  10049ee4 f   coredll:COREDLL.dll
 0001:00048ef4       SetCommTimeouts            10049ef4 f   coredll:COREDLL.dll
 0001:00048f04       GetCommState               10049f04 f   coredll:COREDLL.dll
 0001:00048f14       SetLastError               10049f14 f   coredll:COREDLL.dll
 0001:00048f24       CreateFileW                10049f24 f   coredll:COREDLL.dll
 0001:00048f34       wcscat                     10049f34 f   coredll:COREDLL.dll
 0001:00048f44       WriteFile                  10049f44 f   coredll:COREDLL.dll
 0001:00048f54       ReadFile                   10049f54 f   coredll:COREDLL.dll
 0001:00048f64       GetTickCount               10049f64 f   coredll:COREDLL.dll
 0001:00048f74       GetProcAddressW            10049f74 f   coredll:COREDLL.dll
 0001:00048f84       FreeLibrary                10049f84 f   coredll:COREDLL.dll
 0001:00048f94       LoadLibraryW               10049f94 f   coredll:COREDLL.dll
 0001:00048fa4       __CxxThrowException        10049fa4 f   coredll:COREDLL.dll
 0001:00048fb4       ??_7type_info@@6B@         10049fb4 f   coredll:COREDLL.dll
 0001:00048fc4       ??0exception@std@@QAA@ABV01@@Z 10049fc4 f   coredll:COREDLL.dll
 0001:00048fd4       ??1exception@std@@UAA@XZ   10049fd4 f   coredll:COREDLL.dll
 0001:00048fe4       ??0exception@std@@QAA@XZ   10049fe4 f   coredll:COREDLL.dll
 0001:00048ff4       ??0exception@std@@QAA@PBD@Z 10049ff4 f   coredll:COREDLL.dll
 0001:00049004       ?what@exception@std@@UBAPBDXZ 1004a004 f   coredll:COREDLL.dll
 0001:00049014       StringCchCopyW             1004a014 f   coredll:COREDLL.dll
 0001:00049024       wcschr                     1004a024 f   coredll:COREDLL.dll
 0001:00049034       __report_gsfailure         1004a034 f   coredll:COREDLL.dll
 0001:00049044       LocalReAlloc               1004a044 f   coredll:COREDLL.dll
 0001:00049054       LocalAlloc                 1004a054 f   coredll:COREDLL.dll
 0001:00049064       LocalSize                  1004a064 f   coredll:COREDLL.dll
 0001:00049074       __security_gen_cookie      1004a074 f   coredll:COREDLL.dll
 0001:00049084       EventModify                1004a084 f   coredll:COREDLL.dll
 0001:00049094       StringCchVPrintfW          1004a094 f   coredll:COREDLL.dll
 0001:000490a4       StringCchVPrintfA          1004a0a4 f   coredll:COREDLL.dll
 0001:000490b4       RegCloseKey                1004a0b4 f   coredll:COREDLL.dll
 0001:000490c4       RegQueryValueExW           1004a0c4 f   coredll:COREDLL.dll
 0001:000490d4       RegCreateKeyExW            1004a0d4 f   coredll:COREDLL.dll
 0001:000490e4       RegSetValueExW             1004a0e4 f   coredll:COREDLL.dll
 0001:000490f4       rand                       1004a0f4 f   coredll:COREDLL.dll
 0001:00049104       __itos                     1004a104 f   coredll:COREDLL.dll
 0001:00049114       __muls                     1004a114 f   coredll:COREDLL.dll
 0001:00049124       __stoi                     1004a124 f   coredll:COREDLL.dll
 0001:00049134       _wcsnicmp                  1004a134 f   coredll:COREDLL.dll
 0001:00049144       WideCharToMultiByte        1004a144 f   coredll:COREDLL.dll
 0001:00049154       CreateEventW               1004a154 f   coredll:COREDLL.dll
 0001:00049164       WaitForSingleObject        1004a164 f   coredll:COREDLL.dll
 0001:00049174       __C_specific_handler       1004a174 f   coredll:COREDLL.dll
 0001:00049184       WaitForMultipleObjects     1004a184 f   coredll:COREDLL.dll
 0001:00049194       InterlockedDecrement       1004a194 f   coredll:COREDLL.dll
 0001:000491a4       InterlockedIncrement       1004a1a4 f   coredll:COREDLL.dll
 0001:000491b4       UnmapViewOfFile            1004a1b4 f   coredll:COREDLL.dll
 0001:000491c4       MapViewOfFile              1004a1c4 f   coredll:COREDLL.dll
 0001:000491d4       CreateFileMappingW         1004a1d4 f   coredll:COREDLL.dll
 0001:000491e4       GetFileSize                1004a1e4 f   coredll:COREDLL.dll
 0001:000491f4       SystemTimeToFileTime       1004a1f4 f   coredll:COREDLL.dll
 0001:00049204       GetSystemTime              1004a204 f   coredll:COREDLL.dll
 0001:00049214       memmove                    1004a214 f   coredll:COREDLL.dll
 0001:00049224       LoadStringW                1004a224 f   coredll:COREDLL.dll
 0001:00049234       CreateSemaphoreW           1004a234 f   coredll:COREDLL.dll
 0001:00049244       _wcsicmp                   1004a244 f   coredll:COREDLL.dll
 0001:00049254       ReleaseSemaphore           1004a254 f   coredll:COREDLL.dll
 0001:00049264       __GSHandlerCheckCommon     1004a264 f   LIBCMTD:gshandler.obj
 0001:000492ac       __GSHandlerCheck           1004a2ac f   LIBCMTD:gshandler.obj
 0001:000492dc       strcpy_s                   1004a2dc f   LIBCMTD:strcpy_s.obj
 0001:00049730       __InternalCxxFrameHandler  1004a730 f   LIBCMTD:frame_ce.obj
 0001:0004990c       __CxxFrameHandler3         1004a90c f   LIBCMTD:frame_ce.obj
 0001:0004a0e8       __FrameUnwindToState       1004b0e8 f   LIBCMTD:frame_ce.obj
 0001:0004ae94       ?_DestructExceptionObject@@YAXPAUEHExceptionRecord@@E@Z 1004be94 f   LIBCMTD:frame_ce.obj
 0001:0004afe4       ?_OffsetToAddress@@YAPAXHPAKK@Z 1004bfe4 f   LIBCMTD:frame_ce.obj
 0001:0004b070       ?FindFrameInfo@@YAPAU_FrameInfo@@PAK@Z 1004c070 f   LIBCMTD:frame_ce.obj
 0001:0004b0f8       ?FindCatchFrameInfo@@YAPAU_FrameInfo@@PAK@Z 1004c0f8 f   LIBCMTD:frame_ce.obj
 0001:0004b17c       ?_GetRangeOfTrysToCheck@@YAPBU_s_TryBlockMapEntry@@PBU_s_FuncInfo@@HHPAI1@Z 1004c17c f   LIBCMTD:frame_ce.obj
 0001:0004b274       __GSHandlerCheck_EH        1004c274 f   LIBCMTD:gshandlereh.obj
 0001:0004b308       _invalid_parameter         1004c308 f   LIBCMTD:invarginternal.obj
 0001:0004b354       _CrtSetReportHookT2        1004c354 f   LIBCMTD:dbgrpt.obj
 0001:0004b820       _CrtDbgReportW             1004c820 f   LIBCMTD:dbgrpt.obj
 0001:0004b898       _CrtDbgReportTV            1004c898 f i LIBCMTD:dbgrpt.obj
 0001:0004b8f4       __crtMessageWindowW        1004c8f4 f   LIBCMTD:dbgrpt.obj
 0001:0004bfcc       _invoke_watson_if_error    1004cfcc f i LIBCMTD:dbgrpt.obj
 0001:0004c020       memcpy_s                   1004d020 f   LIBCMTD:memcpy_s.obj
 0001:0004c2d8       memmove_s                  1004d2d8 f   LIBCMTD:memmove_s.obj
 0001:0004c54c       GetCRTStorage              1004d54c f   LIBCMTD:corecrt.obj
 0001:0004c65c       TlsAlloc                   1004d65c f i LIBCMTD:corecrt.obj
 0001:0004c698       TlsFree                    1004d698 f i LIBCMTD:corecrt.obj
 0001:0004c6dc       ?FindFrameForUnwind@@YAPAKPAKPBU_s_FuncInfo@@@Z 1004d6dc f   LIBCMTD:mdframe_arm.obj
 0001:0004c774       ?FindCatchFrame@@YAPAKPAKK@Z 1004d774 f   LIBCMTD:mdframe_arm.obj
 0001:0004c80c       ?AdjustFrameForCatch@@YAPAKPAKPBU_s_FuncInfo@@@Z 1004d80c f   LIBCMTD:mdframe_arm.obj
 0001:0004c8ac       ?GetCurrentState@@YAHPAKPAU_DISPATCHER_CONTEXT@@PBU_s_FuncInfo@@@Z 1004d8ac f   LIBCMTD:ehstate_arm_mips.obj
 0001:0004c988       _CallSettingFrame          1004d988     LIBCMTD:handlers_arm.obj
 0001:0004c9cc       _invoke_watson             1004d9cc f   LIBCMTD:invarg.obj
 0001:0004ca00       _mtinitlocks               1004da00 f   LIBCMTD:mlock.obj
 0001:0004cb18       _mtdeletelocks             1004db18 f   LIBCMTD:mlock.obj
 0001:0004cc9c       _mtinitlocknum             1004dc9c f   LIBCMTD:mlock.obj
 0001:0004ce04       _lock                      1004de04 f   LIBCMTD:mlock.obj
 0001:0004cf00       _unlock                    1004df00 f   LIBCMTD:mlock.obj
 0001:0004cf40       _lockerr_exit              1004df40 f   LIBCMTD:mlock.obj
 0001:0004cf68       _CrtDbgBreak               1004df68 f   LIBCMTD:dbgrptt.obj
 0001:0004cf70       _CrtSetReportMode          1004df70 f   LIBCMTD:dbgrptt.obj
 0001:0004d198       _CrtSetReportFile          1004e198 f   LIBCMTD:dbgrptt.obj
 0001:0004d334       _CrtSetReportHook          1004e334 f   LIBCMTD:dbgrptt.obj
 0001:0004d378       _CrtGetReportHook          1004e378 f   LIBCMTD:dbgrptt.obj
 0001:0004d3a0       _VCrtDbgReportW            1004e3a0 f   LIBCMTD:dbgrptt.obj
 0001:0004df58       __crtMessageBoxW           1004ef58 f   LIBCMTD:crtmbox.obj
 0001:0004e1bc       wcsncpy_s                  1004f1bc f   LIBCMTD:wcsncpy_s.obj
 0001:0004e7bc       wcscpy_s                   1004f7bc f   LIBCMTD:wcscpy_s.obj
 0001:0004ec30       _initp_misc_initcrit       1004fc30 f   LIBCMTD:initcrit.obj
 0001:0004ec5c       __crtInitCritSecAndSpinCount 1004fc5c f   LIBCMTD:initcrit.obj
 0001:0004ed8c       _amsg_exit                 1004fd8c f   LIBCMTD:crt0dat.obj
 0001:0004edb8       __crtExitProcess           1004fdb8 f   LIBCMTD:crt0dat.obj
 0001:0004ee00       wcscat_s                   1004fe00 f   LIBCMTD:wcscat_s.obj
 0001:0004f3e4       _itow_s                    100503e4 f   LIBCMTD:xtows.obj
 0001:0004fa70       _ltow_s                    10050a70 f   LIBCMTD:xtows.obj
 0001:0004faf0       _ultow_s                   10050af0 f   LIBCMTD:xtows.obj
 0001:0004fb44       _encode_pointer            10050b44 f   LIBCMTD:tidtable.obj
 0001:0004fb6c       _encoded_null              10050b6c f   LIBCMTD:tidtable.obj
 0001:0004fba4       _decode_pointer            10050ba4 f   LIBCMTD:tidtable.obj
 0001:0004fbcc       ??0_Init_locks@std@@QAA@XZ 10050bcc f   libcpmtd:xlock.obj
 0001:0004fc2c       ??1_Init_locks@std@@QAA@XZ 10050c2c f   libcpmtd:xlock.obj
 0001:0004fc84       ?_Init_locks_ctor@_Init_locks@std@@CAXPAV12@@Z 10050c84 f   libcpmtd:xlock.obj
 0001:0004fcdc       ?_Init_locks_dtor@_Init_locks@std@@CAXPAV12@@Z 10050cdc f   libcpmtd:xlock.obj
 0001:0004fd34       ??0_Lockit@std@@QAA@XZ     10050d34 f   libcpmtd:xlock.obj
 0001:0004fd68       ??0_Lockit@std@@QAA@H@Z    10050d68 f   libcpmtd:xlock.obj
 0001:0004fda4       ??1_Lockit@std@@QAA@XZ     10050da4 f   libcpmtd:xlock.obj
 0001:0004fdd4       ?_Lockit_ctor@_Lockit@std@@CAXPAV12@@Z 10050dd4 f   libcpmtd:xlock.obj
 0001:0004fdf8       ?_Lockit_ctor@_Lockit@std@@CAXPAV12@H@Z 10050df8 f   libcpmtd:xlock.obj
 0001:0004fe30       ?_Lockit_dtor@_Lockit@std@@CAXPAV12@@Z 10050e30 f   libcpmtd:xlock.obj
 0001:0004fe60       ?_Debug_message@std@@YAXPBD0@Z 10050e60 f   libcpmtd:stdthrow.obj
 0001:0004ff20       ?_Debug_message@std@@YAXPB_W0I@Z 10050f20 f   libcpmtd:stdthrow.obj
 0001:0004ff60       ?_Debug_message@std@@YAXPBG0I@Z 10050f60 f   libcpmtd:stdthrow.obj
 0001:0004ff7c       ?_Throw@std@@YAXABVexception@1@@Z 10050f7c f   libcpmtd:stdthrow.obj
 0001:0004ffb4       ??$_Debug_pointer@D@std@@YAXPBDPB_WI@Z 10050fb4 f i libcpmtd:string.obj
 0001:0004ffdc       ??0invalid_argument@std@@QAA@ABV?$basic_string@DU?$char_traits@D@std@@V?$allocator@D@2@@1@@Z 10050fdc f i libcpmtd:string.obj
 0001:0005000c       ??1invalid_argument@std@@UAA@XZ 1005100c f i libcpmtd:string.obj
 0001:00050038       ??_Einvalid_argument@std@@UAAPAXI@Z 10051038 f i libcpmtd:string.obj
 0001:00050038       ??_Ginvalid_argument@std@@UAAPAXI@Z 10051038 f i libcpmtd:string.obj
 0001:00050084       ??0out_of_range@std@@QAA@ABV?$basic_string@DU?$char_traits@D@std@@V?$allocator@D@2@@1@@Z 10051084 f i libcpmtd:string.obj
 0001:000500b4       ??1out_of_range@std@@UAA@XZ 100510b4 f i libcpmtd:string.obj
 0001:000500e0       ??_Eout_of_range@std@@UAAPAXI@Z 100510e0 f i libcpmtd:string.obj
 0001:000500e0       ??_Gout_of_range@std@@UAAPAXI@Z 100510e0 f i libcpmtd:string.obj
 0001:00050134       ?_Xlen@_String_base@std@@SAXXZ 10051134 f   libcpmtd:string.obj
 0001:000501c4       ?_Xran@_String_base@std@@SAXXZ 100511c4 f   libcpmtd:string.obj
 0001:0005024c       ??0out_of_range@std@@QAA@ABV01@@Z 1005124c f i libcpmtd:string.obj
 0001:00050284       ?_Xinvarg@_String_base@std@@SAXXZ 10051284 f   libcpmtd:string.obj
 0001:0005030c       ??0invalid_argument@std@@QAA@ABV01@@Z 1005130c f i libcpmtd:string.obj
 0001:0005033c       _Once                      1005133c f   libcpmtd:xmtx.obj
 0001:000503c8       _Mtxinit                   100513c8 f   libcpmtd:xmtx.obj
 0001:000503e4       _Mtxdst                    100513e4 f   libcpmtd:xmtx.obj
 0001:00050400       _Mtxlock                   10051400 f   libcpmtd:xmtx.obj
 0001:0005041c       _Mtxunlock                 1005141c f   libcpmtd:xmtx.obj
 0001:00050438       ?terminate@std@@YAXXZ      10051438 f   coredll:COREDLL.dll
 0001:00050448       _snwprintf                 10051448 f   coredll:COREDLL.dll
 0001:00050458       GetModuleFileNameW         10051458 f   coredll:COREDLL.dll
 0001:00050468       TlsSetValue                10051468 f   coredll:COREDLL.dll
 0001:00050478       TlsGetValue                10051478 f   coredll:COREDLL.dll
 0001:00050488       InterlockedCompareExchange 10051488 f   coredll:COREDLL.dll
 0001:00050498       TlsCall                    10051498 f   coredll:COREDLL.dll
 0001:000504a8       RaiseException             100514a8 f   coredll:COREDLL.dll
 0001:000504b8       wcstombs                   100514b8 f   coredll:COREDLL.dll
 0001:000504c8       _vsnwprintf                100514c8 f   coredll:COREDLL.dll
 0001:000504d8       OutputDebugStringW         100514d8 f   coredll:COREDLL.dll
 0001:000504e8       TerminateProcess           100514e8 f   coredll:COREDLL.dll
 0001:000504f8       fputs                      100514f8 f   coredll:COREDLL.dll
 0001:00050508       _getstdfilex               10051508 f   coredll:COREDLL.dll
 0001:00050518       fflush                     10051518 f   coredll:COREDLL.dll
 0001:00050528       InterlockedExchange        10051528 f   coredll:COREDLL.dll
 0002:00003b54       ??_7CriticalSection@@6B@   10055b54     SDKRIL.obj
 0002:0001971c       ??_C@_1DC@POOIKBAO@?$AAI?$AAT?$AAE?$AAR?$AAA?$AAT?$AAO?$AAR?$AA?5?$AAL?$AAI?$AAS?$AAT?$AA?5?$AAC?$AAO?$AAR?$AAR?$AAU?$AAP?$AAT?$AAE?$AAD?$AA?$CB?$AA?$AA@ 1006b71c     SwiNotify.obj
 0002:00019750       ??_C@_1IE@BKKAAKCG@?$AAC?$AA?3?$AA?2?$AAP?$AAr?$AAo?$AAg?$AAr?$AAa?$AAm?$AA?5?$AAF?$AAi?$AAl?$AAe?$AAs?$AA?2?$AAM?$AAi?$AAc?$AAr?$AAo?$AAs?$AAo?$AAf?$AAt?$AA?5?$AAV?$AAi?$AAs?$AAu?$AAa@ 1006b750     SwiNotify.obj
 0002:000198d0       ??_C@_1EE@BBMFLDOC@?$AAl?$AAi?$AAs?$AAt?$AA?5?$AAe?$AAr?$AAa?$AAs?$AAe?$AA?5?$AAi?$AAt?$AAe?$AAr?$AAa?$AAt?$AAo?$AAr?$AA?5?$AAo?$AAu?$AAt?$AAs?$AAi?$AAd?$AAe?$AA?5?$AAr?$AAa?$AAn?$AAg@ 1006b8d0     SwiNotify.obj
 0002:00019918       ??_C@_1HM@HPOOGGJN@?$AAC?$AA?3?$AA?2?$AAP?$AAr?$AAo?$AAg?$AAr?$AAa?$AAm?$AA?5?$AAF?$AAi?$AAl?$AAe?$AAs?$AA?2?$AAM?$AAi?$AAc?$AAr?$AAo?$AAs?$AAo?$AAf?$AAt?$AA?5?$AAV?$AAi?$AAs?$AAu?$AAa@ 1006b918     SwiNotify.obj
 0002:00019b60       ??_C@_1EG@BPNHNPIG@?$AAl?$AAi?$AAs?$AAt?$AA?5?$AAi?$AAn?$AAs?$AAe?$AAr?$AAt?$AA?5?$AAi?$AAt?$AAe?$AAr?$AAa?$AAt?$AAo?$AAr?$AA?5?$AAo?$AAu?$AAt?$AAs?$AAi?$AAd?$AAe?$AA?5?$AAr?$AAa?$AAn@ 1006bb60     SwiNotify.obj
 0002:00019d04       ??_C@_1BO@MEPPHOO@?$AA?$CC?$AAo?$AAu?$AAt?$AA?5?$AAo?$AAf?$AA?5?$AAr?$AAa?$AAn?$AAg?$AAe?$AA?$CC?$AA?$AA@ 1006bd04     SwiNotify.obj
 0002:00019d28       ??_C@_1NM@FHHOPBGE@?$AAs?$AAt?$AAd?$AA?3?$AA?3?$AAl?$AAi?$AAs?$AAt?$AA?$DM?$AAs?$AAt?$AAr?$AAu?$AAc?$AAt?$AA?5?$AAs?$AAz?$AAC?$AAa?$AAl?$AAl?$AAb?$AAa?$AAc?$AAk?$AAI?$AAt?$AAe?$AAm?$AA?0@ 1006bd28     SwiNotify.obj
 0002:00019e08       ??_C@_1FG@CMLDHNON@?$AA?$CI?$AA?$CC?$AAS?$AAt?$AAa?$AAn?$AAd?$AAa?$AAr?$AAd?$AA?5?$AAC?$AA?$CL?$AA?$CL?$AA?5?$AAL?$AAi?$AAb?$AAr?$AAa?$AAr?$AAi?$AAe?$AAs?$AA?5?$AAO?$AAu?$AAt?$AA?5?$AAo?$AAf?$AA?5@ 1006be08     SwiNotify.obj
 0002:00019e60       ??_C@_1EC@HILJLMMC@?$AAl?$AAi?$AAs?$AAt?$AA?5?$AAi?$AAt?$AAe?$AAr?$AAa?$AAt?$AAo?$AAr?$AA?5?$AAn?$AAo?$AAt?$AA?5?$AAd?$AAe?$AAr?$AAe?$AAf?$AAe?$AAr?$AAe?$AAn?$AAc?$AAa?$AAb?$AAl?$AAe@ 1006be60     SwiNotify.obj
 0002:00019ea8       ??_C@_1NE@JDKDJOMI@?$AAs?$AAt?$AAd?$AA?3?$AA?3?$AAl?$AAi?$AAs?$AAt?$AA?$DM?$AAs?$AAt?$AAr?$AAu?$AAc?$AAt?$AA?5?$AAs?$AAz?$AAN?$AAo?$AAt?$AAi?$AAf?$AAy?$AAI?$AAt?$AAe?$AAm?$AA?0?$AAc?$AAl@ 1006bea8     SwiNotify.obj
 0002:00019fec       ??_C@_0BB@MOGOBHAF@list?$DMT?$DO?5too?5long?$AA@ 1006bfec     SwiNotify.obj
 0002:0001a074       ?npos@?$basic_string@DU?$char_traits@D@std@@V?$allocator@D@2@@std@@2IB 1006c074     SwiNotify.obj
 0002:0001a1d8       ??_C@_1NO@HHEEMAMN@?$AAs?$AAt?$AAd?$AA?3?$AA?3?$AAl?$AAi?$AAs?$AAt?$AA?$DM?$AAs?$AAt?$AAr?$AAu?$AAc?$AAt?$AA?5?$AAs?$AAz?$AAC?$AAa?$AAl?$AAl?$AAb?$AAa?$AAc?$AAk?$AAI?$AAt?$AAe?$AAm?$AA?0@ 1006c1d8     SwiNotify.obj
 0002:0001a2b8       ??_C@_1EA@DOGAGKDH@?$AAl?$AAi?$AAs?$AAt?$AA?5?$AAi?$AAt?$AAe?$AAr?$AAa?$AAt?$AAo?$AAr?$AA?5?$AAn?$AAo?$AAt?$AA?5?$AAi?$AAn?$AAc?$AAr?$AAe?$AAm?$AAe?$AAn?$AAt?$AAa?$AAb?$AAl?$AAe?$AA?$AA@ 1006c2b8     SwiNotify.obj
 0002:0001a2f8       ??_C@_1CG@JNLFBNGN@?$AA?$CC?$AAi?$AAn?$AAv?$AAa?$AAl?$AAi?$AAd?$AA?5?$AAa?$AAr?$AAg?$AAu?$AAm?$AAe?$AAn?$AAt?$AA?$CC?$AA?$AA@ 1006c2f8     SwiNotify.obj
 0002:0001a320       ??_C@_1NG@KPILEFHN@?$AAs?$AAt?$AAd?$AA?3?$AA?3?$AAl?$AAi?$AAs?$AAt?$AA?$DM?$AAs?$AAt?$AAr?$AAu?$AAc?$AAt?$AA?5?$AAs?$AAz?$AAC?$AAa?$AAl?$AAl?$AAb?$AAa?$AAc?$AAk?$AAI?$AAt?$AAe?$AAm?$AA?0@ 1006c320     SwiNotify.obj
 0002:0001a3f8       ??_C@_1FO@OCPOOAIA@?$AA?$CI?$AA?$CC?$AAS?$AAt?$AAa?$AAn?$AAd?$AAa?$AAr?$AAd?$AA?5?$AAC?$AA?$CL?$AA?$CL?$AA?5?$AAL?$AAi?$AAb?$AAr?$AAa?$AAr?$AAi?$AAe?$AAs?$AA?5?$AAI?$AAn?$AAv?$AAa?$AAl?$AAi?$AAd@ 1006c3f8     SwiNotify.obj
 0002:0001a458       ??_C@_1DI@MDELDGPI@?$AAl?$AAi?$AAs?$AAt?$AA?5?$AAi?$AAt?$AAe?$AAr?$AAa?$AAt?$AAo?$AAr?$AAs?$AA?5?$AAi?$AAn?$AAc?$AAo?$AAm?$AAp?$AAa?$AAt?$AAi?$AAb?$AAl?$AAe?$AA?$AA@ 1006c458     SwiNotify.obj
 0002:0001a4c8       ??_C@_1NG@KIPLILDM@?$AAs?$AAt?$AAd?$AA?3?$AA?3?$AAl?$AAi?$AAs?$AAt?$AA?$DM?$AAs?$AAt?$AAr?$AAu?$AAc?$AAt?$AA?5?$AAs?$AAz?$AAN?$AAo?$AAt?$AAi?$AAf?$AAy?$AAI?$AAt?$AAe?$AAm?$AA?0?$AAc?$AAl@ 1006c4c8     SwiNotify.obj
 0002:0001a5a0       ??_C@_1MO@JOPNAGLH@?$AAs?$AAt?$AAd?$AA?3?$AA?3?$AAl?$AAi?$AAs?$AAt?$AA?$DM?$AAs?$AAt?$AAr?$AAu?$AAc?$AAt?$AA?5?$AAs?$AAz?$AAN?$AAo?$AAt?$AAi?$AAf?$AAy?$AAI?$AAt?$AAe?$AAm?$AA?0?$AAc?$AAl@ 1006c5a0     SwiNotify.obj
 0002:0001a798       ??_C@_1IC@HKDJIJDA@?$AAC?$AA?3?$AA?2?$AAP?$AAr?$AAo?$AAg?$AAr?$AAa?$AAm?$AA?5?$AAF?$AAi?$AAl?$AAe?$AAs?$AA?2?$AAM?$AAi?$AAc?$AAr?$AAo?$AAs?$AAo?$AAf?$AAt?$AA?5?$AAV?$AAi?$AAs?$AAu?$AAa@ 1006c798     SwiNotify.obj
 0002:0001a81c       ??_C@_1CK@EOPGIILJ@?$AAi?$AAn?$AAv?$AAa?$AAl?$AAi?$AAd?$AA?5?$AAn?$AAu?$AAl?$AAl?$AA?5?$AAp?$AAo?$AAi?$AAn?$AAt?$AAe?$AAr?$AA?$AA@ 1006c81c     SwiNotify.obj
 0002:0001a9ac       ??_C@_1DM@PIGEIECN@?$AAl?$AAi?$AAs?$AAt?$AA?5?$AAi?$AAn?$AAs?$AAe?$AAr?$AAt?$AAi?$AAo?$AAn?$AA?5?$AAo?$AAv?$AAe?$AAr?$AAl?$AAa?$AAp?$AAs?$AA?5?$AAr?$AAa?$AAn?$AAg?$AAe?$AA?$AA@ 1006c9ac     SwiNotify.obj
 0002:0001aad0       ??_C@_1NG@FLMJDHPN@?$AAs?$AAt?$AAd?$AA?3?$AA?3?$AAl?$AAi?$AAs?$AAt?$AA?$DM?$AAs?$AAt?$AAr?$AAu?$AAc?$AAt?$AA?5?$AAs?$AAz?$AAN?$AAo?$AAt?$AAi?$AAf?$AAy?$AAI?$AAt?$AAe?$AAm?$AA?0?$AAc?$AAl@ 1006cad0     SwiNotify.obj
 0002:0001aba8       ??_C@_1EA@JDNDELPC@?$AAl?$AAi?$AAs?$AAt?$AA?5?$AAi?$AAt?$AAe?$AAr?$AAa?$AAt?$AAo?$AAr?$AA?5?$AAn?$AAo?$AAt?$AA?5?$AAd?$AAe?$AAc?$AAr?$AAe?$AAm?$AAe?$AAn?$AAt?$AAa?$AAb?$AAl?$AAe?$AA?$AA@ 1006cba8     SwiNotify.obj
 0002:0001bb38       ??_C@_11LOCGONAA@?$AA?$AA@ 1006db38     toolbox:toolbox_i.obj
 0002:0001bb3c       ??_C@_19GGMAHBDP@?$AA?$DM?$AAc?$AAr?$AA?$DO?$AA?$AA@ 1006db3c     toolbox:toolbox_i.obj
 0002:0001bb48       ??_C@_19CHKHCDBO@?$AA?$DM?$AAl?$AAf?$AA?$DO?$AA?$AA@ 1006db48     toolbox:toolbox_i.obj
 0002:0001bb54       ??_C@_06LKNEJLBE@?$FL?$CF02x?$FN?$AA@ 1006db54     toolbox:toolbox_i.obj
 0002:0001bb5c       ??_C@_04GCCPKCML@?$DMcr?$DO?$AA@ 1006db5c     toolbox:toolbox_i.obj
 0002:0001bb64       ??_C@_04CBGDLJDB@?$DMlf?$DO?$AA@ 1006db64     toolbox:toolbox_i.obj
 0002:0001bb70       ??_7?$GrowableThingCollection@PAG@@6B@ 1006db70     toolbox:toolbox_i.obj
 0002:0001bbc0       ??_7?$GrowableThingCollection@PAX@@6B@ 1006dbc0     toolbox:toolbox_i.obj
 0002:0001bc10       ??_7?$GrowableThingCollection@UTaskListTaskData@TaskList@@@@6B@ 1006dc10     toolbox:toolbox_i.obj
 0002:0001bc60       ??_7?$GrowablePointerCollection@G@@6B@ 1006dc60     toolbox:toolbox_i.obj
 0002:0001bcac       ??_7StringCollection@@6B@  1006dcac     toolbox:toolbox_i.obj
 0002:0001bcbc       ??_7SortedStringCollection@@6B@ 1006dcbc     toolbox:toolbox_i.obj
 0002:0001bcd0       ??_C@_1DM@MADKGDLO@?$AA?$CI?$AAL?$AA?$CC?$AAB?$AAu?$AAf?$AAf?$AAe?$AAr?$AA?5?$AAi?$AAs?$AA?5?$AAt?$AAo?$AAo?$AA?5?$AAs?$AAm?$AAa?$AAl?$AAl?$AA?$CC?$AA?5?$AA?$CG?$AA?$CG?$AA?5?$AA0?$AA?$CJ?$AA?$AA@ 1006dcd0     LIBCMTD:strcpy_s.obj
 0002:0001bd0c       ??_C@_1CI@HCPHDDLE@?$AAB?$AAu?$AAf?$AAf?$AAe?$AAr?$AA?5?$AAi?$AAs?$AA?5?$AAt?$AAo?$AAo?$AA?5?$AAs?$AAm?$AAa?$AAl?$AAl?$AA?$AA@ 1006dd0c     LIBCMTD:strcpy_s.obj
 0002:0001bd34       ??_C@_1CG@OFBJMIGJ@?$AA?$CI?$AA?$CI?$AA?$CI?$AA_?$AAS?$AAr?$AAc?$AA?$CJ?$AA?$CJ?$AA?$CJ?$AA?5?$AA?$CB?$AA?$DN?$AA?5?$AAN?$AAU?$AAL?$AAL?$AA?$AA@ 1006dd34     LIBCMTD:strcpy_s.obj
 0002:0001bd5c       ??_C@_1BC@CFJEPFGF@?$AAs?$AAt?$AAr?$AAc?$AAp?$AAy?$AA_?$AAs?$AA?$AA@ 1006dd5c     LIBCMTD:strcpy_s.obj
 0002:0001bd70       ??_C@_1FE@IPADLOPJ@?$AAf?$AA?3?$AA?2?$AAs?$AAp?$AA?2?$AAv?$AAc?$AAt?$AAo?$AAo?$AAl?$AAs?$AA?2?$AAc?$AAr?$AAt?$AAc?$AAe?$AA?2?$AAc?$AAr?$AAt?$AAw?$AA3?$AA2?$AA?2?$AAh?$AA?2?$AAt?$AAc?$AAs@ 1006dd70     LIBCMTD:strcpy_s.obj
 0002:0001bdc8       ??_C@_1FC@NCPEPIBI@?$AA?$CI?$AA?$CI?$AA_?$AAD?$AAs?$AAt?$AA?$CJ?$AA?$CJ?$AA?5?$AA?$CB?$AA?$DN?$AA?5?$AAN?$AAU?$AAL?$AAL?$AA?5?$AA?$CG?$AA?$CG?$AA?5?$AA?$CI?$AA?$CI?$AA_?$AAS?$AAi?$AAz?$AAe?$AAI?$AAn?$AAB?$AAy?$AAt@ 1006ddc8     LIBCMTD:strcpy_s.obj
 0002:0001be1c       ??_C@_17LGKOMLJ@?$AA?4?$AA?4?$AA?4?$AA?$AA@ 1006de1c     LIBCMTD:dbgrpt.obj
 0002:0001be24       ??_C@_1CC@CGHMNGDG@?$AAA?$AAs?$AAs?$AAe?$AAr?$AAt?$AAi?$AAo?$AAn?$AA?5?$AAF?$AAa?$AAi?$AAl?$AAe?$AAd?$AA?$AA@ 1006de24     LIBCMTD:dbgrpt.obj
 0002:0001be48       ??_C@_1M@ILHOPKA@?$AAE?$AAr?$AAr?$AAo?$AAr?$AA?$AA@ 1006de48     LIBCMTD:dbgrpt.obj
 0002:0001be54       ??_C@_1BA@GLMCNLEM@?$AAW?$AAa?$AAr?$AAn?$AAi?$AAn?$AAg?$AA?$AA@ 1006de54     LIBCMTD:dbgrpt.obj
 0002:0001be68       ??_C@_1FI@PHIAFFHM@?$AA?$CI?$AA?$CC?$AAT?$AAh?$AAe?$AA?5?$AAh?$AAo?$AAo?$AAk?$AA?5?$AAf?$AAu?$AAn?$AAc?$AAt?$AAi?$AAo?$AAn?$AA?5?$AAi?$AAs?$AA?5?$AAn?$AAo?$AAt?$AA?5?$AAi?$AAn?$AA?5?$AAt?$AAh@ 1006de68     LIBCMTD:dbgrpt.obj
 0002:0001bec0       ??_C@_1CG@JBJEFOCM@?$AAp?$AAf?$AAn?$AAN?$AAe?$AAw?$AAH?$AAo?$AAo?$AAk?$AA?5?$AA?$CB?$AA?$DN?$AA?5?$AAN?$AAU?$AAL?$AAL?$AA?$AA@ 1006dec0     LIBCMTD:dbgrpt.obj
 0002:0001bee8       ??_C@_1CI@OOAHIOG@?$AA_?$AAC?$AAr?$AAt?$AAS?$AAe?$AAt?$AAR?$AAe?$AAp?$AAo?$AAr?$AAt?$AAH?$AAo?$AAo?$AAk?$AAT?$AA2?$AA?$AA@ 1006dee8     LIBCMTD:dbgrpt.obj
 0002:0001bf10       ??_C@_1FC@DDJKODKC@?$AAf?$AA?3?$AA?2?$AAs?$AAp?$AA?2?$AAv?$AAc?$AAt?$AAo?$AAo?$AAl?$AAs?$AA?2?$AAc?$AAr?$AAt?$AAc?$AAe?$AA?2?$AAc?$AAr?$AAt?$AAw?$AA3?$AA2?$AA?2?$AAm?$AAi?$AAs?$AAc?$AA?2@ 1006df10     LIBCMTD:dbgrpt.obj
 0002:0001bf68       ??_C@_1HI@OFEHGPPC@?$AAm?$AAo?$AAd?$AAe?$AA?5?$AA?$DN?$AA?$DN?$AA?5?$AA_?$AAC?$AAR?$AAT?$AA_?$AAR?$AAP?$AAT?$AAH?$AAO?$AAO?$AAK?$AA_?$AAI?$AAN?$AAS?$AAT?$AAA?$AAL?$AAL?$AA?5?$AA?$HM?$AA?$HM?$AA?5@ 1006df68     LIBCMTD:dbgrpt.obj
 0002:0001bfe0       ??_C@_1EG@PEOEAKBB@?$AAM?$AAi?$AAc?$AAr?$AAo?$AAs?$AAo?$AAf?$AAt?$AA?5?$AAV?$AAi?$AAs?$AAu?$AAa?$AAl?$AA?5?$AAC?$AA?$CL?$AA?$CL?$AA?5?$AAD?$AAe?$AAb?$AAu?$AAg?$AA?5?$AAL?$AAi?$AAb?$AAr?$AAa@ 1006dfe0     LIBCMTD:dbgrpt.obj
 0002:0001c028       ??_C@_1JI@EACPGHID@?$AAw?$AAc?$AAs?$AAc?$AAp?$AAy?$AA_?$AAs?$AA?$CI?$AAs?$AAz?$AAO?$AAu?$AAt?$AAM?$AAe?$AAs?$AAs?$AAa?$AAg?$AAe?$AA?0?$AA?5?$AA4?$AA0?$AA9?$AA6?$AA?0?$AA?5?$AAL?$AA?$CC?$AA_@ 1006e028     LIBCMTD:dbgrpt.obj
 0002:0001c0c0       ??_C@_1FG@BBOLDHGF@?$AA_?$AAC?$AAr?$AAt?$AAD?$AAb?$AAg?$AAR?$AAe?$AAp?$AAo?$AAr?$AAt?$AA?3?$AA?5?$AAS?$AAt?$AAr?$AAi?$AAn?$AAg?$AA?5?$AAt?$AAo?$AAo?$AA?5?$AAl?$AAo?$AAn?$AAg?$AA?5?$AAo@ 1006e0c0     LIBCMTD:dbgrpt.obj
 0002:0001c118       ??_C@_1KG@MFHGLLO@?$AAD?$AAe?$AAb?$AAu?$AAg?$AA?5?$AA?$CF?$AAs?$AA?$CB?$AA?6?$AA?6?$AAP?$AAr?$AAo?$AAg?$AAr?$AAa?$AAm?$AA?3?$AA?5?$AA?$CF?$AAs?$AA?$CF?$AAs?$AA?$CF?$AAs?$AA?$CF?$AAs?$AA?$CF?$AAs?$AA?$CF?$AAs@ 1006e118     LIBCMTD:dbgrpt.obj
 0002:0001c1c0       ??_C@_1BE@CGCJKGHI@?$AA?6?$AAM?$AAo?$AAd?$AAu?$AAl?$AAe?$AA?3?$AA?5?$AA?$AA@ 1006e1c0     LIBCMTD:dbgrpt.obj
 0002:0001c1d4       ??_C@_1BA@LNHECFIM@?$AA?6?$AAF?$AAi?$AAl?$AAe?$AA?3?$AA?5?$AA?$AA@ 1006e1d4     LIBCMTD:dbgrpt.obj
 0002:0001c1e4       ??_C@_1BA@GLLGCPCK@?$AA?6?$AAL?$AAi?$AAn?$AAe?$AA?3?$AA?5?$AA?$AA@ 1006e1e4     LIBCMTD:dbgrpt.obj
 0002:0001c1f4       ??_C@_13LBAGMAIH@?$AA?6?$AA?$AA@ 1006e1f4     LIBCMTD:dbgrpt.obj
 0002:0001c1f8       ??_C@_1BK@PEDCIPMA@?$AAE?$AAx?$AAp?$AAr?$AAe?$AAs?$AAs?$AAi?$AAo?$AAn?$AA?3?$AA?5?$AA?$AA@ 1006e1f8     LIBCMTD:dbgrpt.obj
 0002:0001c218       ??_C@_1JM@GKDPCMEA@?$AAw?$AAc?$AAs?$AAn?$AAc?$AAp?$AAy?$AA_?$AAs?$AA?$CI?$AAs?$AAz?$AAS?$AAh?$AAo?$AAr?$AAt?$AAP?$AAr?$AAo?$AAg?$AAN?$AAa?$AAm?$AAe?$AA?0?$AA?5?$AA2?$AA6?$AA0?$AA?5?$AA?9@ 1006e218     LIBCMTD:dbgrpt.obj
 0002:0001c2b8       ??_C@_1GI@DEDNNLCI@?$AAw?$AAc?$AAs?$AAc?$AAp?$AAy?$AA_?$AAs?$AA?$CI?$AAs?$AAz?$AAE?$AAx?$AAe?$AAN?$AAa?$AAm?$AAe?$AA?0?$AA?5?$AA2?$AA6?$AA0?$AA?0?$AA?5?$AAL?$AA?$CC?$AA?$DM?$AAp?$AAr?$AAo?$AAg@ 1006e2b8     LIBCMTD:dbgrpt.obj
 0002:0001c320       ??_C@_1CI@PGJIFDEK@?$AA_?$AA_?$AAc?$AAr?$AAt?$AAM?$AAe?$AAs?$AAs?$AAa?$AAg?$AAe?$AAW?$AAi?$AAn?$AAd?$AAo?$AAw?$AAW?$AA?$AA@ 1006e320     LIBCMTD:dbgrpt.obj
 0002:0001c348       ??_C@_1CO@EAEJAADC@?$AA?$DM?$AAp?$AAr?$AAo?$AAg?$AAr?$AAa?$AAm?$AA?5?$AAn?$AAa?$AAm?$AAe?$AA?5?$AAu?$AAn?$AAk?$AAn?$AAo?$AAw?$AAn?$AA?$DO?$AA?$AA@ 1006e348     LIBCMTD:dbgrpt.obj
 0002:0001c378       ??_C@_1CK@DDKKOLAN@?$AAs?$AAi?$AAz?$AAe?$AAI?$AAn?$AAB?$AAy?$AAt?$AAe?$AAs?$AA?5?$AA?$DO?$AA?$DN?$AA?5?$AAc?$AAo?$AAu?$AAn?$AAt?$AA?$AA@ 1006e378     LIBCMTD:memcpy_s.obj
 0002:0001c3a4       ??_C@_1BI@DCHLDCPP@?$AAs?$AAr?$AAc?$AA?5?$AA?$CB?$AA?$DN?$AA?5?$AAN?$AAU?$AAL?$AAL?$AA?$AA@ 1006e3a4     LIBCMTD:memcpy_s.obj
 0002:0001c3bc       ??_C@_1BC@GKHDJMGB@?$AAm?$AAe?$AAm?$AAc?$AAp?$AAy?$AA_?$AAs?$AA?$AA@ 1006e3bc     LIBCMTD:memcpy_s.obj
 0002:0001c3d0       ??_C@_1FK@BOBCAACJ@?$AAf?$AA?3?$AA?2?$AAs?$AAp?$AA?2?$AAv?$AAc?$AAt?$AAo?$AAo?$AAl?$AAs?$AA?2?$AAc?$AAr?$AAt?$AAc?$AAe?$AA?2?$AAc?$AAr?$AAt?$AAw?$AA3?$AA2?$AA?2?$AAs?$AAt?$AAr?$AAi?$AAn@ 1006e3d0     LIBCMTD:memcpy_s.obj
 0002:0001c42c       ??_C@_1BI@GKKCBDMD@?$AAd?$AAs?$AAt?$AA?5?$AA?$CB?$AA?$DN?$AA?5?$AAN?$AAU?$AAL?$AAL?$AA?$AA@ 1006e42c     LIBCMTD:memcpy_s.obj
 0002:0001c444       ??_C@_1BE@NMKKBGPA@?$AAm?$AAe?$AAm?$AAm?$AAo?$AAv?$AAe?$AA_?$AAs?$AA?$AA@ 1006e444     LIBCMTD:memmove_s.obj
 0002:0001c458       ??_C@_1FM@JMDLOEFB@?$AAf?$AA?3?$AA?2?$AAs?$AAp?$AA?2?$AAv?$AAc?$AAt?$AAo?$AAo?$AAl?$AAs?$AA?2?$AAc?$AAr?$AAt?$AAc?$AAe?$AA?2?$AAc?$AAr?$AAt?$AAw?$AA3?$AA2?$AA?2?$AAs?$AAt?$AAr?$AAi?$AAn@ 1006e458     LIBCMTD:memmove_s.obj
 0002:0001c4b4       ??_C@_0BJ@IPHDMCNM@fatal?5error?5in?5_lock?5?$CD0?6?$AA@ 1006e4b4     LIBCMTD:mlock.obj
 0002:0001c4d0       ??_C@_1NK@LOFHIHFC@?$AAf?$AAM?$AAo?$AAd?$AAe?$AA?5?$AA?$DN?$AA?$DN?$AA?5?$AA_?$AAC?$AAR?$AAT?$AAD?$AAB?$AAG?$AA_?$AAR?$AAE?$AAP?$AAO?$AAR?$AAT?$AA_?$AAM?$AAO?$AAD?$AAE?$AA?5?$AA?$HM?$AA?$HM?$AA?5@ 1006e4d0     LIBCMTD:dbgrptt.obj
 0002:0001c5ac       ??_C@_1CE@FIHIECNJ@?$AA_?$AAC?$AAr?$AAt?$AAS?$AAe?$AAt?$AAR?$AAe?$AAp?$AAo?$AAr?$AAt?$AAM?$AAo?$AAd?$AAe?$AA?$AA@ 1006e5ac     LIBCMTD:dbgrptt.obj
 0002:0001c5d0       ??_C@_1FE@PLIBPAGC@?$AAf?$AA?3?$AA?2?$AAs?$AAp?$AA?2?$AAv?$AAc?$AAt?$AAo?$AAo?$AAl?$AAs?$AA?2?$AAc?$AAr?$AAt?$AAc?$AAe?$AA?2?$AAc?$AAr?$AAt?$AAw?$AA3?$AA2?$AA?2?$AAm?$AAi?$AAs?$AAc?$AA?2@ 1006e5d0     LIBCMTD:dbgrptt.obj
 0002:0001c628       ??_C@_1FA@IFFFOLDJ@?$AAn?$AAR?$AAp?$AAt?$AAT?$AAy?$AAp?$AAe?$AA?5?$AA?$DO?$AA?$DN?$AA?5?$AA0?$AA?5?$AA?$CG?$AA?$CG?$AA?5?$AAn?$AAR?$AAp?$AAt?$AAT?$AAy?$AAp?$AAe?$AA?5?$AA?$DM?$AA?5?$AA_?$AAC?$AAR?$AAT@ 1006e628     LIBCMTD:dbgrptt.obj
 0002:0001c678       ??_C@_1CE@IKKEDCME@?$AA_?$AAC?$AAr?$AAt?$AAS?$AAe?$AAt?$AAR?$AAe?$AAp?$AAo?$AAr?$AAt?$AAF?$AAi?$AAl?$AAe?$AA?$AA@ 1006e678     LIBCMTD:dbgrptt.obj
 0002:0001c6a0       ??_C@_1MA@LBAMNNOB@?$AAs?$AAt?$AAr?$AAc?$AAp?$AAy?$AA_?$AAs?$AA?$CI?$AAs?$AAz?$AAO?$AAu?$AAt?$AAM?$AAe?$AAs?$AAs?$AAa?$AAg?$AAe?$AA2?$AA?0?$AA?5?$AA4?$AA0?$AA9?$AA6?$AA?0?$AA?5?$AA?$CC?$AA_@ 1006e6a0     LIBCMTD:dbgrptt.obj
 0002:0001c760       ??_C@_0DP@GNPEPHJD@_CrtDbgReport?3?5String?5too?5long?5o@ 1006e760     LIBCMTD:dbgrptt.obj
 0002:0001c7a0       ??_C@_1FI@DBAIJPJE@?$AAw?$AAc?$AAs?$AAc?$AAp?$AAy?$AA_?$AAs?$AA?$CI?$AAs?$AAz?$AAO?$AAu?$AAt?$AAM?$AAe?$AAs?$AAs?$AAa?$AAg?$AAe?$AA?0?$AA?5?$AA4?$AA0?$AA9?$AA6?$AA?0?$AA?5?$AAs?$AAz?$AAL@ 1006e7a0     LIBCMTD:dbgrptt.obj
 0002:0001c7f8       ??_C@_1BI@JIDBEPIG@?$AA?$CF?$AAs?$AA?$CI?$AA?$CF?$AAd?$AA?$CJ?$AA?5?$AA?3?$AA?5?$AA?$CF?$AAs?$AA?$AA@ 1006e7f8     LIBCMTD:dbgrptt.obj
 0002:0001c810       ??_C@_1EK@PHCBEDKB@?$AAw?$AAc?$AAs?$AAc?$AAa?$AAt?$AA_?$AAs?$AA?$CI?$AAs?$AAz?$AAL?$AAi?$AAn?$AAe?$AAM?$AAe?$AAs?$AAs?$AAa?$AAg?$AAe?$AA?0?$AA?5?$AA4?$AA0?$AA9?$AA6?$AA?0?$AA?5?$AAL?$AA?$CC@ 1006e810     LIBCMTD:dbgrptt.obj
 0002:0001c860       ??_C@_1EK@NMDFGHMF@?$AAw?$AAc?$AAs?$AAc?$AAa?$AAt?$AA_?$AAs?$AA?$CI?$AAs?$AAz?$AAL?$AAi?$AAn?$AAe?$AAM?$AAe?$AAs?$AAs?$AAa?$AAg?$AAe?$AA?0?$AA?5?$AA4?$AA0?$AA9?$AA6?$AA?0?$AA?5?$AAL?$AA?$CC@ 1006e860     LIBCMTD:dbgrptt.obj
 0002:0001c8ac       ??_C@_13CMNBPIDO@?$AA?$AN?$AA?$AA@ 1006e8ac     LIBCMTD:dbgrptt.obj
 0002:0001c8b0       ??_C@_1FK@HPADHBBD@?$AAw?$AAc?$AAs?$AAc?$AAa?$AAt?$AA_?$AAs?$AA?$CI?$AAs?$AAz?$AAL?$AAi?$AAn?$AAe?$AAM?$AAe?$AAs?$AAs?$AAa?$AAg?$AAe?$AA?0?$AA?5?$AA4?$AA0?$AA9?$AA6?$AA?0?$AA?5?$AAs?$AAz@ 1006e8b0     LIBCMTD:dbgrptt.obj
 0002:0001c910       ??_C@_1KO@DGAHENCH@?$AAw?$AAc?$AAs?$AAc?$AAp?$AAy?$AA_?$AAs?$AA?$CI?$AAs?$AAz?$AAL?$AAi?$AAn?$AAe?$AAM?$AAe?$AAs?$AAs?$AAa?$AAg?$AAe?$AA?0?$AA?5?$AA4?$AA0?$AA9?$AA6?$AA?0?$AA?5?$AAs?$AAz@ 1006e910     LIBCMTD:dbgrptt.obj
 0002:0001c9c0       ??_C@_1CE@OJBNHDMO@?$AAA?$AAs?$AAs?$AAe?$AAr?$AAt?$AAi?$AAo?$AAn?$AA?5?$AAf?$AAa?$AAi?$AAl?$AAe?$AAd?$AA?$CB?$AA?$AA@ 1006e9c0     LIBCMTD:dbgrptt.obj
 0002:0001c9e4       ??_C@_1CG@FFFGGODN@?$AAA?$AAs?$AAs?$AAe?$AAr?$AAt?$AAi?$AAo?$AAn?$AA?5?$AAf?$AAa?$AAi?$AAl?$AAe?$AAd?$AA?3?$AA?5?$AA?$AA@ 1006e9e4     LIBCMTD:dbgrptt.obj
 0002:0001ca10       ??_C@_1JK@KHFABAEO@?$AAw?$AAc?$AAs?$AAc?$AAp?$AAy?$AA_?$AAs?$AA?$CI?$AAs?$AAz?$AAU?$AAs?$AAe?$AAr?$AAM?$AAe?$AAs?$AAs?$AAa?$AAg?$AAe?$AA?0?$AA?5?$AA4?$AA0?$AA9?$AA6?$AA?0?$AA?5?$AAL?$AA?$CC@ 1006ea10     LIBCMTD:dbgrptt.obj
 0002:0001caac       ??_C@_1BA@ELMMDCFC@?$AA?0?$AA?5?$AAL?$AAi?$AAn?$AAe?$AA?5?$AA?$AA@ 1006eaac     LIBCMTD:dbgrptt.obj
 0002:0001cabc       ??_C@_1BO@OCHMLCAG@?$AA?$DM?$AAf?$AAi?$AAl?$AAe?$AA?5?$AAu?$AAn?$AAk?$AAn?$AAo?$AAw?$AAn?$AA?$DO?$AA?$AA@ 1006eabc     LIBCMTD:dbgrptt.obj
 0002:0001cae0       ??_C@_1EM@MJFLEDMB@?$AAS?$AAe?$AAc?$AAo?$AAn?$AAd?$AA?5?$AAC?$AAh?$AAa?$AAn?$AAc?$AAe?$AA?5?$AAA?$AAs?$AAs?$AAe?$AAr?$AAt?$AAi?$AAo?$AAn?$AA?5?$AAF?$AAa?$AAi?$AAl?$AAe?$AAd?$AA?3?$AA?5@ 1006eae0     LIBCMTD:dbgrptt.obj
 0002:0001cb30       ??_C@_1FA@CNLLOMHI@?$AA_?$AAi?$AAt?$AAo?$AAw?$AA_?$AAs?$AA?$CI?$AAn?$AAL?$AAi?$AAn?$AAe?$AA?0?$AA?5?$AAs?$AAz?$AAL?$AAi?$AAn?$AAe?$AAM?$AAe?$AAs?$AAs?$AAa?$AAg?$AAe?$AA?0?$AA?5?$AA4?$AA0@ 1006eb30     LIBCMTD:dbgrptt.obj
 0002:0001cb80       ??_C@_1CA@HPALHDOD@?$AA_?$AAV?$AAC?$AAr?$AAt?$AAD?$AAb?$AAg?$AAR?$AAe?$AAp?$AAo?$AAr?$AAt?$AAW?$AA?$AA@ 1006eb80     LIBCMTD:dbgrptt.obj
 0002:0001cba0       ??_C@_1CG@MKBKDNCP@?$AAG?$AAe?$AAt?$AAL?$AAa?$AAs?$AAt?$AAA?$AAc?$AAt?$AAi?$AAv?$AAe?$AAP?$AAo?$AAp?$AAu?$AAp?$AA?$AA@ 1006eba0     LIBCMTD:crtmbox.obj
 0002:0001cbc8       ??_C@_1CA@HNKPMKAN@?$AAG?$AAe?$AAt?$AAA?$AAc?$AAt?$AAi?$AAv?$AAe?$AAW?$AAi?$AAn?$AAd?$AAo?$AAw?$AA?$AA@ 1006ebc8     LIBCMTD:crtmbox.obj
 0002:0001cbe8       ??_C@_1BI@OGPGOOGK@?$AAM?$AAe?$AAs?$AAs?$AAa?$AAg?$AAe?$AAB?$AAo?$AAx?$AAW?$AA?$AA@ 1006ebe8     LIBCMTD:crtmbox.obj
 0002:0001cc00       ??_C@_1BI@IENOMFML@?$AAC?$AAO?$AAR?$AAE?$AAD?$AAL?$AAL?$AA?4?$AAD?$AAL?$AAL?$AA?$AA@ 1006ec00     LIBCMTD:crtmbox.obj
 0002:0001cc18       ??_C@_1BE@PMMBFFCC@?$AAw?$AAc?$AAs?$AAn?$AAc?$AAp?$AAy?$AA_?$AAs?$AA?$AA@ 1006ec18     LIBCMTD:wcsncpy_s.obj
 0002:0001cc30       ??_C@_1FG@OHHBDIEA@?$AAf?$AA?3?$AA?2?$AAs?$AAp?$AA?2?$AAv?$AAc?$AAt?$AAo?$AAo?$AAl?$AAs?$AA?2?$AAc?$AAr?$AAt?$AAc?$AAe?$AA?2?$AAc?$AAr?$AAt?$AAw?$AA3?$AA2?$AA?2?$AAh?$AA?2?$AAt?$AAc?$AAs@ 1006ec30     LIBCMTD:wcsncpy_s.obj
 0002:0001cc88       ??_C@_1FC@PFMLEHKI@?$AA?$CI?$AA?$CI?$AA_?$AAD?$AAs?$AAt?$AA?$CJ?$AA?$CJ?$AA?5?$AA?$CB?$AA?$DN?$AA?5?$AAN?$AAU?$AAL?$AAL?$AA?5?$AA?$CG?$AA?$CG?$AA?5?$AA?$CI?$AA?$CI?$AA_?$AAS?$AAi?$AAz?$AAe?$AAI?$AAn?$AAW?$AAo?$AAr@ 1006ec88     LIBCMTD:wcsncpy_s.obj
 0002:0001ccdc       ??_C@_1BC@KIONAFPO@?$AAw?$AAc?$AAs?$AAc?$AAp?$AAy?$AA_?$AAs?$AA?$AA@ 1006ecdc     LIBCMTD:wcscpy_s.obj
 0002:0001ccf0       ??_C@_1FA@MJKDNFFB@?$AA?$CI?$AAL?$AA?$CC?$AAS?$AAt?$AAr?$AAi?$AAn?$AAg?$AA?5?$AAi?$AAs?$AA?5?$AAn?$AAo?$AAt?$AA?5?$AAn?$AAu?$AAl?$AAl?$AA?5?$AAt?$AAe?$AAr?$AAm?$AAi?$AAn?$AAa?$AAt?$AAe?$AAd@ 1006ecf0     LIBCMTD:wcscat_s.obj
 0002:0001cd40       ??_C@_1DM@FHLMIEG@?$AAS?$AAt?$AAr?$AAi?$AAn?$AAg?$AA?5?$AAi?$AAs?$AA?5?$AAn?$AAo?$AAt?$AA?5?$AAn?$AAu?$AAl?$AAl?$AA?5?$AAt?$AAe?$AAr?$AAm?$AAi?$AAn?$AAa?$AAt?$AAe?$AAd?$AA?$AA@ 1006ed40     LIBCMTD:wcscat_s.obj
 0002:0001cd7c       ??_C@_1BC@PLIEPKPJ@?$AAw?$AAc?$AAs?$AAc?$AAa?$AAt?$AA_?$AAs?$AA?$AA@ 1006ed7c     LIBCMTD:wcscat_s.obj
 0002:0001cd90       ??_C@_1FE@EHLIBGFJ@?$AAf?$AA?3?$AA?2?$AAs?$AAp?$AA?2?$AAv?$AAc?$AAt?$AAo?$AAo?$AAl?$AAs?$AA?2?$AAc?$AAr?$AAt?$AAc?$AAe?$AA?2?$AAc?$AAr?$AAt?$AAw?$AA3?$AA2?$AA?2?$AAh?$AA?2?$AAt?$AAc?$AAs@ 1006ed90     LIBCMTD:wcscat_s.obj
 0002:0001cde4       ??_C@_1CM@HABGDNLJ@?$AAl?$AAe?$AAn?$AAg?$AAt?$AAh?$AA?5?$AA?$DM?$AA?5?$AAs?$AAi?$AAz?$AAe?$AAI?$AAn?$AAT?$AAC?$AAh?$AAa?$AAr?$AAs?$AA?$AA@ 1006ede4     LIBCMTD:xtows.obj
 0002:0001ce10       ??_C@_1DE@PCJGDBBD@?$AA2?$AA?5?$AA?$DM?$AA?$DN?$AA?5?$AAr?$AAa?$AAd?$AAi?$AAx?$AA?5?$AA?$CG?$AA?$CG?$AA?5?$AAr?$AAa?$AAd?$AAi?$AAx?$AA?5?$AA?$DM?$AA?$DN?$AA?5?$AA3?$AA6?$AA?$AA@ 1006ee10     LIBCMTD:xtows.obj
 0002:0001ce48       ??_C@_1FA@MKGGAGEI@?$AAs?$AAi?$AAz?$AAe?$AAI?$AAn?$AAT?$AAC?$AAh?$AAa?$AAr?$AAs?$AA?5?$AA?$DO?$AA?5?$AA?$CI?$AAs?$AAi?$AAz?$AAe?$AA_?$AAt?$AA?$CJ?$AA?$CI?$AAi?$AAs?$AA_?$AAn?$AAe?$AAg?$AA?5?$AA?$DP@ 1006ee48     LIBCMTD:xtows.obj
 0002:0001ce98       ??_C@_1CC@JNJFIMGE@?$AAs?$AAi?$AAz?$AAe?$AAI?$AAn?$AAT?$AAC?$AAh?$AAa?$AAr?$AAs?$AA?5?$AA?$DO?$AA?5?$AA0?$AA?$AA@ 1006ee98     LIBCMTD:xtows.obj
 0002:0001cebc       ??_C@_1O@NCBFODOE@?$AAx?$AAt?$AAo?$AAw?$AA_?$AAs?$AA?$AA@ 1006eebc     LIBCMTD:xtows.obj
 0002:0001ced0       ??_C@_1FE@LAGNOOBA@?$AAf?$AA?3?$AA?2?$AAs?$AAp?$AA?2?$AAv?$AAc?$AAt?$AAo?$AAo?$AAl?$AAs?$AA?2?$AAc?$AAr?$AAt?$AAc?$AAe?$AA?2?$AAc?$AAr?$AAt?$AAw?$AA3?$AA2?$AA?2?$AAc?$AAo?$AAn?$AAv?$AAe@ 1006eed0     LIBCMTD:xtows.obj
 0002:0001cf24       ??_C@_1BI@ICGGMGLK@?$AAb?$AAu?$AAf?$AA?5?$AA?$CB?$AA?$DN?$AA?5?$AAN?$AAU?$AAL?$AAL?$AA?$AA@ 1006ef24     LIBCMTD:xtows.obj
 0002:0001cf3c       ??_C@_0P@GHFPNOJB@bad?5allocation?$AA@ 1006ef3c     libcpmtd:stdthrow.obj
 0002:0001cf4c       ??_C@_01EEMJAFIK@?6?$AA@   1006ef4c     libcpmtd:stdthrow.obj
 0002:0001cf50       ??_C@_07CIFAGBMG@unknown?$AA@ 1006ef50     libcpmtd:stdthrow.obj
 0002:0001cf58       ??_C@_0M@LLHBPFNE@exception?3?5?$AA@ 1006ef58     libcpmtd:stdthrow.obj
 0002:0001cf64       ?skipws@?$_Iosb@H@std@@2W4_Fmtflags@12@B 1006ef64     libcpmtd:string.obj
 0002:0001cf68       ?unitbuf@?$_Iosb@H@std@@2W4_Fmtflags@12@B 1006ef68     libcpmtd:string.obj
 0002:0001cf6c       ?uppercase@?$_Iosb@H@std@@2W4_Fmtflags@12@B 1006ef6c     libcpmtd:string.obj
 0002:0001cf70       ?showbase@?$_Iosb@H@std@@2W4_Fmtflags@12@B 1006ef70     libcpmtd:string.obj
 0002:0001cf74       ?showpoint@?$_Iosb@H@std@@2W4_Fmtflags@12@B 1006ef74     libcpmtd:string.obj
 0002:0001cf78       ?showpos@?$_Iosb@H@std@@2W4_Fmtflags@12@B 1006ef78     libcpmtd:string.obj
 0002:0001cf7c       ?left@?$_Iosb@H@std@@2W4_Fmtflags@12@B 1006ef7c     libcpmtd:string.obj
 0002:0001cf80       ?right@?$_Iosb@H@std@@2W4_Fmtflags@12@B 1006ef80     libcpmtd:string.obj
 0002:0001cf84       ?internal@?$_Iosb@H@std@@2W4_Fmtflags@12@B 1006ef84     libcpmtd:string.obj
 0002:0001cf88       ?dec@?$_Iosb@H@std@@2W4_Fmtflags@12@B 1006ef88     libcpmtd:string.obj
 0002:0001cf8c       ?oct@?$_Iosb@H@std@@2W4_Fmtflags@12@B 1006ef8c     libcpmtd:string.obj
 0002:0001cf90       ?hex@?$_Iosb@H@std@@2W4_Fmtflags@12@B 1006ef90     libcpmtd:string.obj
 0002:0001cf94       ?scientific@?$_Iosb@H@std@@2W4_Fmtflags@12@B 1006ef94     libcpmtd:string.obj
 0002:0001cf98       ?fixed@?$_Iosb@H@std@@2W4_Fmtflags@12@B 1006ef98     libcpmtd:string.obj
 0002:0001cf9c       ?boolalpha@?$_Iosb@H@std@@2W4_Fmtflags@12@B 1006ef9c     libcpmtd:string.obj
 0002:0001cfa0       ?_Stdio@?$_Iosb@H@std@@2W4_Fmtflags@12@B 1006efa0     libcpmtd:string.obj
 0002:0001cfa4       ?adjustfield@?$_Iosb@H@std@@2W4_Fmtflags@12@B 1006efa4     libcpmtd:string.obj
 0002:0001cfa8       ?basefield@?$_Iosb@H@std@@2W4_Fmtflags@12@B 1006efa8     libcpmtd:string.obj
 0002:0001cfac       ?floatfield@?$_Iosb@H@std@@2W4_Fmtflags@12@B 1006efac     libcpmtd:string.obj
 0002:0001cfb0       ?goodbit@?$_Iosb@H@std@@2W4_Iostate@12@B 1006efb0     libcpmtd:string.obj
 0002:0001cfb4       ?eofbit@?$_Iosb@H@std@@2W4_Iostate@12@B 1006efb4     libcpmtd:string.obj
 0002:0001cfb8       ?failbit@?$_Iosb@H@std@@2W4_Iostate@12@B 1006efb8     libcpmtd:string.obj
 0002:0001cfbc       ?badbit@?$_Iosb@H@std@@2W4_Iostate@12@B 1006efbc     libcpmtd:string.obj
 0002:0001cfc0       ?_Hardfail@?$_Iosb@H@std@@2W4_Iostate@12@B 1006efc0     libcpmtd:string.obj
 0002:0001cfc4       ?in@?$_Iosb@H@std@@2W4_Openmode@12@B 1006efc4     libcpmtd:string.obj
 0002:0001cfc8       ?out@?$_Iosb@H@std@@2W4_Openmode@12@B 1006efc8     libcpmtd:string.obj
 0002:0001cfcc       ?ate@?$_Iosb@H@std@@2W4_Openmode@12@B 1006efcc     libcpmtd:string.obj
 0002:0001cfd0       ?app@?$_Iosb@H@std@@2W4_Openmode@12@B 1006efd0     libcpmtd:string.obj
 0002:0001cfd4       ?trunc@?$_Iosb@H@std@@2W4_Openmode@12@B 1006efd4     libcpmtd:string.obj
 0002:0001cfd8       ?_Nocreate@?$_Iosb@H@std@@2W4_Openmode@12@B 1006efd8     libcpmtd:string.obj
 0002:0001cfdc       ?_Noreplace@?$_Iosb@H@std@@2W4_Openmode@12@B 1006efdc     libcpmtd:string.obj
 0002:0001cfe0       ?binary@?$_Iosb@H@std@@2W4_Openmode@12@B 1006efe0     libcpmtd:string.obj
 0002:0001cfe4       ?beg@?$_Iosb@H@std@@2W4_Seekdir@12@B 1006efe4     libcpmtd:string.obj
 0002:0001cfe8       ?cur@?$_Iosb@H@std@@2W4_Seekdir@12@B 1006efe8     libcpmtd:string.obj
 0002:0001cfec       ?end@?$_Iosb@H@std@@2W4_Seekdir@12@B 1006efec     libcpmtd:string.obj
 0002:0001cff4       ??_7bad_alloc@std@@6B@     1006eff4     libcpmtd:string.obj
 0002:0001d000       ??_C@_1FE@OGIJMGPN@?$AAf?$AA?3?$AA?2?$AAs?$AAp?$AA?2?$AAv?$AAc?$AAt?$AAo?$AAo?$AAl?$AAs?$AA?2?$AAc?$AAr?$AAt?$AAc?$AAe?$AA?2?$AAc?$AAr?$AAt?$AAw?$AA3?$AA2?$AA?2?$AAs?$AAt?$AAd?$AAh?$AAp@ 1006f000     libcpmtd:string.obj
 0002:0001d058       ??_7logic_error@std@@6B@   1006f058     libcpmtd:string.obj
 0002:0001d064       ??_7invalid_argument@std@@6B@ 1006f064     libcpmtd:string.obj
 0002:0001d070       ??_7length_error@std@@6B@  1006f070     libcpmtd:string.obj
 0002:0001d07c       ??_7out_of_range@std@@6B@  1006f07c     libcpmtd:string.obj
 0002:0001d0d0       ??_C@_0BA@JFNIOLAK@string?5too?5long?$AA@ 1006f0d0     libcpmtd:string.obj
 0002:0001d12c       ??_C@_0BI@CFPLBAOH@invalid?5string?5position?$AA@ 1006f12c     libcpmtd:string.obj
 0002:0001d190       ??_C@_0BI@ILCMCLF@invalid?5string?5argument?$AA@ 1006f190     libcpmtd:string.obj
 0002:0001d21c       ??_R4bad_alloc@std@@6B@    1006f21c     libcpmtd:string.obj
 0002:0001d230       ??_R3bad_alloc@std@@8      1006f230     libcpmtd:string.obj
 0002:0001d240       ??_R2bad_alloc@std@@8      1006f240     libcpmtd:string.obj
 0002:0001d24c       ??_R1A@?0A@EA@bad_alloc@std@@8 1006f24c     libcpmtd:string.obj
 0002:0001d268       ??_R1A@?0A@EA@exception@std@@8 1006f268     libcpmtd:string.obj
 0002:0001d284       ??_R3exception@std@@8      1006f284     libcpmtd:string.obj
 0002:0001d294       ??_R2exception@std@@8      1006f294     libcpmtd:string.obj
 0002:0001d29c       ??_R4logic_error@std@@6B@  1006f29c     libcpmtd:string.obj
 0002:0001d2b0       ??_R3logic_error@std@@8    1006f2b0     libcpmtd:string.obj
 0002:0001d2c0       ??_R2logic_error@std@@8    1006f2c0     libcpmtd:string.obj
 0002:0001d2cc       ??_R1A@?0A@EA@logic_error@std@@8 1006f2cc     libcpmtd:string.obj
 0002:0001d2e8       ??_R4invalid_argument@std@@6B@ 1006f2e8     libcpmtd:string.obj
 0002:0001d2fc       ??_R3invalid_argument@std@@8 1006f2fc     libcpmtd:string.obj
 0002:0001d30c       ??_R2invalid_argument@std@@8 1006f30c     libcpmtd:string.obj
 0002:0001d31c       ??_R1A@?0A@EA@invalid_argument@std@@8 1006f31c     libcpmtd:string.obj
 0002:0001d338       ??_R4length_error@std@@6B@ 1006f338     libcpmtd:string.obj
 0002:0001d34c       ??_R3length_error@std@@8   1006f34c     libcpmtd:string.obj
 0002:0001d35c       ??_R2length_error@std@@8   1006f35c     libcpmtd:string.obj
 0002:0001d36c       ??_R1A@?0A@EA@length_error@std@@8 1006f36c     libcpmtd:string.obj
 0002:0001d388       ??_R4out_of_range@std@@6B@ 1006f388     libcpmtd:string.obj
 0002:0001d39c       ??_R3out_of_range@std@@8   1006f39c     libcpmtd:string.obj
 0002:0001d3ac       ??_R2out_of_range@std@@8   1006f3ac     libcpmtd:string.obj
 0002:0001d3bc       ??_R1A@?0A@EA@out_of_range@std@@8 1006f3bc     libcpmtd:string.obj
 0002:0001d62c       _TI3?AVlength_error@std@@  1006f62c     SwiNotify.obj
 0002:0001d63c       _CTA3?AVlength_error@std@@ 1006f63c     SwiNotify.obj
 0002:0001d64c       _CT??_R0?AVlength_error@std@@@8??0length_error@std@@QAA@ABV01@@Z44 1006f64c     SwiNotify.obj
 0002:0001d668       _CT??_R0?AVlogic_error@std@@@8??0logic_error@std@@QAA@ABV01@@Z44 1006f668     SwiNotify.obj
 0002:0001d684       _CT??_R0?AVexception@std@@@8??0exception@std@@QAA@ABV01@@Z12 1006f684     SwiNotify.obj
 0002:0001d6a0       _TI2?AVbad_alloc@std@@     1006f6a0     SwiNotify.obj
 0002:0001d6b0       _CTA2?AVbad_alloc@std@@    1006f6b0     SwiNotify.obj
 0002:0001d6bc       _CT??_R0?AVbad_alloc@std@@@8??0bad_alloc@std@@QAA@ABV01@@Z12 1006f6bc     SwiNotify.obj
 0002:0001d6d8       _TI3?AVout_of_range@std@@  1006f6d8     libcpmtd:string.obj
 0002:0001d6e8       _CTA3?AVout_of_range@std@@ 1006f6e8     libcpmtd:string.obj
 0002:0001d6f8       _CT??_R0?AVout_of_range@std@@@8??0out_of_range@std@@QAA@ABV01@@Z44 1006f6f8     libcpmtd:string.obj
 0002:0001d714       _TI3?AVinvalid_argument@std@@ 1006f714     libcpmtd:string.obj
 0002:0001d724       _CTA3?AVinvalid_argument@std@@ 1006f724     libcpmtd:string.obj
 0002:0001d734       _CT??_R0?AVinvalid_argument@std@@@8??0invalid_argument@std@@QAA@ABV01@@Z44 1006f734     libcpmtd:string.obj
 0002:0001d750       __IMPORT_DESCRIPTOR_ccoreutl 1006f750     ccoreutl:ccoreutl.dll
 0002:0001d764       __IMPORT_DESCRIPTOR_WS2    1006f764     ws2:WS2.dll
 0002:0001d778       __IMPORT_DESCRIPTOR_sw_utilityG 1006f778     sw_utilityG:sw_utilityG.dll
 0002:0001d78c       __IMPORT_DESCRIPTOR_COREDLL 1006f78c     coredll:COREDLL.dll
 0002:0001d7a0       __NULL_IMPORT_DESCRIPTOR   1006f7a0     ccoreutl:ccoreutl.dll
 0003:00000000       __imp_CreateFileW          10076000     coredll:COREDLL.dll
 0003:00000004       __imp_fflush               10076004     coredll:COREDLL.dll
 0003:00000008       __imp__getstdfilex         10076008     coredll:COREDLL.dll
 0003:0000000c       __imp_fputs                1007600c     coredll:COREDLL.dll
 0003:00000010       __imp_TerminateProcess     10076010     coredll:COREDLL.dll
 0003:00000014       __imp_OutputDebugStringW   10076014     coredll:COREDLL.dll
 0003:00000018       __imp__vsnwprintf          10076018     coredll:COREDLL.dll
 0003:0000001c       __imp_wcstombs             1007601c     coredll:COREDLL.dll
 0003:00000020       __imp_RaiseException       10076020     coredll:COREDLL.dll
 0003:00000024       __imp_TlsCall              10076024     coredll:COREDLL.dll
 0003:00000028       __imp_InterlockedCompareExchange 10076028     coredll:COREDLL.dll
 0003:0000002c       __imp_TlsGetValue          1007602c     coredll:COREDLL.dll
 0003:00000030       __imp_TlsSetValue          10076030     coredll:COREDLL.dll
 0003:00000034       __imp_GetModuleFileNameW   10076034     coredll:COREDLL.dll
 0003:00000038       __imp__snwprintf           10076038     coredll:COREDLL.dll
 0003:0000003c       __imp_?terminate@std@@YAXXZ 1007603c     coredll:COREDLL.dll
 0003:00000040       __imp___rt_udiv            10076040     coredll:COREDLL.dll
 0003:00000044       __imp_strlen               10076044     coredll:COREDLL.dll
 0003:00000048       __imp_strstr               10076048     coredll:COREDLL.dll
 0003:0000004c       __imp_strcmp               1007604c     coredll:COREDLL.dll
 0003:00000050       __imp_memcmp               10076050     coredll:COREDLL.dll
 0003:00000054       __imp_strspn               10076054     coredll:COREDLL.dll
 0003:00000058       __imp_LocalFree            10076058     coredll:COREDLL.dll
 0003:0000005c       __imp_LocalAllocTrace      1007605c     coredll:COREDLL.dll
 0003:00000060       __imp_strchr               10076060     coredll:COREDLL.dll
 0003:00000064       __imp_wcslen               10076064     coredll:COREDLL.dll
 0003:00000068       __imp_??3@YAXPAX@Z         10076068     coredll:COREDLL.dll
 0003:0000006c       __imp_??2@YAPAXI@Z         1007606c     coredll:COREDLL.dll
 0003:00000070       __imp_memset               10076070     coredll:COREDLL.dll
 0003:00000074       __imp_NKDbgPrintfW         10076074     coredll:COREDLL.dll
 0003:00000078       __imp_EnterCriticalSection 10076078     coredll:COREDLL.dll
 0003:0000007c       __imp_LeaveCriticalSection 1007607c     coredll:COREDLL.dll
 0003:00000080       __imp_GetLastError         10076080     coredll:COREDLL.dll
 0003:00000084       __imp_swscanf              10076084     coredll:COREDLL.dll
 0003:00000088       __imp__snprintf            10076088     coredll:COREDLL.dll
 0003:0000008c       __imp_??_V@YAXPAX@Z        1007608c     coredll:COREDLL.dll
 0003:00000090       __imp_??_U@YAPAXI@Z        10076090     coredll:COREDLL.dll
 0003:00000094       __imp_sscanf               10076094     coredll:COREDLL.dll
 0003:00000098       __imp_free                 10076098     coredll:COREDLL.dll
 0003:0000009c       __imp_malloc               1007609c     coredll:COREDLL.dll
 0003:000000a0       __imp_CloseHandle          100760a0     coredll:COREDLL.dll
 0003:000000a4       __imp_CreateThread         100760a4     coredll:COREDLL.dll
 0003:000000a8       __imp_InitializeCriticalSection 100760a8     coredll:COREDLL.dll
 0003:000000ac       __imp_DeleteCriticalSection 100760ac     coredll:COREDLL.dll
 0003:000000b0       __imp_Sleep                100760b0     coredll:COREDLL.dll
 0003:000000b4       __imp_strtoul              100760b4     coredll:COREDLL.dll
 0003:000000b8       __imp_abs                  100760b8     coredll:COREDLL.dll
 0003:000000bc       __imp_strncpy              100760bc     coredll:COREDLL.dll
 0003:000000c0       __imp___rt_udiv64by64      100760c0     coredll:COREDLL.dll
 0003:000000c4       __imp_memcpy               100760c4     coredll:COREDLL.dll
 0003:000000c8       __imp_wcscmp               100760c8     coredll:COREDLL.dll
 0003:000000cc       __imp_wcsncpy              100760cc     coredll:COREDLL.dll
 0003:000000d0       __imp_MultiByteToWideChar  100760d0     coredll:COREDLL.dll
 0003:000000d4       __imp_wcsstr               100760d4     coredll:COREDLL.dll
 0003:000000d8       __imp_sprintf              100760d8     coredll:COREDLL.dll
 0003:000000dc       __imp_wcscpy               100760dc     coredll:COREDLL.dll
 0003:000000e0       __imp_atol                 100760e0     coredll:COREDLL.dll
 0003:000000e4       __imp_strcat               100760e4     coredll:COREDLL.dll
 0003:000000e8       __imp_strcpy               100760e8     coredll:COREDLL.dll
 0003:000000ec       __imp___rt_sdiv            100760ec     coredll:COREDLL.dll
 0003:000000f0       __imp__wtol                100760f0     coredll:COREDLL.dll
 0003:000000f4       __imp_swprintf             100760f4     coredll:COREDLL.dll
 0003:000000f8       __imp_PurgeComm            100760f8     coredll:COREDLL.dll
 0003:000000fc       __imp_SetCommState         100760fc     coredll:COREDLL.dll
 0003:00000100       __imp_toupper              10076100     coredll:COREDLL.dll
 0003:00000104       __imp_SetupComm            10076104     coredll:COREDLL.dll
 0003:00000108       __imp_SetCommTimeouts      10076108     coredll:COREDLL.dll
 0003:0000010c       __imp_GetCommState         1007610c     coredll:COREDLL.dll
 0003:00000110       __imp_SetLastError         10076110     coredll:COREDLL.dll
 0003:00000114       __imp_InterlockedExchange  10076114     coredll:COREDLL.dll
 0003:00000118       __imp_wcscat               10076118     coredll:COREDLL.dll
 0003:0000011c       __imp_WriteFile            1007611c     coredll:COREDLL.dll
 0003:00000120       __imp_ReadFile             10076120     coredll:COREDLL.dll
 0003:00000124       __imp_GetTickCount         10076124     coredll:COREDLL.dll
 0003:00000128       __imp_GetProcAddressW      10076128     coredll:COREDLL.dll
 0003:0000012c       __imp_FreeLibrary          1007612c     coredll:COREDLL.dll
 0003:00000130       __imp_LoadLibraryW         10076130     coredll:COREDLL.dll
 0003:00000134       __imp___CxxThrowException  10076134     coredll:COREDLL.dll
 0003:00000138       __imp_??_7type_info@@6B@   10076138     coredll:COREDLL.dll
 0003:0000013c       __imp_??0exception@std@@QAA@ABV01@@Z 1007613c     coredll:COREDLL.dll
 0003:00000140       __imp_??1exception@std@@UAA@XZ 10076140     coredll:COREDLL.dll
 0003:00000144       __imp_??0exception@std@@QAA@XZ 10076144     coredll:COREDLL.dll
 0003:00000148       __imp_??0exception@std@@QAA@PBD@Z 10076148     coredll:COREDLL.dll
 0003:0000014c       __imp_?what@exception@std@@UBAPBDXZ 1007614c     coredll:COREDLL.dll
 0003:00000150       __imp_StringCchCopyW       10076150     coredll:COREDLL.dll
 0003:00000154       __imp_wcschr               10076154     coredll:COREDLL.dll
 0003:00000158       __imp___report_gsfailure   10076158     coredll:COREDLL.dll
 0003:0000015c       __imp_LocalReAlloc         1007615c     coredll:COREDLL.dll
 0003:00000160       __imp_LocalAlloc           10076160     coredll:COREDLL.dll
 0003:00000164       __imp_LocalSize            10076164     coredll:COREDLL.dll
 0003:00000168       __imp___security_gen_cookie 10076168     coredll:COREDLL.dll
 0003:0000016c       __imp_EventModify          1007616c     coredll:COREDLL.dll
 0003:00000170       __imp_StringCchVPrintfW    10076170     coredll:COREDLL.dll
 0003:00000174       __imp_StringCchVPrintfA    10076174     coredll:COREDLL.dll
 0003:00000178       __imp_RegCloseKey          10076178     coredll:COREDLL.dll
 0003:0000017c       __imp_RegQueryValueExW     1007617c     coredll:COREDLL.dll
 0003:00000180       __imp_RegCreateKeyExW      10076180     coredll:COREDLL.dll
 0003:00000184       __imp_RegSetValueExW       10076184     coredll:COREDLL.dll
 0003:00000188       __imp_rand                 10076188     coredll:COREDLL.dll
 0003:0000018c       __imp___itos               1007618c     coredll:COREDLL.dll
 0003:00000190       __imp___muls               10076190     coredll:COREDLL.dll
 0003:00000194       __imp___stoi               10076194     coredll:COREDLL.dll
 0003:00000198       __imp__wcsnicmp            10076198     coredll:COREDLL.dll
 0003:0000019c       __imp_WideCharToMultiByte  1007619c     coredll:COREDLL.dll
 0003:000001a0       __imp_CreateEventW         100761a0     coredll:COREDLL.dll
 0003:000001a4       __imp_WaitForSingleObject  100761a4     coredll:COREDLL.dll
 0003:000001a8       __imp___C_specific_handler 100761a8     coredll:COREDLL.dll
 0003:000001ac       __imp_WaitForMultipleObjects 100761ac     coredll:COREDLL.dll
 0003:000001b0       __imp_InterlockedDecrement 100761b0     coredll:COREDLL.dll
 0003:000001b4       __imp_InterlockedIncrement 100761b4     coredll:COREDLL.dll
 0003:000001b8       __imp_UnmapViewOfFile      100761b8     coredll:COREDLL.dll
 0003:000001bc       __imp_MapViewOfFile        100761bc     coredll:COREDLL.dll
 0003:000001c0       __imp_CreateFileMappingW   100761c0     coredll:COREDLL.dll
 0003:000001c4       __imp_GetFileSize          100761c4     coredll:COREDLL.dll
 0003:000001c8       __imp_SystemTimeToFileTime 100761c8     coredll:COREDLL.dll
 0003:000001cc       __imp_GetSystemTime        100761cc     coredll:COREDLL.dll
 0003:000001d0       __imp_memmove              100761d0     coredll:COREDLL.dll
 0003:000001d4       __imp_LoadStringW          100761d4     coredll:COREDLL.dll
 0003:000001d8       __imp_CreateSemaphoreW     100761d8     coredll:COREDLL.dll
 0003:000001dc       __imp__wcsicmp             100761dc     coredll:COREDLL.dll
 0003:000001e0       __imp_ReleaseSemaphore     100761e0     coredll:COREDLL.dll
 0003:000001e4       \177COREDLL_NULL_THUNK_DATA 100761e4     coredll:COREDLL.dll
 0003:000001e8       __imp_ntohl                100761e8     ws2:WS2.dll
 0003:000001ec       __imp_inet_ntoa            100761ec     ws2:WS2.dll
 0003:000001f0       \177WS2_NULL_THUNK_DATA    100761f0     ws2:WS2.dll
 0003:000001f4       __imp_?ConvertGSMMixedToUnicode@@YA_NIQBDIQAGIAAI@Z 100761f4     ccoreutl:ccoreutl.dll
 0003:000001f8       \177ccoreutl_NULL_THUNK_DATA 100761f8     ccoreutl:ccoreutl.dll
 0003:000001fc       __imp_?LogW@@YAXPBGZZ      100761fc     sw_utilityG:sw_utilityG.dll
 0003:00000200       __imp_?GetRegValue@@YAJPAUHKEY__@@PBG1PAGPAK@Z 10076200     sw_utilityG:sw_utilityG.dll
 0003:00000204       __imp_?SW_AtoT@@YAPAGPAGPADK@Z 10076204     sw_utilityG:sw_utilityG.dll
 0003:00000208       __imp_?LogStoreFileLine@@YAXPAGH@Z 10076208     sw_utilityG:sw_utilityG.dll
 0003:0000020c       __imp_?LogC@@YAXPBGZZ      1007620c     sw_utilityG:sw_utilityG.dll
 0003:00000210       __imp_?TBD_Assert@@YA_N_NQBG1H@Z 10076210     sw_utilityG:sw_utilityG.dll
 0003:00000214       __imp_?TBD_Output@@YAXW4TBD_CLASS_TYPE@@W4TBD_OUTPUT_LEVEL@@QBGZZ 10076214     sw_utilityG:sw_utilityG.dll
 0003:00000218       __imp_?SW_TtoA@@YAPADPADPAGK@Z 10076218     sw_utilityG:sw_utilityG.dll
 0003:0000021c       __imp_?DisplayRawData@@YAXIPAEHPBG@Z 1007621c     sw_utilityG:sw_utilityG.dll
 0003:00000220       __imp_?WriteLog@@YAXKPBGZZ 10076220     sw_utilityG:sw_utilityG.dll
 0003:00000224       \177sw_utilityG_NULL_THUNK_DATA 10076224     sw_utilityG:sw_utilityG.dll
 0003:00000228       __xc_a                     10076228     corelibc:crt0init.obj
 0003:00000244       __xc_z                     10076244     corelibc:crt0init.obj
 0003:00000248       __xi_a                     10076248     corelibc:crt0init.obj
 0003:0000024c       __xi_z                     1007624c     corelibc:crt0init.obj
 0003:00000250       __xp_a                     10076250     corelibc:crt0init.obj
 0003:00000254       __xp_z                     10076254     corelibc:crt0init.obj
 0003:00000258       __xt_a                     10076258     corelibc:crt0init.obj
 0003:0000025c       __xt_z                     1007625c     corelibc:crt0init.obj
 0003:0000026c       ?GOBI2SWIRoam@@3PAGA       1007626c     SDKRILCdma.obj
 0003:00000278       ?GOBI2SWICDMACarrierID@@3PAW4SWI_TYPE_CarrierID@@A 10076278     SDKRILCdma.obj
 0003:000002c0       ?GOBI2SWICDMACarrierName@@3PAPAGA 100762c0     SDKRILCdma.obj
 0003:00000308       ?SWI2GOBIOMADMSessionType@@3PAJA 10076308     SDKRILCdma.obj
 0003:000006b0       ?errGobiAPI@@3PAW4SWI_RCODE@@A 100766b0     SwiError.obj
 0003:00000728       ?errGobiModule1@@3PAW4SWI_RCODE@@A 10076728     SwiError.obj
 0003:00000874       ?errGobiModule2@@3PAW4SWI_RCODE@@A 10076874     SwiError.obj
 0003:00000888       ?GOBI2SWIPowerMode@@3PAW4SWI_TYPE_Power@@A 10076888     SwiError.obj
 0003:00000c1c       ?g_CB_SignalStrength@@3CA  10076c1c     SwiNotify.obj
 0003:00000c20       ?g_iCdmaRssi@@3HA          10076c20     SwiNotify.obj
 0003:00000c24       ?g_iCdmaEcio@@3HA          10076c24     SwiNotify.obj
 0003:00000c28       ?g_iHdrRssi@@3HA           10076c28     SwiNotify.obj
 0003:00000c2c       ?g_iHdrEcio@@3HA           10076c2c     SwiNotify.obj
 0003:00000c30       ?GOBI2SWIOTASPState@@3PAW4SWI_TYPE_OTASPState@@A 10076c30     SwiNotify.obj
 0003:00000c5c       ??_R0?AVlength_error@std@@@8 10076c5c     SwiNotify.obj
 0003:00000c7c       ??_R0?AVlogic_error@std@@@8 10076c7c     SwiNotify.obj
 0003:00000c9c       ??_R0?AVexception@std@@@8  10076c9c     SwiNotify.obj
 0003:00000cb8       ??_R0?AVbad_alloc@std@@@8  10076cb8     SwiNotify.obj
 0003:00000cd4       __security_cookie_complement 10076cd4     corelibc:seccook.obj
 0003:00000cd8       __security_cookie          10076cd8     corelibc:seccook.obj
 0003:00000e10       _crtAssertBusy             10076e10     LIBCMTD:dbgrptt.obj
 0003:00000e14       _CrtDbgMode                10076e14     LIBCMTD:dbgrptt.obj
 0003:00000e20       _CrtDbgFile                10076e20     LIBCMTD:dbgrptt.obj
 0003:00000e2c       _aexit_rtn                 10076e2c     LIBCMTD:crt0dat.obj
 0003:00000e3c       ??_R0?AVinvalid_argument@std@@@8 10076e3c     libcpmtd:string.obj
 0003:00000e60       ??_R0?AVout_of_range@std@@@8 10076e60     libcpmtd:string.obj
 0003:00000e80       ?g_WirelessTech@@3W4SWI_TYPE_WirelessTech@@A 10076e80     SDKRIL.obj
 0003:00000e84       ?g_IsRUIM@@3EA             10076e84     SDKRIL.obj
 0003:00000e88       ?g_StrFirmwareVersion@@3PADA 10076e88     SDKRIL.obj
 0003:00000ee0       ?g_StrBootVersion@@3PADA   10076ee0     SDKRIL.obj
 0003:00000f38       ?g_StrPRIVersion@@3PADA    10076f38     SDKRIL.obj
 0003:00000f90       ?g_NotifyCallback@@3P6AXPAUSwiNotifyVariant@@@ZA 10076f90     SDKRIL.obj
 0003:00000f94       ?g_bIsCMEErrNumeric@@3HA   10076f94     SDKRIL.obj
 0003:00000f98       ?g_GobiInstance@@3VCSwiGobiDll@@A 10076f98     SDKRIL.obj
 0003:000012c0       ?g_ATPortInstance@@3VCSwiATPort@@A 100772c0     SDKRIL.obj
 0003:0000150c       ?g_Notify@@3VCSwiNotify@@A 1007750c     SDKRIL.obj
 0003:00001528       ?theSWICR@@3VCriticalSection@@A 10077528     SDKRIL.obj
 0003:00001540       ?g_MSLSet@@3UMSLData@@A    10077540     SDKRILCdma.obj
 0003:00001584       ?g_SPCStr@@3PADA           10077584     SDKRILCdma.obj
 0003:00001590       ?g_msgListArray@@3PAUMSG_LIST_ENTRY@@A 10077590     SDKRILCdma.obj
 0003:000034d0       ?g_StoreRawSms@@3USWI_STRUCT_RawSms@@A 100794d0     SDKRILCdma.obj
 0003:000038e0       ?g_hSmsSendNotifyThread@@3PAXA 100798e0     SDKRILCdma.obj
 0003:000038e4       ?g_DataSessionID@@3KA      100798e4     SDKRILCdma.obj
 0003:000038e8       ?g_OMADMPRLsessionID@@3GA  100798e8     SDKRILCdma.obj
 0003:000038ea       ?g_bSCM@@3EA               100798ea     SDKRILCdma.obj
 0003:000038eb       ?g_bSCI@@3EA               100798eb     SDKRILCdma.obj
 0003:000038ec       ?g_OMADMDCsessionID@@3GA   100798ec     SDKRILCdma.obj
 0003:000038ee       ?g_bRegHomeSID@@3EA        100798ee     SDKRILCdma.obj
 0003:000038ef       ?g_bRegForSID@@3EA         100798ef     SDKRILCdma.obj
 0003:000038f0       ?g_bRegForNID@@3EA         100798f0     SDKRILCdma.obj
 0003:000038f1       ?g_bForceRev0@@3EA         100798f1     SDKRILCdma.obj
 0003:000038f2       ?g_bCustomSCP@@3EA         100798f2     SDKRILCdma.obj
 0003:000038f4       ?g_ulProtocol@@3KA         100798f4     SDKRILCdma.obj
 0003:000038f8       ?g_ulBroadCast@@3KA        100798f8     SDKRILCdma.obj
 0003:000038fc       ?g_ulApp@@3KA              100798fc     SDKRILCdma.obj
 0003:00003900       ?g_ulRoaming@@3KA          10079900     SDKRILCdma.obj
 0003:00003908       ?g_sAirServerList@@3USWI_STRUCT_AirServerList@@A 10079908     SDKRILGsm.obj
 0003:00003cf8       ?g_RATInfoList@@3URATINFOList@@A 10079cf8     SDKRILGsm.obj
 0003:00003e90       ?g_PlmnList@@3UNWINFOList@@A 10079e90     SDKRILGsm.obj
 0003:0000747c       ?g_PlmnMode@@3W4SWI_TYPE_PLMN_Mode@@A 1007d47c     SDKRILGsm.obj
 0003:00007480       ?g_ulDataSessionId@@3KA    1007d480     SDKRILGsm.obj
 0003:00007484       ?g_bSwiPhonebookReadySent@@3HA 1007d484     SDKRILGsm.obj
 0003:00007488       ?g_GsmSmsSource@@3KA       1007d488     SDKRILGsm.obj
 0003:0000748c       ?g_GsmPinType@@3KA         1007d48c     SDKRILGsm.obj
 0003:00007490       __@@_PchSym_@00@UluurxzoPyfrowUirotlyrUdrmwldhLnlyrovLGLkiluvhhrlmzoLhwpLSzineErTUwvyftPdnGOFUhwpiroUhgwzucOlyq@ 1007d490     stdafx.obj
 0003:00007494       ?mpFNSetSessionStateCB@CSwiGobiDll@@1P6AKP6AXKK@Z@ZA 1007d494     SwiGobiDll.obj
 0003:00007498       ?mpFNSetDataBearerCB@CSwiGobiDll@@1P6AKP6AXK@Z@ZA 1007d498     SwiGobiDll.obj
 0003:0000749c       ?mpFNSetDormancyStatusCB@CSwiGobiDll@@1P6AKP6AXK@Z@ZA 1007d49c     SwiGobiDll.obj
 0003:000074a0       ?mpFNSetMobileIPStatusCB@CSwiGobiDll@@1P6AKP6AXK@Z@ZA 1007d4a0     SwiGobiDll.obj
 0003:000074a4       ?mpFNSetActivationStatusCB@CSwiGobiDll@@1P6AKP6AXK@Z@ZA 1007d4a4     SwiGobiDll.obj
 0003:000074a8       ?mpFNSetPowerCB@CSwiGobiDll@@1P6AKP6AXK@Z@ZA 1007d4a8     SwiGobiDll.obj
 0003:000074ac       ?mpFNSetRoamingIndicatorCB@CSwiGobiDll@@1P6AKP6AXK@Z@ZA 1007d4ac     SwiGobiDll.obj
 0003:000074b0       ?mpFNSetSignalStrengthCB@CSwiGobiDll@@1P6AKP6AXCK@ZEPAC@ZA 1007d4b0     SwiGobiDll.obj
 0003:000074b4       ?mpFNSetRFInfoCB@CSwiGobiDll@@1P6AKP6AXKKK@Z@ZA 1007d4b4     SwiGobiDll.obj
 0003:000074b8       ?mpFNSetNewSMSCB@CSwiGobiDll@@1P6AKP6AXKK@Z@ZA 1007d4b8     SwiGobiDll.obj
 0003:000074bc       ?mpFNSetNewSMSCBCB@CSwiGobiDll@@1P6AKP6AXEKEGPAE@Z@ZA 1007d4bc     SwiGobiDll.obj
 0003:000074c0       ?mpFNSetVoiceMsgCB@CSwiGobiDll@@1P6AKP6AXEPAE00@Z@ZA 1007d4c0     SwiGobiDll.obj
 0003:000074c4       ?mpFNSetDataCapabilitiesCB@CSwiGobiDll@@1P6AKP6AXEPAE@Z@ZA 1007d4c4     SwiGobiDll.obj
 0003:000074c8       ?mpFNSetByteTotalsCB@CSwiGobiDll@@1P6AKP6AX_K0@ZE@ZA 1007d4c8     SwiGobiDll.obj
 0003:000074cc       ?mpFNSetOMADMStateCB@CSwiGobiDll@@1P6AKP6AXKK@Z@ZA 1007d4cc     SwiGobiDll.obj
 0003:000074d0       ?mpFNSetOMADMNIAlertCB@CSwiGobiDll@@1P6AKP6AXKG@Z@ZA 1007d4d0     SwiGobiDll.obj
 0003:000074d4       ?mpFNSetCallInfoCB@CSwiGobiDll@@1P6AKP6AXPAUarrCallInfo@@PAUarrRemotePartyNum@@PAUarrRemotePartyName@@PAUarrAlertingType@@PAUarrSvcOption@@PAUarrCallEndReason@@PAUarrAlphaIDInfo@@PAUarrPeerNumInfo@@PAUarrDiagInfo@@77PAUarrAlertingPattern@@@Z@ZA 1007d4d4     SwiGobiDll.obj
 0003:000074d8       ?mpFNSetInfoRecCB@CSwiGobiDll@@1P6AKP6AXPAEPAUsignalInfo@@PAUcallerIDInfo@@PAD330PAUpeerNumInfo@@44PAUredirectNumInfo@@0000PAUlineCtlInfo@@PAUextDisplayInfo@@@Z@ZA 1007d4d8     SwiGobiDll.obj
 0003:000074dc       ?mpFNSetUSSDInfoCB@CSwiGobiDll@@1P6AKP6AXPAEPAUUSSInfo@@@Z@ZA 1007d4dc     SwiGobiDll.obj
 0003:000074e0       ?mpFNSetPhonebookRecordReadCB@CSwiGobiDll@@1P6AKP6AXEGPAUarrPBInfo@@@Z@ZA 1007d4e0     SwiGobiDll.obj
 0003:000074e4       ?mpFNSetAllPbInitDoneCB@CSwiGobiDll@@1P6AKP6AXEPAEPAG@Z@ZA 1007d4e4     SwiGobiDll.obj
 0003:000074e8       ?mpFNSetEmergencyListCB@CSwiGobiDll@@1P6AKP6AXEPAUemergencyNumberEntry@@@Z@ZA 1007d4e8     SwiGobiDll.obj
 0003:000074ec       ?mpFNSetNITZCB@CSwiGobiDll@@1P6AKP6AXGEEEEEEEE@Z@ZA 1007d4ec     SwiGobiDll.obj
 0003:000074f0       ?mpFNSetEmergencyModeCB@CSwiGobiDll@@1P6AKP6AXPAE@Z@ZA 1007d4f0     SwiGobiDll.obj
 0003:000074f4       ?mpFNSetOMAEXEventCB@CSwiGobiDll@@1P6AKP6AXPAUFUMOInfo@@PAUOMAInfo@@@Z@ZA 1007d4f4     SwiGobiDll.obj
 0003:000074f8       ?m_NotifyCallback@CSwiNotify@@2P6AXPAUSwiNotifyVariant@@@ZA 1007d4f8     SwiNotify.obj
 0003:000074fc       ?m_pGobi@CSwiNotify@@0PAVCSwiGobiDll@@A 1007d4fc     SwiNotify.obj
 0003:00007500       ?m_pSwiNotify@CSwiNotify@@0PAV1@A 1007d500     SwiNotify.obj
 0003:00007504       ?g_CB_RadioInterface@@3KA  1007d504     SwiNotify.obj
 0003:00007508       ?g_DataCapsMask@@3W4eDataCaps@@A 1007d508     SwiNotify.obj
 0003:0000750c       ?g_OMADMsessionType@@3KA   1007d50c     SwiNotify.obj
 0003:00007510       ?g_sessionID@@3GA          1007d510     SwiNotify.obj
 0003:000076b4       __onexitend                1007d6b4     <common>
 0003:000076b8       __onexitbegin              1007d6b8     <common>
 0003:000076bc       _exitflag                  1007d6bc     <common>
 0003:000076c0       _pRawDllMain               1007d6c0     <common>
 0003:000076c4       _pfnReportHook             1007d6c4     <common>
 0003:000076c8       _pReportHookListW          1007d6c8     <common>
 0003:000076cc       _pReportHookList           1007d6cc     <common>

 entry point at        0001:00044584

 Static symbols

 0001:fffff058       __unwind$18609             10000058 f   libcpmtd:string.obj
 0001:fffff058       __unwind$18984             10000058 f   libcpmtd:string.obj
 0001:fffff060       __unwind$19542             10000060 f   libcpmtd:string.obj
 0001:fffff068       __unwind$18537             10000068 f   libcpmtd:string.obj
 0001:fffff108       __catch$18380              10000108 f   libcpmtd:string.obj
 0001:fffff144       __catch$18378              10000144 f   libcpmtd:string.obj
 0001:00002370       ?BSCompareListValues@@YAHPBX0@Z 10003370 f   parse.obj
 0001:00002480       ?BSCompareListStrings@@YAHPBX0@Z 10003480 f   parse.obj
 0001:000354ac       __unwind$55180             100364ac f   SwiNotify.obj
 0001:000355d8       __unwind$55270             100365d8 f   SwiNotify.obj
 0001:0003572c       __unwind$55303             1003672c f   SwiNotify.obj
 0001:00035880       __unwind$55336             10036880 f   SwiNotify.obj
 0001:000359fc       __unwind$55371             100369fc f   SwiNotify.obj
 0001:00035b40       __unwind$55402             10036b40 f   SwiNotify.obj
 0001:0003622c       __unwind$55485             1003722c f   SwiNotify.obj
 0001:00036488       __unwind$55540             10037488 f   SwiNotify.obj
 0001:00036580       __unwind$55564             10037580 f   SwiNotify.obj
 0001:0003679c       __unwind$55602             1003779c f   SwiNotify.obj
 0001:000367b4       __unwind$55603             100377b4 f   SwiNotify.obj
 0001:000367cc       __unwind$55604             100377cc f   SwiNotify.obj
 0001:000367e4       __unwind$55605             100377e4 f   SwiNotify.obj
 0001:000367fc       __unwind$55606             100377fc f   SwiNotify.obj
 0001:00036850       __unwind$55747             10037850 f   SwiNotify.obj
 0001:000370e0       __unwind$55809             100380e0 f   SwiNotify.obj
 0001:000370f8       __unwind$55810             100380f8 f   SwiNotify.obj
 0001:00037110       __unwind$55811             10038110 f   SwiNotify.obj
 0001:00037128       __unwind$55812             10038128 f   SwiNotify.obj
 0001:00037140       __unwind$55814             10038140 f   SwiNotify.obj
 0001:00037158       __unwind$55815             10038158 f   SwiNotify.obj
 0001:00037170       __unwind$55816             10038170 f   SwiNotify.obj
 0001:00037188       __unwind$55818             10038188 f   SwiNotify.obj
 0001:000371a0       __unwind$55819             100381a0 f   SwiNotify.obj
 0001:000371b8       __unwind$55821             100381b8 f   SwiNotify.obj
 0001:000371d0       __unwind$55822             100381d0 f   SwiNotify.obj
 0001:000371e8       __unwind$55823             100381e8 f   SwiNotify.obj
 0001:00037200       __unwind$55825             10038200 f   SwiNotify.obj
 0001:00037218       __unwind$55826             10038218 f   SwiNotify.obj
 0001:000391e8       __unwind$56160             1003a1e8 f   SwiNotify.obj
 0001:00039208       __unwind$56161             1003a208 f   SwiNotify.obj
 0001:00039228       __unwind$56162             1003a228 f   SwiNotify.obj
 0001:00039240       __unwind$56164             1003a240 f   SwiNotify.obj
 0001:00039258       __unwind$56165             1003a258 f   SwiNotify.obj
 0001:00039270       __unwind$56167             1003a270 f   SwiNotify.obj
 0001:00039974       __unwind$56255             1003a974 f   SwiNotify.obj
 0001:00039994       __unwind$56256             1003a994 f   SwiNotify.obj
 0001:000399b4       __unwind$56257             1003a9b4 f   SwiNotify.obj
 0001:000399cc       __unwind$56259             1003a9cc f   SwiNotify.obj
 0001:000399e4       __unwind$56260             1003a9e4 f   SwiNotify.obj
 0001:000399fc       __unwind$56262             1003a9fc f   SwiNotify.obj
 0001:0003a364       __unwind$56346             1003b364 f   SwiNotify.obj
 0001:0003a38c       __unwind$56347             1003b38c f   SwiNotify.obj
 0001:0003a3b4       __unwind$56348             1003b3b4 f   SwiNotify.obj
 0001:0003a3d4       __unwind$56350             1003b3d4 f   SwiNotify.obj
 0001:0003a3f4       __unwind$56351             1003b3f4 f   SwiNotify.obj
 0001:0003a414       __unwind$56353             1003b414 f   SwiNotify.obj
 0001:0003a938       __unwind$56432             1003b938 f   SwiNotify.obj
 0001:0003a958       __unwind$56433             1003b958 f   SwiNotify.obj
 0001:0003a978       __unwind$56434             1003b978 f   SwiNotify.obj
 0001:0003a990       __unwind$56436             1003b990 f   SwiNotify.obj
 0001:0003a9a8       __unwind$56437             1003b9a8 f   SwiNotify.obj
 0001:0003a9c0       __unwind$56439             1003b9c0 f   SwiNotify.obj
 0001:0003adf4       __unwind$56502             1003bdf4 f   SwiNotify.obj
 0001:0003ae14       __unwind$56503             1003be14 f   SwiNotify.obj
 0001:0003ae34       __unwind$56504             1003be34 f   SwiNotify.obj
 0001:0003ae4c       __unwind$56506             1003be4c f   SwiNotify.obj
 0001:0003ae64       __unwind$56507             1003be64 f   SwiNotify.obj
 0001:0003ae7c       __unwind$56509             1003be7c f   SwiNotify.obj
 0001:0003b2b4       __unwind$56573             1003c2b4 f   SwiNotify.obj
 0001:0003b2d4       __unwind$56574             1003c2d4 f   SwiNotify.obj
 0001:0003b2f4       __unwind$56575             1003c2f4 f   SwiNotify.obj
 0001:0003b30c       __unwind$56577             1003c30c f   SwiNotify.obj
 0001:0003b324       __unwind$56578             1003c324 f   SwiNotify.obj
 0001:0003b33c       __unwind$56580             1003c33c f   SwiNotify.obj
 0001:0003b7bc       __unwind$56642             1003c7bc f   SwiNotify.obj
 0001:0003b7dc       __unwind$56643             1003c7dc f   SwiNotify.obj
 0001:0003b7fc       __unwind$56644             1003c7fc f   SwiNotify.obj
 0001:0003b814       __unwind$56646             1003c814 f   SwiNotify.obj
 0001:0003b82c       __unwind$56647             1003c82c f   SwiNotify.obj
 0001:0003b844       __unwind$56649             1003c844 f   SwiNotify.obj
 0001:0003bc80       __unwind$56711             1003cc80 f   SwiNotify.obj
 0001:0003bca0       __unwind$56712             1003cca0 f   SwiNotify.obj
 0001:0003bcc0       __unwind$56713             1003ccc0 f   SwiNotify.obj
 0001:0003bcd8       __unwind$56715             1003ccd8 f   SwiNotify.obj
 0001:0003bcf0       __unwind$56716             1003ccf0 f   SwiNotify.obj
 0001:0003bd08       __unwind$56718             1003cd08 f   SwiNotify.obj
 0001:0003c0d8       __unwind$56779             1003d0d8 f   SwiNotify.obj
 0001:0003c0f8       __unwind$56780             1003d0f8 f   SwiNotify.obj
 0001:0003c118       __unwind$56781             1003d118 f   SwiNotify.obj
 0001:0003c130       __unwind$56783             1003d130 f   SwiNotify.obj
 0001:0003c148       __unwind$56784             1003d148 f   SwiNotify.obj
 0001:0003c160       __unwind$56786             1003d160 f   SwiNotify.obj
 0001:0003c844       __unwind$55679             1003d844 f i SwiNotify.obj
 0001:0003c9cc       __unwind$55712             1003d9cc f i SwiNotify.obj
 0001:0003ca84       __unwind$55730             1003da84 f i SwiNotify.obj
 0001:0003ce10       __unwind$56883             1003de10 f i SwiNotify.obj
 0001:0003ce58       __unwind$56900             1003de58 f i SwiNotify.obj
 0001:0003d14c       __unwind$56954             1003e14c f i SwiNotify.obj
 0001:0003d164       __unwind$56955             1003e164 f i SwiNotify.obj
 0001:0003d17c       __unwind$56956             1003e17c f i SwiNotify.obj
 0001:0003d344       __unwind$56997             1003e344 f i SwiNotify.obj
 0001:0003d38c       __unwind$57014             1003e38c f i SwiNotify.obj
 0001:0003d724       __unwind$57088             1003e724 f i SwiNotify.obj
 0001:0003d73c       __unwind$57089             1003e73c f i SwiNotify.obj
 0001:0003d754       __unwind$57090             1003e754 f i SwiNotify.obj
 0001:0003d864       __unwind$57138             1003e864 f i SwiNotify.obj
 0001:0003d87c       __unwind$57139             1003e87c f i SwiNotify.obj
 0001:0003d9dc       __unwind$57187             1003e9dc f i SwiNotify.obj
 0001:0003d9f4       __unwind$57188             1003e9f4 f i SwiNotify.obj
 0001:0003dcec       __unwind$57290             1003ecec f i SwiNotify.obj
 0001:0003ddb8       __catch$57312              1003edb8 f i SwiNotify.obj
 0001:0003e160       __unwind$57393             1003f160 f i SwiNotify.obj
 0001:0003e22c       __catch$57414              1003f22c f i SwiNotify.obj
 0001:0003ea6c       __catch$57622              1003fa6c f i SwiNotify.obj
 0001:0003eba8       __unwind$57648             1003fba8 f i SwiNotify.obj
 0001:0003ec6c       __unwind$57681             1003fc6c f i SwiNotify.obj
 0001:0003ee1c       __unwind$57740             1003fe1c f i SwiNotify.obj
 0001:0003ee70       __unwind$57759             1003fe70 f i SwiNotify.obj
 0001:0003f7fc       __catch$57954              100407fc f i SwiNotify.obj
 0001:0003f938       __unwind$57980             10040938 f i SwiNotify.obj
 0001:0003fa9c       __unwind$58039             10040a9c f i SwiNotify.obj
 0001:0003fcb8       __unwind$58087             10040cb8 f i SwiNotify.obj
 0001:0003ff24       __unwind$58145             10040f24 f i SwiNotify.obj
 0001:0003ffb0       __unwind$58167             10040fb0 f i SwiNotify.obj
 0001:000401e0       __catch$58196              100411e0 f i SwiNotify.obj
 0001:00040218       __catch$58194              10041218 f i SwiNotify.obj
 0001:00040c18       __unwind$58515             10041c18 f i SwiNotify.obj
 0001:00040ec0       __catch$58590              10041ec0 f i SwiNotify.obj
 0001:00040ee8       __unwind$58591             10041ee8 f i SwiNotify.obj
 0001:00040f00       __unwind$58592             10041f00 f i SwiNotify.obj
 0001:00040f18       __unwind$58593             10041f18 f i SwiNotify.obj
 0001:000411d4       __unwind$58699             100421d4 f i SwiNotify.obj
 0001:000411f4       __unwind$58700             100421f4 f i SwiNotify.obj
 0001:00041214       __unwind$58701             10042214 f i SwiNotify.obj
 0001:00041234       __unwind$58702             10042234 f i SwiNotify.obj
 0001:00041254       __unwind$58703             10042254 f i SwiNotify.obj
 0001:000413e8       __catch$58759              100423e8 f i SwiNotify.obj
 0001:00041494       __unwind$58760             10042494 f i SwiNotify.obj
 0001:000414ac       __unwind$58761             100424ac f i SwiNotify.obj
 0001:000414c4       __unwind$58762             100424c4 f i SwiNotify.obj
 0001:000414dc       __unwind$58763             100424dc f i SwiNotify.obj
 0001:000414f4       __unwind$58765             100424f4 f i SwiNotify.obj
 0001:0004150c       __unwind$58767             1004250c f i SwiNotify.obj
 0001:000416fc       __unwind$58857             100426fc f i SwiNotify.obj
 0001:0004171c       __unwind$58858             1004271c f i SwiNotify.obj
 0001:0004173c       __unwind$58859             1004273c f i SwiNotify.obj
 0001:000417b0       __unwind$58895             100427b0 f i SwiNotify.obj
 0001:00041a9c       ?BSCompareChars@@YAHPBX0@Z 10042a9c f   util.obj
 0001:00044674       _initterm                  10045674 f   corelibc:crt0dat.obj
 0001:00044714       doexit                     10045714 f   corelibc:crt0dat.obj
 0001:00049988       ?FindHandler@@YAEPAUEHExceptionRecord@@PAKPAU_CONTEXT@@PAU_DISPATCHER_CONTEXT@@PBU_s_FuncInfo@@H@Z 1004a988 f   LIBCMTD:frame_ce.obj
 0001:00049f7c       ?TypeMatch@@YAHPBU_s_HandlerType@@PBU_s_CatchableType@@PBU_s_ThrowInfo@@@Z 1004af7c f   LIBCMTD:frame_ce.obj
 0001:0004a340       ?FrameUnwindFilter@@YAHPAU_EXCEPTION_POINTERS@@@Z 1004b340 f   LIBCMTD:frame_ce.obj
 0001:0004a3cc       ?CallCatchBlock@@YAPAXPAUEHExceptionRecord@@PAKPAU_CONTEXT@@PBU_s_FuncInfo@@PAXHK@Z 1004b3cc f   LIBCMTD:frame_ce.obj
 0001:0004a968       ?CanThisExceptionObjectBeDestructed@@YAEPAUEHExceptionRecord@@E@Z 1004b968 f   LIBCMTD:frame_ce.obj
 0001:0004abf4       ?BuildCatchObject@@YAXPAUEHExceptionRecord@@PAKPBU_s_HandlerType@@PBU_s_CatchableType@@@Z 1004bbf4 f   LIBCMTD:frame_ce.obj
 0001:0004af44       ?AdjustPointer@@YAPAXPAXABUPMD@@@Z 1004bf44 f   LIBCMTD:frame_ce.obj
 0001:0004ed50       __crtInitCritSecNoSpinCount 1004fd50 f   LIBCMTD:initcrit.obj
 0001:0004f494       xtow_s                     10050494 f   LIBCMTD:xtows.obj
 0001:00050188       __unwind$18810             10051188 f   libcpmtd:string.obj
 0001:00050218       __unwind$19010             10051218 f   libcpmtd:string.obj
 0001:000502d8       __unwind$19588             100512d8 f   libcpmtd:string.obj
 0001:00050538       ??__Eg_GobiInstance@@YAXXZ 10051538 f   SDKRIL.obj
 0001:00050558       ??__Eg_ATPortInstance@@YAXXZ 10051558 f   SDKRIL.obj
 0001:00050578       ??__Eg_Notify@@YAXXZ       10051578 f   SDKRIL.obj
 0001:00050598       ??__EtheSWICR@@YAXXZ       10051598 f   SDKRIL.obj
 0001:000505b8       ??__Einitlocks@std@@YAXXZ  100515b8 f   libcpmtd:xlock.obj
 0001:000505f4       ??__Fg_GobiInstance@@YAXXZ 100515f4 f   SDKRIL.obj
 0001:00050608       ??__Fg_ATPortInstance@@YAXXZ 10051608 f   SDKRIL.obj
 0001:0005061c       ??__Fg_Notify@@YAXXZ       1005161c f   SDKRIL.obj
 0001:00050630       ??__FtheSWICR@@YAXXZ       10051630 f   SDKRIL.obj
 0001:00050644       ??__Finitlocks@std@@YAXXZ  10051644 f   libcpmtd:xlock.obj

 Exports

  ordinal    name

        1    ??0CSwiGobiDll@@QAA@XZ (public: __cdecl CSwiGobiDll::CSwiGobiDll(void))
        2    ??1CSwiGobiDll@@QAA@XZ (public: __cdecl CSwiGobiDll::~CSwiGobiDll(void))
        3    ??4CSwiGobiDll@@QAAAAV0@ABV0@@Z (public: class CSwiGobiDll & __cdecl CSwiGobiDll::operator=(class CSwiGobiDll const &))
        4    ?ActivateAutomatic@CSwiGobiDll@@QAAKPAD@Z (public: unsigned long __cdecl CSwiGobiDll::ActivateAutomatic(char *))
        5    ?ActivateManual@CSwiGobiDll@@QAAKPADG00KPAE00@Z (public: unsigned long __cdecl CSwiGobiDll::ActivateManual(char *,unsigned short,char *,char *,unsigned long,unsigned char *,char *,char *))
        6    ?AnserCall@CSwiGobiDll@@QAAKPAE0@Z (public: unsigned long __cdecl CSwiGobiDll::AnserCall(unsigned char *,unsigned char *))
        7    ?AnswerUSSD@CSwiGobiDll@@QAAKPAUUSSInfo@@@Z (public: unsigned long __cdecl CSwiGobiDll::AnswerUSSD(struct USSInfo *))
        8    ?CancelUSSD@CSwiGobiDll@@QAAKXZ (public: unsigned long __cdecl CSwiGobiDll::CancelUSSD(void))
        9    ?ChangeBarringPwd@CSwiGobiDll@@QAAKPAUcallBarringPwd@@PAGPAUalphaIDInfo@@PAE3PAUccSUPSType@@@Z (public: unsigned long __cdecl CSwiGobiDll::ChangeBarringPwd(struct callBarringPwd *,unsigned short *,struct alphaIDInfo *,unsigned char *,unsigned char *,struct ccSUPSType *))
       10    ?Cleanup@CSwiGobiDll@@IAAXXZ (protected: void __cdecl CSwiGobiDll::Cleanup(void))
       11    ?Connect@CSwiGobiDll@@QAAKXZ (public: unsigned long __cdecl CSwiGobiDll::Connect(void))
       12    ?DMSUIMChangePIN@CSwiGobiDll@@QAAKKPAD0PAK1@Z (public: unsigned long __cdecl CSwiGobiDll::DMSUIMChangePIN(unsigned long,char *,char *,unsigned long *,unsigned long *))
       13    ?DMSUIMGetControlKeyStatus@CSwiGobiDll@@QAAKKPAK00@Z (public: unsigned long __cdecl CSwiGobiDll::DMSUIMGetControlKeyStatus(unsigned long,unsigned long *,unsigned long *,unsigned long *))
       14    ?DMSUIMGetICCID@CSwiGobiDll@@QAAKEPAD@Z (public: unsigned long __cdecl CSwiGobiDll::DMSUIMGetICCID(unsigned char,char *))
       15    ?DMSUIMGetPINStatus@CSwiGobiDll@@QAAKKPAK00@Z (public: unsigned long __cdecl CSwiGobiDll::DMSUIMGetPINStatus(unsigned long,unsigned long *,unsigned long *,unsigned long *))
       16    ?DMSUIMSetControlKeyProtection@CSwiGobiDll@@QAAKKKPADPAK@Z (public: unsigned long __cdecl CSwiGobiDll::DMSUIMSetControlKeyProtection(unsigned long,unsigned long,char *,unsigned long *))
       17    ?DMSUIMSetPINProtection@CSwiGobiDll@@QAAKKKPADPAK1@Z (public: unsigned long __cdecl CSwiGobiDll::DMSUIMSetPINProtection(unsigned long,unsigned long,char *,unsigned long *,unsigned long *))
       18    ?DMSUIMUnblockControlKey@CSwiGobiDll@@QAAKKPADPAK@Z (public: unsigned long __cdecl CSwiGobiDll::DMSUIMUnblockControlKey(unsigned long,char *,unsigned long *))
       19    ?DMSUIMUnblockPIN@CSwiGobiDll@@QAAKKPAD0PAK1@Z (public: unsigned long __cdecl CSwiGobiDll::DMSUIMUnblockPIN(unsigned long,char *,char *,unsigned long *,unsigned long *))
       20    ?DMSUIMVerifyPIN@CSwiGobiDll@@QAAKKPADPAK1@Z (public: unsigned long __cdecl CSwiGobiDll::DMSUIMVerifyPIN(unsigned long,char *,unsigned long *,unsigned long *))
       21    ?DeletePhonebookRecord@CSwiGobiDll@@QAAKPAEPAG1@Z (public: unsigned long __cdecl CSwiGobiDll::DeletePhonebookRecord(unsigned char *,unsigned short *,unsigned short *))
       22    ?DeleteSMS@CSwiGobiDll@@QAAKKPAK0@Z (public: unsigned long __cdecl CSwiGobiDll::DeleteSMS(unsigned long,unsigned long *,unsigned long *))
       23    ?DialCall@CSwiGobiDll@@QAAKPAUtDialReqParam@@PAEPAUalphaIDInfo@@1PAUccSUPSType@@@Z (public: unsigned long __cdecl CSwiGobiDll::DialCall(struct tDialReqParam *,unsigned char *,struct alphaIDInfo *,unsigned char *,struct ccSUPSType *))
       24    ?DisableCallbacks@CSwiGobiDll@@QAAXXZ (public: void __cdecl CSwiGobiDll::DisableCallbacks(void))
       25    ?Disconnect@CSwiGobiDll@@QAAKXZ (public: unsigned long __cdecl CSwiGobiDll::Disconnect(void))
       26    ?EndCall@CSwiGobiDll@@QAAKPAE0@Z (public: unsigned long __cdecl CSwiGobiDll::EndCall(unsigned char *,unsigned char *))
       27    ?ForceXTRADownload@CSwiGobiDll@@QAAKXZ (public: unsigned long __cdecl CSwiGobiDll::ForceXTRADownload(void))
       28    ?Get3Gpp2SubscriptionInfo@CSwiGobiDll@@QAAKPAEPAUMinBasedImsi@@PAUTrueImsi@@00@Z (public: unsigned long __cdecl CSwiGobiDll::Get3Gpp2SubscriptionInfo(unsigned char *,struct MinBasedImsi *,struct TrueImsi *,unsigned char *,unsigned char *))
       29    ?GetACCOLC@CSwiGobiDll@@QAAKPAE@Z (public: unsigned long __cdecl CSwiGobiDll::GetACCOLC(unsigned char *))
       30    ?GetAGPSConfig@CSwiGobiDll@@QAAKPAK0@Z (public: unsigned long __cdecl CSwiGobiDll::GetAGPSConfig(unsigned long *,unsigned long *))
       31    ?GetANAAAAuthenticationStatus@CSwiGobiDll@@QAAKPAK@Z (public: unsigned long __cdecl CSwiGobiDll::GetANAAAAuthenticationStatus(unsigned long *))
       32    ?GetActivationState@CSwiGobiDll@@QAAKPAK@Z (public: unsigned long __cdecl CSwiGobiDll::GetActivationState(unsigned long *))
       33    ?GetActiveMobileIPProfile@CSwiGobiDll@@QAAKPAE@Z (public: unsigned long __cdecl CSwiGobiDll::GetActiveMobileIPProfile(unsigned char *))
       34    ?GetAllCallInfo@CSwiGobiDll@@QAAKPAUarrCallInfo@@PAUarrRemotePartyNum@@PAUarrRemotePartyName@@PAUarrAlertingType@@PAUarrUUSInfo@@PAUarrSvcOption@@PAE6PAUarrCallEndReason@@PAUarrAlphaIDInfo@@PAUarrPeerNumInfo@@PAUarrDiagInfo@@99PAUarrAlertingPattern@@@Z (public: unsigned long __cdecl CSwiGobiDll::GetAllCallInfo(struct arrCallInfo *,struct arrRemotePartyNum *,struct arrRemotePartyName *,struct arrAlertingType *,struct arrUUSInfo *,struct arrSvcOption *,unsigned char *,unsigned char *,struct arrCallEndReason *,struct arrAlphaIDInfo *,struct arrPeerNumInfo *,struct arrDiagInfo *,struct arrPeerNumInfo *,struct arrPeerNumInfo *,struct arrAlertingPattern *))
       35    ?GetAudioProfile@CSwiGobiDll@@QAAKPAE@Z (public: unsigned long __cdecl CSwiGobiDll::GetAudioProfile(unsigned char *))
       36    ?GetAutoInputGain@CSwiGobiDll@@QAAKPAE@Z (public: unsigned long __cdecl CSwiGobiDll::GetAutoInputGain(unsigned char *))
       37    ?GetAutoOutputGain@CSwiGobiDll@@QAAKPAE@Z (public: unsigned long __cdecl CSwiGobiDll::GetAutoOutputGain(unsigned char *))
       38    ?GetAutoconnect@CSwiGobiDll@@QAAKPAK@Z (public: unsigned long __cdecl CSwiGobiDll::GetAutoconnect(unsigned long *))
       39    ?GetByteTotals@CSwiGobiDll@@QAAKPAK0@Z (public: unsigned long __cdecl CSwiGobiDll::GetByteTotals(unsigned long *,unsigned long *))
       40    ?GetCDMANetworkParameters@CSwiGobiDll@@QAAKPAE000000PAK111@Z (public: unsigned long __cdecl CSwiGobiDll::GetCDMANetworkParameters(unsigned char *,unsigned char *,unsigned char *,unsigned char *,unsigned char *,unsigned char *,unsigned char *,unsigned long *,unsigned long *,unsigned long *,unsigned long *))
       41    ?GetCLIR@CSwiGobiDll@@QAAKPAUstatusResp@@PAGPAUalphaIDInfo@@PAE3PAUccSUPSType@@@Z (public: unsigned long __cdecl CSwiGobiDll::GetCLIR(struct statusResp *,unsigned short *,struct alphaIDInfo *,unsigned char *,unsigned char *,struct ccSUPSType *))
       42    ?GetCallBarring@CSwiGobiDll@@QAAKPAE00PAGPAUalphaIDInfo@@00PAUccSUPSType@@@Z (public: unsigned long __cdecl CSwiGobiDll::GetCallBarring(unsigned char *,unsigned char *,unsigned char *,unsigned short *,struct alphaIDInfo *,unsigned char *,unsigned char *,struct ccSUPSType *))
       43    ?GetCallForwarding@CSwiGobiDll@@QAAKPAE0PAUgetCallFWInfo@@0PAUalphaIDInfo@@00PAUccSUPSType@@PAUgetExtCallFWInfo@@@Z (public: unsigned long __cdecl CSwiGobiDll::GetCallForwarding(unsigned char *,unsigned char *,struct getCallFWInfo *,unsigned char *,struct alphaIDInfo *,unsigned char *,unsigned char *,struct ccSUPSType *,struct getExtCallFWInfo *))
       44    ?GetCallWaiting@CSwiGobiDll@@QAAKPAE0PAGPAUalphaIDInfo@@00PAUccSUPSType@@@Z (public: unsigned long __cdecl CSwiGobiDll::GetCallWaiting(unsigned char *,unsigned char *,unsigned short *,struct alphaIDInfo *,unsigned char *,unsigned char *,struct ccSUPSType *))
       45    ?GetCellLocationInfo@CSwiGobiDll@@QAAKPAUgeranCellInfo@@PAUumtsCellInfo@@PAUcdmaCellInfo@@PAK@Z (public: unsigned long __cdecl CSwiGobiDll::GetCellLocationInfo(struct geranCellInfo *,struct umtsCellInfo *,struct cdmaCellInfo *,unsigned long *))
       46    ?GetConnectedDeviceID@CSwiGobiDll@@QAAKKPAD@Z (public: unsigned long __cdecl CSwiGobiDll::GetConnectedDeviceID(unsigned long,char *))
       47    ?GetConnectionRate@CSwiGobiDll@@QAAKPAK000@Z (public: unsigned long __cdecl CSwiGobiDll::GetConnectionRate(unsigned long *,unsigned long *,unsigned long *,unsigned long *))
       48    ?GetCwePkgsInfo@CSwiGobiDll@@QAAKPAGPAE010101010101@Z (public: unsigned long __cdecl CSwiGobiDll::GetCwePkgsInfo(unsigned short *,unsigned char *,unsigned short *,unsigned char *,unsigned short *,unsigned char *,unsigned short *,unsigned char *,unsigned short *,unsigned char *,unsigned short *,unsigned char *,unsigned short *,unsigned char *))
       49    ?GetDLLVersion@CSwiGobiDll@@QAAKXZ (public: unsigned long __cdecl CSwiGobiDll::GetDLLVersion(void))
       50    ?GetDataBearerTechnology@CSwiGobiDll@@QAAKPAK@Z (public: unsigned long __cdecl CSwiGobiDll::GetDataBearerTechnology(unsigned long *))
       51    ?GetDefaultProfile@CSwiGobiDll@@QAAKKPAK0000EPADE1E1@Z (public: unsigned long __cdecl CSwiGobiDll::GetDefaultProfile(unsigned long,unsigned long *,unsigned long *,unsigned long *,unsigned long *,unsigned long *,unsigned char,char *,unsigned char,char *,unsigned char,char *))
       52    ?GetDeviceCapabilities@CSwiGobiDll@@QAAKPAK0000PAE@Z (public: unsigned long __cdecl CSwiGobiDll::GetDeviceCapabilities(unsigned long *,unsigned long *,unsigned long *,unsigned long *,unsigned long *,unsigned char *))
       53    ?GetDormancyState@CSwiGobiDll@@QAAKPAK@Z (public: unsigned long __cdecl CSwiGobiDll::GetDormancyState(unsigned long *))
       54    ?GetDunCallInfo@CSwiGobiDll@@QAAKPAKPAE101111PA_KPAG221100002221@Z (public: unsigned long __cdecl CSwiGobiDll::GetDunCallInfo(unsigned long *,unsigned char *,unsigned char *,unsigned long *,unsigned char *,unsigned char *,unsigned char *,unsigned char *,unsigned __int64 *,unsigned short *,unsigned __int64 *,unsigned __int64 *,unsigned char *,unsigned char *,unsigned long *,unsigned long *,unsigned long *,unsigned long *,unsigned __int64 *,unsigned __int64 *,unsigned __int64 *,unsigned char *))
       55    ?GetERIFile@CSwiGobiDll@@QAAKPAKPAE@Z (public: unsigned long __cdecl CSwiGobiDll::GetERIFile(unsigned long *,unsigned char *))
       56    ?GetEchoCancelMode@CSwiGobiDll@@QAAKPAE@Z (public: unsigned long __cdecl CSwiGobiDll::GetEchoCancelMode(unsigned char *))
       57    ?GetFirmwareInfo@CSwiGobiDll@@QAAKPAK0000@Z (public: unsigned long __cdecl CSwiGobiDll::GetFirmwareInfo(unsigned long *,unsigned long *,unsigned long *,unsigned long *,unsigned long *))
       58    ?GetFirmwareRevision@CSwiGobiDll@@QAAKEPAD@Z (public: unsigned long __cdecl CSwiGobiDll::GetFirmwareRevision(unsigned char,char *))
       59    ?GetFirmwareRevisions@CSwiGobiDll@@QAAKEPADE0E0@Z (public: unsigned long __cdecl CSwiGobiDll::GetFirmwareRevisions(unsigned char,char *,unsigned char,char *,unsigned char,char *))
       60    ?GetHardwareRevision@CSwiGobiDll@@QAAKEPAD@Z (public: unsigned long __cdecl CSwiGobiDll::GetHardwareRevision(unsigned char,char *))
       61    ?GetHomeNetwork@CSwiGobiDll@@QAAKPAG0EPAD00@Z (public: unsigned long __cdecl CSwiGobiDll::GetHomeNetwork(unsigned short *,unsigned short *,unsigned char,char *,unsigned short *,unsigned short *))
       62    ?GetIMSI@CSwiGobiDll@@QAAKEPAD@Z (public: unsigned long __cdecl CSwiGobiDll::GetIMSI(unsigned char,char *))
       63    ?GetIPAddress@CSwiGobiDll@@QAAKPAK@Z (public: unsigned long __cdecl CSwiGobiDll::GetIPAddress(unsigned long *))
       64    ?GetIPConfiguration@CSwiGobiDll@@QAAKPAK0000@Z (public: unsigned long __cdecl CSwiGobiDll::GetIPConfiguration(unsigned long *,unsigned long *,unsigned long *,unsigned long *,unsigned long *))
       65    ?GetImageInfoW@CSwiGobiDll@@QAAKPBGPAK1111@Z (public: unsigned long __cdecl CSwiGobiDll::GetImageInfoW(unsigned short const *,unsigned long *,unsigned long *,unsigned long *,unsigned long *,unsigned long *))
       66    ?GetImagePreference@CSwiGobiDll@@QAAKPAKPAE@Z (public: unsigned long __cdecl CSwiGobiDll::GetImagePreference(unsigned long *,unsigned char *))
       67    ?GetImageStoreW@CSwiGobiDll@@QAAKGPAG@Z (public: unsigned long __cdecl CSwiGobiDll::GetImageStoreW(unsigned short,unsigned short *))
       68    ?GetLastMobileIPError@CSwiGobiDll@@QAAKPAK@Z (public: unsigned long __cdecl CSwiGobiDll::GetLastMobileIPError(unsigned long *))
       69    ?GetManufacturer@CSwiGobiDll@@QAAKEPAD@Z (public: unsigned long __cdecl CSwiGobiDll::GetManufacturer(unsigned char,char *))
       70    ?GetMicVolume@CSwiGobiDll@@QAAKPAG@Z (public: unsigned long __cdecl CSwiGobiDll::GetMicVolume(unsigned short *))
       71    ?GetMobileIP@CSwiGobiDll@@QAAKPAK@Z (public: unsigned long __cdecl CSwiGobiDll::GetMobileIP(unsigned long *))
       72    ?GetMobileIPParameters@CSwiGobiDll@@QAAKPAKPAE11111@Z (public: unsigned long __cdecl CSwiGobiDll::GetMobileIPParameters(unsigned long *,unsigned char *,unsigned char *,unsigned char *,unsigned char *,unsigned char *,unsigned char *))
       73    ?GetMobileIPProfile@CSwiGobiDll@@QAAKEPAEPAK110EPAD11@Z (public: unsigned long __cdecl CSwiGobiDll::GetMobileIPProfile(unsigned char,unsigned char *,unsigned long *,unsigned long *,unsigned long *,unsigned char *,unsigned char,char *,unsigned long *,unsigned long *))
       74    ?GetModelID@CSwiGobiDll@@QAAKEPAD@Z (public: unsigned long __cdecl CSwiGobiDll::GetModelID(unsigned char,char *))
       75    ?GetNMEAConfig@CSwiGobiDll@@QAAKPAE00PAG@Z (public: unsigned long __cdecl CSwiGobiDll::GetNMEAConfig(unsigned char *,unsigned char *,unsigned char *,unsigned short *))
       76    ?GetNetworkPreference@CSwiGobiDll@@QAAKPAK00@Z (public: unsigned long __cdecl CSwiGobiDll::GetNetworkPreference(unsigned long *,unsigned long *,unsigned long *))
       77    ?GetNetworkTime@CSwiGobiDll@@QAAKPA_KPAK@Z (public: unsigned long __cdecl CSwiGobiDll::GetNetworkTime(unsigned __int64 *,unsigned long *))
       78    ?GetNoiseSuppression@CSwiGobiDll@@QAAKPAE@Z (public: unsigned long __cdecl CSwiGobiDll::GetNoiseSuppression(unsigned char *))
       79    ?GetOfflineReason@CSwiGobiDll@@QAAKPAK0@Z (public: unsigned long __cdecl CSwiGobiDll::GetOfflineReason(unsigned long *,unsigned long *))
       80    ?GetPDSDefaults@CSwiGobiDll@@QAAKPAKPAE00@Z (public: unsigned long __cdecl CSwiGobiDll::GetPDSDefaults(unsigned long *,unsigned char *,unsigned long *,unsigned long *))
       81    ?GetPDSState@CSwiGobiDll@@QAAKPAK0@Z (public: unsigned long __cdecl CSwiGobiDll::GetPDSState(unsigned long *,unsigned long *))
       82    ?GetPRLVersion@CSwiGobiDll@@QAAKPAG@Z (public: unsigned long __cdecl CSwiGobiDll::GetPRLVersion(unsigned short *))
       83    ?GetPacketStatus@CSwiGobiDll@@QAAKPAK00000@Z (public: unsigned long __cdecl CSwiGobiDll::GetPacketStatus(unsigned long *,unsigned long *,unsigned long *,unsigned long *,unsigned long *,unsigned long *))
       84    ?GetPhonebookCapabilities@CSwiGobiDll@@QAAKPAEPAG1100@Z (public: unsigned long __cdecl CSwiGobiDll::GetPhonebookCapabilities(unsigned char *,unsigned short *,unsigned short *,unsigned short *,unsigned char *,unsigned char *))
       85    ?GetPortAutomaticTracking@CSwiGobiDll@@QAAKPAK@Z (public: unsigned long __cdecl CSwiGobiDll::GetPortAutomaticTracking(unsigned long *))
       86    ?GetPower@CSwiGobiDll@@QAAKPAK@Z (public: unsigned long __cdecl CSwiGobiDll::GetPower(unsigned long *))
       87    ?GetRFInfo@CSwiGobiDll@@QAAKPAE0@Z (public: unsigned long __cdecl CSwiGobiDll::GetRFInfo(unsigned char *,unsigned char *))
       88    ?GetRTREConfig@CSwiGobiDll@@QAAKPAE0@Z (public: unsigned long __cdecl CSwiGobiDll::GetRTREConfig(unsigned char *,unsigned char *))
       89    ?GetRXPCMFilter@CSwiGobiDll@@QAAKPAG0PAK0@Z (public: unsigned long __cdecl CSwiGobiDll::GetRXPCMFilter(unsigned short *,unsigned short *,unsigned long *,unsigned short *))
       90    ?GetSMS@CSwiGobiDll@@QAAKKKPAK00PAE@Z (public: unsigned long __cdecl CSwiGobiDll::GetSMS(unsigned long,unsigned long,unsigned long *,unsigned long *,unsigned long *,unsigned char *))
       91    ?GetSMSCAddress@CSwiGobiDll@@QAAKEPADE0@Z (public: unsigned long __cdecl CSwiGobiDll::GetSMSCAddress(unsigned char,char *,unsigned char,char *))
       92    ?GetSMSList@CSwiGobiDll@@QAAKKPAK0PAE@Z (public: unsigned long __cdecl CSwiGobiDll::GetSMSList(unsigned long,unsigned long *,unsigned long *,unsigned char *))
       93    ?GetSerialNumbers@CSwiGobiDll@@QAAKEPADE0E0@Z (public: unsigned long __cdecl CSwiGobiDll::GetSerialNumbers(unsigned char,char *,unsigned char,char *,unsigned char,char *))
       94    ?GetServiceAutomaticTracking@CSwiGobiDll@@QAAKPAK@Z (public: unsigned long __cdecl CSwiGobiDll::GetServiceAutomaticTracking(unsigned long *))
       95    ?GetServingNetwork@CSwiGobiDll@@QAAKPAK000PAE10PAG2EPAD@Z (public: unsigned long __cdecl CSwiGobiDll::GetServingNetwork(unsigned long *,unsigned long *,unsigned long *,unsigned long *,unsigned char *,unsigned char *,unsigned long *,unsigned short *,unsigned short *,unsigned char,char *))
       96    ?GetServingNetworkCaps@CSwiGobiDll@@QAAKPAE0@Z (public: unsigned long __cdecl CSwiGobiDll::GetServingNetworkCaps(unsigned char *,unsigned char *))
       97    ?GetSessionDuration@CSwiGobiDll@@QAAKPA_K@Z (public: unsigned long __cdecl CSwiGobiDll::GetSessionDuration(unsigned __int64 *))
       98    ?GetSessionState@CSwiGobiDll@@QAAKPAK@Z (public: unsigned long __cdecl CSwiGobiDll::GetSessionState(unsigned long *))
       99    ?GetSideToneGain@CSwiGobiDll@@QAAKPAG@Z (public: unsigned long __cdecl CSwiGobiDll::GetSideToneGain(unsigned short *))
      100    ?GetSignalStrengths@CSwiGobiDll@@QAAKPAKPAC0@Z (public: unsigned long __cdecl CSwiGobiDll::GetSignalStrengths(unsigned long *,signed char *,unsigned long *))
      101    ?GetTXPCMFilter@CSwiGobiDll@@QAAKPAG0PAK0@Z (public: unsigned long __cdecl CSwiGobiDll::GetTXPCMFilter(unsigned short *,unsigned short *,unsigned long *,unsigned short *))
      102    ?GetVoiceNumber@CSwiGobiDll@@QAAKEPADE0@Z (public: unsigned long __cdecl CSwiGobiDll::GetVoiceNumber(unsigned char,char *,unsigned char,char *))
      103    ?GetWaitingMessage@CSwiGobiDll@@QAAKPAUwaitingMsgInfo@@@Z (public: unsigned long __cdecl CSwiGobiDll::GetWaitingMessage(struct waitingMsgInfo *))
      104    ?GetWirelessTech@CSwiGobiDll@@QAA?AW4SWI_TYPE_WirelessTech@@XZ (public: enum SWI_TYPE_WirelessTech __cdecl CSwiGobiDll::GetWirelessTech(void))
      105    ?GetXTRAAutomaticDownload@CSwiGobiDll@@QAAKPAKPAG@Z (public: unsigned long __cdecl CSwiGobiDll::GetXTRAAutomaticDownload(unsigned long *,unsigned short *))
      106    ?GetXTRANetwork@CSwiGobiDll@@QAAKPAK@Z (public: unsigned long __cdecl CSwiGobiDll::GetXTRANetwork(unsigned long *))
      107    ?GetXTRAValidity@CSwiGobiDll@@QAAKPAG00@Z (public: unsigned long __cdecl CSwiGobiDll::GetXTRAValidity(unsigned short *,unsigned short *,unsigned short *))
      108    ?Initialize@CSwiGobiDll@@QAA_NXZ (public: bool __cdecl CSwiGobiDll::Initialize(void))
      109    ?InitiateDomainAttach@CSwiGobiDll@@QAAKK@Z (public: unsigned long __cdecl CSwiGobiDll::InitiateDomainAttach(unsigned long))
      110    ?InitiateNetworkRegistration@CSwiGobiDll@@QAAKKGGK@Z (public: unsigned long __cdecl CSwiGobiDll::InitiateNetworkRegistration(unsigned long,unsigned short,unsigned short,unsigned long))
      111    ?IsInitialized@CSwiGobiDll@@QAA_NXZ (public: bool __cdecl CSwiGobiDll::IsInitialized(void))
      112    ?ManageCalls@CSwiGobiDll@@QAAKPAE0PAG@Z (public: unsigned long __cdecl CSwiGobiDll::ManageCalls(unsigned char *,unsigned char *,unsigned short *))
      113    ?ModifySMSStatus@CSwiGobiDll@@QAAKKKK@Z (public: unsigned long __cdecl CSwiGobiDll::ModifySMSStatus(unsigned long,unsigned long,unsigned long))
      114    ?OMADMCancelSession@CSwiGobiDll@@QAAKXZ (public: unsigned long __cdecl CSwiGobiDll::OMADMCancelSession(void))
      115    ?OMADMGetFeatureSettings@CSwiGobiDll@@QAAKPAK0@Z (public: unsigned long __cdecl CSwiGobiDll::OMADMGetFeatureSettings(unsigned long *,unsigned long *))
      116    ?OMADMGetPendingNIA@CSwiGobiDll@@QAAKPAKPAG@Z (public: unsigned long __cdecl CSwiGobiDll::OMADMGetPendingNIA(unsigned long *,unsigned short *))
      117    ?OMADMGetSessionInfo@CSwiGobiDll@@QAAKPAK00PAEPAG2@Z (public: unsigned long __cdecl CSwiGobiDll::OMADMGetSessionInfo(unsigned long *,unsigned long *,unsigned long *,unsigned char *,unsigned short *,unsigned short *))
      118    ?OMADMSendSelection@CSwiGobiDll@@QAAKKG@Z (public: unsigned long __cdecl CSwiGobiDll::OMADMSendSelection(unsigned long,unsigned short))
      119    ?OMADMSetPRLUpdateFeature@CSwiGobiDll@@QAAKK@Z (public: unsigned long __cdecl CSwiGobiDll::OMADMSetPRLUpdateFeature(unsigned long))
      120    ?OMADMSetProvisioningFeature@CSwiGobiDll@@QAAKK@Z (public: unsigned long __cdecl CSwiGobiDll::OMADMSetProvisioningFeature(unsigned long))
      121    ?OMADMStartSession@CSwiGobiDll@@QAAKK@Z (public: unsigned long __cdecl CSwiGobiDll::OMADMStartSession(unsigned long))
      122    ?OMAEXGetSettings@CSwiGobiDll@@QAAKPAE00000@Z (public: unsigned long __cdecl CSwiGobiDll::OMAEXGetSettings(unsigned char *,unsigned char *,unsigned char *,unsigned char *,unsigned char *,unsigned char *))
      123    ?OMAEXInit@CSwiGobiDll@@QAAKXZ (public: unsigned long __cdecl CSwiGobiDll::OMAEXInit(void))
      124    ?OMAEXSelection@CSwiGobiDll@@QAAKPAE@Z (public: unsigned long __cdecl CSwiGobiDll::OMAEXSelection(unsigned char *))
      125    ?OMAEXSessionCancel@CSwiGobiDll@@QAAKXZ (public: unsigned long __cdecl CSwiGobiDll::OMAEXSessionCancel(void))
      126    ?OMAEXSessionGetInfo@CSwiGobiDll@@QAAKPAUomaSessionInfo@@@Z (public: unsigned long __cdecl CSwiGobiDll::OMAEXSessionGetInfo(struct omaSessionInfo *))
      127    ?OMAEXSessionStart@CSwiGobiDll@@QAAKPAE@Z (public: unsigned long __cdecl CSwiGobiDll::OMAEXSessionStart(unsigned char *))
      128    ?OMAEXSetEventReport@CSwiGobiDll@@QAAKXZ (public: unsigned long __cdecl CSwiGobiDll::OMAEXSetEventReport(void))
      129    ?OMAEXSetSettings@CSwiGobiDll@@QAAKPAE00000@Z (public: unsigned long __cdecl CSwiGobiDll::OMAEXSetSettings(unsigned char *,unsigned char *,unsigned char *,unsigned char *,unsigned char *,unsigned char *))
      130    ?OMAEXShutdown@CSwiGobiDll@@QAAKXZ (public: unsigned long __cdecl CSwiGobiDll::OMAEXShutdown(void))
      131    ?OrigUSSD@CSwiGobiDll@@QAAKPAUUSSInfo@@PAGPAUalphaIDInfo@@0PAE3PAUccSUPSType@@@Z (public: unsigned long __cdecl CSwiGobiDll::OrigUSSD(struct USSInfo *,unsigned short *,struct alphaIDInfo *,struct USSInfo *,unsigned char *,unsigned char *,struct ccSUPSType *))
      132    ?PDSInjectTimeReference@CSwiGobiDll@@QAAK_KG@Z (public: unsigned long __cdecl CSwiGobiDll::PDSInjectTimeReference(unsigned __int64,unsigned short))
      133    ?PerformNetworkRATScan@CSwiGobiDll@@QAAKPAE000@Z (public: unsigned long __cdecl CSwiGobiDll::PerformNetworkRATScan(unsigned char *,unsigned char *,unsigned char *,unsigned char *))
      134    ?PerformNetworkScan@CSwiGobiDll@@QAAKPAE0@Z (public: unsigned long __cdecl CSwiGobiDll::PerformNetworkScan(unsigned char *,unsigned char *))
      135    ?PlayAudioTone@CSwiGobiDll@@QAAKPAE@Z (public: unsigned long __cdecl CSwiGobiDll::PlayAudioTone(unsigned char *))
      136    ?ReadPhonebookRecords@CSwiGobiDll@@QAAKPAEPAG111@Z (public: unsigned long __cdecl CSwiGobiDll::ReadPhonebookRecords(unsigned char *,unsigned short *,unsigned short *,unsigned short *,unsigned short *))
      137    ?ResetPDSData@CSwiGobiDll@@QAAKPAK0@Z (public: unsigned long __cdecl CSwiGobiDll::ResetPDSData(unsigned long *,unsigned long *))
      138    ?ResetToFactoryDefaults@CSwiGobiDll@@QAAKPAD@Z (public: unsigned long __cdecl CSwiGobiDll::ResetToFactoryDefaults(char *))
      139    ?SaveSMS@CSwiGobiDll@@QAAKKKKPAEPAK@Z (public: unsigned long __cdecl CSwiGobiDll::SaveSMS(unsigned long,unsigned long,unsigned long,unsigned char *,unsigned long *))
      140    ?SendFlash@CSwiGobiDll@@QAAKPAEPAD00@Z (public: unsigned long __cdecl CSwiGobiDll::SendFlash(unsigned char *,char *,unsigned char *,unsigned char *))
      141    ?SendSMS@CSwiGobiDll@@QAAKKKPAEEPAK@Z (public: unsigned long __cdecl CSwiGobiDll::SendSMS(unsigned long,unsigned long,unsigned char *,unsigned char,unsigned long *))
      142    ?Set3Gpp2SubscriptionInfo@CSwiGobiDll@@QAAKPAEPAUMinBasedImsi@@PAUTrueImsi@@00@Z (public: unsigned long __cdecl CSwiGobiDll::Set3Gpp2SubscriptionInfo(unsigned char *,struct MinBasedImsi *,struct TrueImsi *,unsigned char *,unsigned char *))
      143    ?SetACCOLC@CSwiGobiDll@@QAAKPADE@Z (public: unsigned long __cdecl CSwiGobiDll::SetACCOLC(char *,unsigned char))
      144    ?SetAGPSConfig@CSwiGobiDll@@QAAKKK@Z (public: unsigned long __cdecl CSwiGobiDll::SetAGPSConfig(unsigned long,unsigned long))
      145    ?SetActivationStatusCB@CSwiGobiDll@@SAKP6AXK@Z@Z (public: static unsigned long __cdecl CSwiGobiDll::SetActivationStatusCB(void (__cdecl*)(unsigned long)))
      146    ?SetActiveMobileIPProfile@CSwiGobiDll@@QAAKPADE@Z (public: unsigned long __cdecl CSwiGobiDll::SetActiveMobileIPProfile(char *,unsigned char))
      147    ?SetAllPbInitDoneCB@CSwiGobiDll@@SAKP6AXEPAEPAG@Z@Z (public: static unsigned long __cdecl CSwiGobiDll::SetAllPbInitDoneCB(void (__cdecl*)(unsigned char,unsigned char *,unsigned short *)))
      148    ?SetAudioProfile@CSwiGobiDll@@QAAKPAE@Z (public: unsigned long __cdecl CSwiGobiDll::SetAudioProfile(unsigned char *))
      149    ?SetAutoInputGain@CSwiGobiDll@@QAAKPAE@Z (public: unsigned long __cdecl CSwiGobiDll::SetAutoInputGain(unsigned char *))
      150    ?SetAutoOutputGain@CSwiGobiDll@@QAAKPAE@Z (public: unsigned long __cdecl CSwiGobiDll::SetAutoOutputGain(unsigned char *))
      151    ?SetAutoconnect@CSwiGobiDll@@QAAKK@Z (public: unsigned long __cdecl CSwiGobiDll::SetAutoconnect(unsigned long))
      152    ?SetByteTotalsCB@CSwiGobiDll@@SAKP6AX_K0@ZE@Z (public: static unsigned long __cdecl CSwiGobiDll::SetByteTotalsCB(void (__cdecl*)(unsigned __int64,unsigned __int64),unsigned char))
      153    ?SetCDMANetworkParameters@CSwiGobiDll@@QAAKPADPAE1PAK222@Z (public: unsigned long __cdecl CSwiGobiDll::SetCDMANetworkParameters(char *,unsigned char *,unsigned char *,unsigned long *,unsigned long *,unsigned long *,unsigned long *))
      154    ?SetCallInfoCB@CSwiGobiDll@@SAKP6AXPAUarrCallInfo@@PAUarrRemotePartyNum@@PAUarrRemotePartyName@@PAUarrAlertingType@@PAUarrSvcOption@@PAUarrCallEndReason@@PAUarrAlphaIDInfo@@PAUarrPeerNumInfo@@PAUarrDiagInfo@@77PAUarrAlertingPattern@@@Z@Z (public: static unsigned long __cdecl CSwiGobiDll::SetCallInfoCB(void (__cdecl*)(struct arrCallInfo *,struct arrRemotePartyNum *,struct arrRemotePartyName *,struct arrAlertingType *,struct arrSvcOption *,struct arrCallEndReason *,struct arrAlphaIDInfo *,struct arrPeerNumInfo *,struct arrDiagInfo *,struct arrPeerNumInfo *,struct arrPeerNumInfo *,struct arrAlertingPattern *)))
      155    ?SetDataBearerCB@CSwiGobiDll@@SAKP6AXK@Z@Z (public: static unsigned long __cdecl CSwiGobiDll::SetDataBearerCB(void (__cdecl*)(unsigned long)))
      156    ?SetDataCapsCB@CSwiGobiDll@@SAKP6AXEPAE@Z@Z (public: static unsigned long __cdecl CSwiGobiDll::SetDataCapsCB(void (__cdecl*)(unsigned char,unsigned char *)))
      157    ?SetDefaultProfile@CSwiGobiDll@@QAAKKPAK0000PAD111@Z (public: unsigned long __cdecl CSwiGobiDll::SetDefaultProfile(unsigned long,unsigned long *,unsigned long *,unsigned long *,unsigned long *,unsigned long *,char *,char *,char *,char *))
      158    ?SetDeviceRemovalCallback@CSwiGobiDll@@QAAKP6AXK@Z@Z (public: unsigned long __cdecl CSwiGobiDll::SetDeviceRemovalCallback(void (__cdecl*)(unsigned long)))
      159    ?SetDormancyStatusCB@CSwiGobiDll@@SAKP6AXK@Z@Z (public: static unsigned long __cdecl CSwiGobiDll::SetDormancyStatusCB(void (__cdecl*)(unsigned long)))
      160    ?SetEchoCancelMode@CSwiGobiDll@@QAAKPAE@Z (public: unsigned long __cdecl CSwiGobiDll::SetEchoCancelMode(unsigned char *))
      161    ?SetEmergencyListCB@CSwiGobiDll@@SAKP6AXEPAUemergencyNumberEntry@@@Z@Z (public: static unsigned long __cdecl CSwiGobiDll::SetEmergencyListCB(void (__cdecl*)(unsigned char,struct emergencyNumberEntry *)))
      162    ?SetEmergencyModeCB@CSwiGobiDll@@SAKP6AXPAE@Z@Z (public: static unsigned long __cdecl CSwiGobiDll::SetEmergencyModeCB(void (__cdecl*)(unsigned char *)))
      163    ?SetImagePreference@CSwiGobiDll@@QAAKKPAEKEPAK0@Z (public: unsigned long __cdecl CSwiGobiDll::SetImagePreference(unsigned long,unsigned char *,unsigned long,unsigned char,unsigned long *,unsigned char *))
      164    ?SetInfoRecCB@CSwiGobiDll@@SAKP6AXPAEPAUsignalInfo@@PAUcallerIDInfo@@PAD330PAUpeerNumInfo@@44PAUredirectNumInfo@@0000PAUlineCtlInfo@@PAUextDisplayInfo@@@Z@Z (public: static unsigned long __cdecl CSwiGobiDll::SetInfoRecCB(void (__cdecl*)(unsigned char *,struct signalInfo *,struct callerIDInfo *,char *,char *,char *,unsigned char *,struct peerNumInfo *,struct peerNumInfo *,struct peerNumInfo *,struct redirectNumInfo *,unsigned char *,unsigned char *,unsigned char *,unsigned char *,struct lineCtlInfo *,struct extDisplayInfo *)))
      165    ?SetMICMuteStatus@CSwiGobiDll@@QAAKPAE@Z (public: unsigned long __cdecl CSwiGobiDll::SetMICMuteStatus(unsigned char *))
      166    ?SetMicVolume@CSwiGobiDll@@QAAKPAG@Z (public: unsigned long __cdecl CSwiGobiDll::SetMicVolume(unsigned short *))
      167    ?SetMobileIP@CSwiGobiDll@@QAAKK@Z (public: unsigned long __cdecl CSwiGobiDll::SetMobileIP(unsigned long))
      168    ?SetMobileIPParameters@CSwiGobiDll@@QAAKPADPAKPAE22222@Z (public: unsigned long __cdecl CSwiGobiDll::SetMobileIPParameters(char *,unsigned long *,unsigned char *,unsigned char *,unsigned char *,unsigned char *,unsigned char *,unsigned char *))
      169    ?SetMobileIPProfile@CSwiGobiDll@@QAAKPADEPAEPAK22102200@Z (public: unsigned long __cdecl CSwiGobiDll::SetMobileIPProfile(char *,unsigned char,unsigned char *,unsigned long *,unsigned long *,unsigned long *,unsigned char *,char *,unsigned long *,unsigned long *,char *,char *))
      170    ?SetMobileIPStatusCB@CSwiGobiDll@@SAKP6AXK@Z@Z (public: static unsigned long __cdecl CSwiGobiDll::SetMobileIPStatusCB(void (__cdecl*)(unsigned long)))
      171    ?SetNITZCB@CSwiGobiDll@@SAKP6AXGEEEEEEEE@Z@Z (public: static unsigned long __cdecl CSwiGobiDll::SetNITZCB(void (__cdecl*)(unsigned short,unsigned char,unsigned char,unsigned char,unsigned char,unsigned char,unsigned char,unsigned char,unsigned char)))
      172    ?SetNMEAConfig@CSwiGobiDll@@QAAKEEEPAG@Z (public: unsigned long __cdecl CSwiGobiDll::SetNMEAConfig(unsigned char,unsigned char,unsigned char,unsigned short *))
      173    ?SetNetworkPreference@CSwiGobiDll@@QAAKKK@Z (public: unsigned long __cdecl CSwiGobiDll::SetNetworkPreference(unsigned long,unsigned long))
      174    ?SetNewSMSCB@CSwiGobiDll@@SAKP6AXKK@Z@Z (public: static unsigned long __cdecl CSwiGobiDll::SetNewSMSCB(void (__cdecl*)(unsigned long,unsigned long)))
      175    ?SetNewSMSCBCB@CSwiGobiDll@@SAKP6AXEKEGPAE@Z@Z (public: static unsigned long __cdecl CSwiGobiDll::SetNewSMSCBCB(void (__cdecl*)(unsigned char,unsigned long,unsigned char,unsigned short,unsigned char *)))
      176    ?SetNoiseSuppression@CSwiGobiDll@@QAAKPAE@Z (public: unsigned long __cdecl CSwiGobiDll::SetNoiseSuppression(unsigned char *))
      177    ?SetOMADMAlertCB@CSwiGobiDll@@SAKP6AXKG@Z@Z (public: static unsigned long __cdecl CSwiGobiDll::SetOMADMAlertCB(void (__cdecl*)(unsigned long,unsigned short)))
      178    ?SetOMADMStateCB@CSwiGobiDll@@SAKP6AXKK@Z@Z (public: static unsigned long __cdecl CSwiGobiDll::SetOMADMStateCB(void (__cdecl*)(unsigned long,unsigned long)))
      179    ?SetOMAEXEventCB@CSwiGobiDll@@SAKP6AXPAUFUMOInfo@@PAUOMAInfo@@@Z@Z (public: static unsigned long __cdecl CSwiGobiDll::SetOMAEXEventCB(void (__cdecl*)(struct FUMOInfo *,struct OMAInfo *)))
      180    ?SetPDSDefaults@CSwiGobiDll@@QAAKKEKK@Z (public: unsigned long __cdecl CSwiGobiDll::SetPDSDefaults(unsigned long,unsigned char,unsigned long,unsigned long))
      181    ?SetPDSState@CSwiGobiDll@@QAAKK@Z (public: unsigned long __cdecl CSwiGobiDll::SetPDSState(unsigned long))
      182    ?SetPhonebookRecordReadCB@CSwiGobiDll@@SAKP6AXEGPAUarrPBInfo@@@Z@Z (public: static unsigned long __cdecl CSwiGobiDll::SetPhonebookRecordReadCB(void (__cdecl*)(unsigned char,unsigned short,struct arrPBInfo *)))
      183    ?SetPortAutomaticTracking@CSwiGobiDll@@QAAKK@Z (public: unsigned long __cdecl CSwiGobiDll::SetPortAutomaticTracking(unsigned long))
      184    ?SetPower@CSwiGobiDll@@QAAKK@Z (public: unsigned long __cdecl CSwiGobiDll::SetPower(unsigned long))
      185    ?SetPowerCB@CSwiGobiDll@@SAKP6AXK@Z@Z (public: static unsigned long __cdecl CSwiGobiDll::SetPowerCB(void (__cdecl*)(unsigned long)))
      186    ?SetRFInfoCB@CSwiGobiDll@@SAKP6AXKKK@Z@Z (public: static unsigned long __cdecl CSwiGobiDll::SetRFInfoCB(void (__cdecl*)(unsigned long,unsigned long,unsigned long)))
      187    ?SetRXGainLevel@CSwiGobiDll@@QAAKPAEPAG1@Z (public: unsigned long __cdecl CSwiGobiDll::SetRXGainLevel(unsigned char *,unsigned short *,unsigned short *))
      188    ?SetRXPCMFilter@CSwiGobiDll@@QAAKPAG0PAK0@Z (public: unsigned long __cdecl CSwiGobiDll::SetRXPCMFilter(unsigned short *,unsigned short *,unsigned long *,unsigned short *))
      189    ?SetReceiverVolume@CSwiGobiDll@@QAAKPAE@Z (public: unsigned long __cdecl CSwiGobiDll::SetReceiverVolume(unsigned char *))
      190    ?SetRoamingIndicatorCB@CSwiGobiDll@@SAKP6AXK@Z@Z (public: static unsigned long __cdecl CSwiGobiDll::SetRoamingIndicatorCB(void (__cdecl*)(unsigned long)))
      191    ?SetSMSBroadcastActivation@CSwiGobiDll@@QAAKEE@Z (public: unsigned long __cdecl CSwiGobiDll::SetSMSBroadcastActivation(unsigned char,unsigned char))
      192    ?SetSMSCAddress@CSwiGobiDll@@QAAKPAD0@Z (public: unsigned long __cdecl CSwiGobiDll::SetSMSCAddress(char *,char *))
      193    ?SetSMSProtocol@CSwiGobiDll@@QAAKE@Z (public: unsigned long __cdecl CSwiGobiDll::SetSMSProtocol(unsigned char))
      194    ?SetSMSRoute@CSwiGobiDll@@QAAKKPAE@Z (public: unsigned long __cdecl CSwiGobiDll::SetSMSRoute(unsigned long,unsigned char *))
      195    ?SetSUPS@CSwiGobiDll@@QAAKPAUvoiceSetSUPSServiceReq@@PAGPAUalphaIDInfo@@PAE3PAUccSUPSType@@@Z (public: unsigned long __cdecl CSwiGobiDll::SetSUPS(struct voiceSetSUPSServiceReq *,unsigned short *,struct alphaIDInfo *,unsigned char *,unsigned char *,struct ccSUPSType *))
      196    ?SetServiceAutomaticTracking@CSwiGobiDll@@QAAKK@Z (public: unsigned long __cdecl CSwiGobiDll::SetServiceAutomaticTracking(unsigned long))
      197    ?SetSessionStateCB@CSwiGobiDll@@SAKP6AXKK@Z@Z (public: static unsigned long __cdecl CSwiGobiDll::SetSessionStateCB(void (__cdecl*)(unsigned long,unsigned long)))
      198    ?SetSideToneGain@CSwiGobiDll@@QAAKPAG@Z (public: unsigned long __cdecl CSwiGobiDll::SetSideToneGain(unsigned short *))
      199    ?SetSignalStrengthCB@CSwiGobiDll@@SAKP6AXCK@ZEPAC@Z (public: static unsigned long __cdecl CSwiGobiDll::SetSignalStrengthCB(void (__cdecl*)(signed char,unsigned long),unsigned char,signed char *))
      200    ?SetSpeakerMuteStatus@CSwiGobiDll@@QAAKPAE@Z (public: unsigned long __cdecl CSwiGobiDll::SetSpeakerMuteStatus(unsigned char *))
      201    ?SetTXPCMFilter@CSwiGobiDll@@QAAKPAG0PAK0@Z (public: unsigned long __cdecl CSwiGobiDll::SetTXPCMFilter(unsigned short *,unsigned short *,unsigned long *,unsigned short *))
      202    ?SetUSSDInfoCB@CSwiGobiDll@@SAKP6AXPAEPAUUSSInfo@@@Z@Z (public: static unsigned long __cdecl CSwiGobiDll::SetUSSDInfoCB(void (__cdecl*)(unsigned char *,struct USSInfo *)))
      203    ?SetVoiceMessageCB@CSwiGobiDll@@SAKP6AXEPAE00@Z@Z (public: static unsigned long __cdecl CSwiGobiDll::SetVoiceMessageCB(void (__cdecl*)(unsigned char,unsigned char *,unsigned char *,unsigned char *)))
      204    ?SetXTRAAutomaticDownload@CSwiGobiDll@@QAAKKG@Z (public: unsigned long __cdecl CSwiGobiDll::SetXTRAAutomaticDownload(unsigned long,unsigned short))
      205    ?SetXTRAEmbeddedClient@CSwiGobiDll@@QAAKEE@Z (public: unsigned long __cdecl CSwiGobiDll::SetXTRAEmbeddedClient(unsigned char,unsigned char))
      206    ?SetXTRANetwork@CSwiGobiDll@@QAAKK@Z (public: unsigned long __cdecl CSwiGobiDll::SetXTRANetwork(unsigned long))
      207    ?SetXTRAValidity@CSwiGobiDll@@QAAKGGG@Z (public: unsigned long __cdecl CSwiGobiDll::SetXTRAValidity(unsigned short,unsigned short,unsigned short))
      208    ?StartDTMF@CSwiGobiDll@@QAAKPAE00@Z (public: unsigned long __cdecl CSwiGobiDll::StartDTMF(unsigned char *,unsigned char *,unsigned char *))
      209    ?StartDataSession@CSwiGobiDll@@QAAKPAD00PAK1@Z (public: unsigned long __cdecl CSwiGobiDll::StartDataSession(char *,char *,char *,unsigned long *,unsigned long *))
      210    ?StopDTMF@CSwiGobiDll@@QAAKPAE0@Z (public: unsigned long __cdecl CSwiGobiDll::StopDTMF(unsigned char *,unsigned char *))
      211    ?StopDataSession@CSwiGobiDll@@QAAKK@Z (public: unsigned long __cdecl CSwiGobiDll::StopDataSession(unsigned long))
      212    ?SwiGetAudioMode@@YA?AW4SWI_RCODE@@PAGK@Z (enum SWI_RCODE __cdecl SwiGetAudioMode(unsigned short *,unsigned long))
      213    ?SwiM2MAV_AudioGetAVCFG@CSwiGobiDll@@QAAKPAUAudioConfig@@PAE@Z (public: unsigned long __cdecl CSwiGobiDll::SwiM2MAV_AudioGetAVCFG(struct AudioConfig *,unsigned char *))
      214    ?SwiM2MAV_AudioGetAVEC@CSwiGobiDll@@QAAKPAE0@Z (public: unsigned long __cdecl CSwiGobiDll::SwiM2MAV_AudioGetAVEC(unsigned char *,unsigned char *))
      215    ?SwiM2MAV_AudioGetAVMute@CSwiGobiDll@@QAAKPAE000@Z (public: unsigned long __cdecl CSwiGobiDll::SwiM2MAV_AudioGetAVMute(unsigned char *,unsigned char *,unsigned char *,unsigned char *))
      216    ?SwiM2MAV_AudioGetAVNS@CSwiGobiDll@@QAAKPAE0@Z (public: unsigned long __cdecl CSwiGobiDll::SwiM2MAV_AudioGetAVNS(unsigned char *,unsigned char *))
      217    ?SwiM2MAV_AudioGetAVRXG@CSwiGobiDll@@QAAKPAEPAG@Z (public: unsigned long __cdecl CSwiGobiDll::SwiM2MAV_AudioGetAVRXG(unsigned char *,unsigned short *))
      218    ?SwiM2MAV_AudioGetAVTXG@CSwiGobiDll@@QAAKPAEPAG@Z (public: unsigned long __cdecl CSwiGobiDll::SwiM2MAV_AudioGetAVTXG(unsigned char *,unsigned short *))
      219    ?SwiM2MAV_AudioGetMicGain@CSwiGobiDll@@QAAKPAEPAG@Z (public: unsigned long __cdecl CSwiGobiDll::SwiM2MAV_AudioGetMicGain(unsigned char *,unsigned short *))
      220    ?SwiM2MAV_AudioGetProfile@CSwiGobiDll@@QAAKPAE000000@Z (public: unsigned long __cdecl CSwiGobiDll::SwiM2MAV_AudioGetProfile(unsigned char *,unsigned char *,unsigned char *,unsigned char *,unsigned char *,unsigned char *,unsigned char *))
      221    ?SwiM2MAV_AudioGetSTG@CSwiGobiDll@@QAAKPAEPAG@Z (public: unsigned long __cdecl CSwiGobiDll::SwiM2MAV_AudioGetSTG(unsigned char *,unsigned short *))
      222    ?SwiM2MAV_AudioGetSpeakerGain@CSwiGobiDll@@QAAKPAEPAG@Z (public: unsigned long __cdecl CSwiGobiDll::SwiM2MAV_AudioGetSpeakerGain(unsigned char *,unsigned short *))
      223    ?SwiM2MAV_AudioGetTxVolume@CSwiGobiDll@@QAAKPAEPAG@Z (public: unsigned long __cdecl CSwiGobiDll::SwiM2MAV_AudioGetTxVolume(unsigned char *,unsigned short *))
      224    ?SwiM2MAV_AudioGetVolDB@CSwiGobiDll@@QAAKPAE00PAG@Z (public: unsigned long __cdecl CSwiGobiDll::SwiM2MAV_AudioGetVolDB(unsigned char *,unsigned char *,unsigned char *,unsigned short *))
      225    ?SwiM2MAV_AudioGetVolume@CSwiGobiDll@@QAAKPAE00@Z (public: unsigned long __cdecl CSwiGobiDll::SwiM2MAV_AudioGetVolume(unsigned char *,unsigned char *,unsigned char *))
      226    ?SwiM2MAV_AudioNVDef@CSwiGobiDll@@QAAKXZ (public: unsigned long __cdecl CSwiGobiDll::SwiM2MAV_AudioNVDef(void))
      227    ?SwiM2MAV_AudioPlayTone@CSwiGobiDll@@QAAKPAE0PAG@Z (public: unsigned long __cdecl CSwiGobiDll::SwiM2MAV_AudioPlayTone(unsigned char *,unsigned char *,unsigned short *))
      228    ?SwiM2MAV_AudioSetAVCFG@CSwiGobiDll@@QAAKPAE00PAUPIFACETable@@@Z (public: unsigned long __cdecl CSwiGobiDll::SwiM2MAV_AudioSetAVCFG(unsigned char *,unsigned char *,unsigned char *,struct PIFACETable *))
      229    ?SwiM2MAV_AudioSetAVEC@CSwiGobiDll@@QAAKPAE0@Z (public: unsigned long __cdecl CSwiGobiDll::SwiM2MAV_AudioSetAVEC(unsigned char *,unsigned char *))
      230    ?SwiM2MAV_AudioSetAVMute@CSwiGobiDll@@QAAKPAE000@Z (public: unsigned long __cdecl CSwiGobiDll::SwiM2MAV_AudioSetAVMute(unsigned char *,unsigned char *,unsigned char *,unsigned char *))
      231    ?SwiM2MAV_AudioSetAVNS@CSwiGobiDll@@QAAKPAE0@Z (public: unsigned long __cdecl CSwiGobiDll::SwiM2MAV_AudioSetAVNS(unsigned char *,unsigned char *))
      232    ?SwiM2MAV_AudioSetAVRXG@CSwiGobiDll@@QAAKPAEPAG@Z (public: unsigned long __cdecl CSwiGobiDll::SwiM2MAV_AudioSetAVRXG(unsigned char *,unsigned short *))
      233    ?SwiM2MAV_AudioSetAVTXG@CSwiGobiDll@@QAAKPAEPAG@Z (public: unsigned long __cdecl CSwiGobiDll::SwiM2MAV_AudioSetAVTXG(unsigned char *,unsigned short *))
      234    ?SwiM2MAV_AudioSetLPBK@CSwiGobiDll@@QAAKPAE@Z (public: unsigned long __cdecl CSwiGobiDll::SwiM2MAV_AudioSetLPBK(unsigned char *))
      235    ?SwiM2MAV_AudioSetMicGain@CSwiGobiDll@@QAAKPAEPAG@Z (public: unsigned long __cdecl CSwiGobiDll::SwiM2MAV_AudioSetMicGain(unsigned char *,unsigned short *))
      236    ?SwiM2MAV_AudioSetProfile@CSwiGobiDll@@QAAKPAE00000@Z (public: unsigned long __cdecl CSwiGobiDll::SwiM2MAV_AudioSetProfile(unsigned char *,unsigned char *,unsigned char *,unsigned char *,unsigned char *,unsigned char *))
      237    ?SwiM2MAV_AudioSetSTG@CSwiGobiDll@@QAAKPAEPAG@Z (public: unsigned long __cdecl CSwiGobiDll::SwiM2MAV_AudioSetSTG(unsigned char *,unsigned short *))
      238    ?SwiM2MAV_AudioSetSpeakerGain@CSwiGobiDll@@QAAKPAEPAG@Z (public: unsigned long __cdecl CSwiGobiDll::SwiM2MAV_AudioSetSpeakerGain(unsigned char *,unsigned short *))
      239    ?SwiM2MAV_AudioSetTxVolume@CSwiGobiDll@@QAAKPAEPAG@Z (public: unsigned long __cdecl CSwiGobiDll::SwiM2MAV_AudioSetTxVolume(unsigned char *,unsigned short *))
      240    ?SwiM2MAV_AudioSetVolDB@CSwiGobiDll@@QAAKPAE00PAG@Z (public: unsigned long __cdecl CSwiGobiDll::SwiM2MAV_AudioSetVolDB(unsigned char *,unsigned char *,unsigned char *,unsigned short *))
      241    ?SwiM2MAV_AudioSetVolume@CSwiGobiDll@@QAAKPAE00@Z (public: unsigned long __cdecl CSwiGobiDll::SwiM2MAV_AudioSetVolume(unsigned char *,unsigned char *,unsigned char *))
      242    ?SwiSetAudioMode@@YA?AW4SWI_RCODE@@GK@Z (enum SWI_RCODE __cdecl SwiSetAudioMode(unsigned short,unsigned long))
      243    ?UIMChangePIN@CSwiGobiDll@@QAAKPAUQMI_UIM_CHANGE_PIN_REQ_SESSION_INFORMATION@@PAUQMI_UIM_CHANGE_PIN_REQ_CHANGE_PIN@@PAUQMI_UIM_CHANGE_PIN_RESP_RETRIES_REMAINING@@@Z (public: unsigned long __cdecl CSwiGobiDll::UIMChangePIN(struct QMI_UIM_CHANGE_PIN_REQ_SESSION_INFORMATION *,struct QMI_UIM_CHANGE_PIN_REQ_CHANGE_PIN *,struct QMI_UIM_CHANGE_PIN_RESP_RETRIES_REMAINING *))
      244    ?UIMGetCardStatus@CSwiGobiDll@@QAAKPAHPAUQMI_UIM_GET_CARD_STATUS_RESP@@@Z (public: unsigned long __cdecl CSwiGobiDll::UIMGetCardStatus(int *,struct QMI_UIM_GET_CARD_STATUS_RESP *))
      245    ?UIMSetPINProtection@CSwiGobiDll@@QAAKPAUQMI_UIM_SET_PIN_PROTECTION_REQ_SESSION_INFORMATION@@PAUQMI_UIM_SET_PIN_PROTECTION_REQ_SET_PIN_PROTECTION@@PAUQMI_UIM_SET_PIN_PROTECTION_RESP_RETRIES_REMAINING@@@Z (public: unsigned long __cdecl CSwiGobiDll::UIMSetPINProtection(struct QMI_UIM_SET_PIN_PROTECTION_REQ_SESSION_INFORMATION *,struct QMI_UIM_SET_PIN_PROTECTION_REQ_SET_PIN_PROTECTION *,struct QMI_UIM_SET_PIN_PROTECTION_RESP_RETRIES_REMAINING *))
      246    ?UIMUnblockPIN@CSwiGobiDll@@QAAKPAUQMI_UIM_UNBLOCK_PIN_REQ_SESSION_INFORMATION@@PAUQMI_UIM_UNBLOCK_PIN_REQ_UNBLOCK_PIN@@PAUQMI_UIM_UNBLOCK_PIN_RESP_RETRIES_REMAINING@@@Z (public: unsigned long __cdecl CSwiGobiDll::UIMUnblockPIN(struct QMI_UIM_UNBLOCK_PIN_REQ_SESSION_INFORMATION *,struct QMI_UIM_UNBLOCK_PIN_REQ_UNBLOCK_PIN *,struct QMI_UIM_UNBLOCK_PIN_RESP_RETRIES_REMAINING *))
      247    ?UIMVerifyPIN@CSwiGobiDll@@QAAKPAUQMI_UIM_VERIFY_PIN_REQ_SESSION_INFORMATION@@PAUQMI_UIM_VERIFY_PIN_REQ_VERIFY_PIN@@PAUQMI_UIM_VERIFY_PIN_RESP_RETRIES_REMAINING@@@Z (public: unsigned long __cdecl CSwiGobiDll::UIMVerifyPIN(struct QMI_UIM_VERIFY_PIN_REQ_SESSION_INFORMATION *,struct QMI_UIM_VERIFY_PIN_REQ_VERIFY_PIN *,struct QMI_UIM_VERIFY_PIN_RESP_RETRIES_REMAINING *))
      248    ?UpgradeFirmwareW@CSwiGobiDll@@QAAKPAG@Z (public: unsigned long __cdecl CSwiGobiDll::UpgradeFirmwareW(unsigned short *))
      249    ?ValidateSPC@CSwiGobiDll@@QAAKPAD@Z (public: unsigned long __cdecl CSwiGobiDll::ValidateSPC(char *))
      250    ?WritePhonebookRecord@CSwiGobiDll@@QAAKPAEPAG1000000@Z (public: unsigned long __cdecl CSwiGobiDll::WritePhonebookRecord(unsigned char *,unsigned short *,unsigned short *,unsigned char *,unsigned char *,unsigned char *,unsigned char *,unsigned char *,unsigned char *))
      251    ?mpFNSetActivationStatusCB@CSwiGobiDll@@1P6AKP6AXK@Z@ZA (protected: static unsigned long (__cdecl* CSwiGobiDll::mpFNSetActivationStatusCB)(void (__cdecl*)(unsigned long)))
      252    ?mpFNSetAllPbInitDoneCB@CSwiGobiDll@@1P6AKP6AXEPAEPAG@Z@ZA (protected: static unsigned long (__cdecl* CSwiGobiDll::mpFNSetAllPbInitDoneCB)(void (__cdecl*)(unsigned char,unsigned char *,unsigned short *)))
      253    ?mpFNSetByteTotalsCB@CSwiGobiDll@@1P6AKP6AX_K0@ZE@ZA (protected: static unsigned long (__cdecl* CSwiGobiDll::mpFNSetByteTotalsCB)(void (__cdecl*)(unsigned __int64,unsigned __int64),unsigned char))
      254    ?mpFNSetCallInfoCB@CSwiGobiDll@@1P6AKP6AXPAUarrCallInfo@@PAUarrRemotePartyNum@@PAUarrRemotePartyName@@PAUarrAlertingType@@PAUarrSvcOption@@PAUarrCallEndReason@@PAUarrAlphaIDInfo@@PAUarrPeerNumInfo@@PAUarrDiagInfo@@77PAUarrAlertingPattern@@@Z@ZA (protected: static unsigned long (__cdecl* CSwiGobiDll::mpFNSetCallInfoCB)(void (__cdecl*)(struct arrCallInfo *,struct arrRemotePartyNum *,struct arrRemotePartyName *,struct arrAlertingType *,struct arrSvcOption *,struct arrCallEndReason *,struct arrAlphaIDInfo *,struct arrPeerNumInfo *,struct arrDiagInfo *,struct arrPeerNumInfo *,struct arrPeerNumInfo *,struct arrAlertingPattern *)))
      255    ?mpFNSetDataBearerCB@CSwiGobiDll@@1P6AKP6AXK@Z@ZA (protected: static unsigned long (__cdecl* CSwiGobiDll::mpFNSetDataBearerCB)(void (__cdecl*)(unsigned long)))
      256    ?mpFNSetDataCapabilitiesCB@CSwiGobiDll@@1P6AKP6AXEPAE@Z@ZA (protected: static unsigned long (__cdecl* CSwiGobiDll::mpFNSetDataCapabilitiesCB)(void (__cdecl*)(unsigned char,unsigned char *)))
      257    ?mpFNSetDormancyStatusCB@CSwiGobiDll@@1P6AKP6AXK@Z@ZA (protected: static unsigned long (__cdecl* CSwiGobiDll::mpFNSetDormancyStatusCB)(void (__cdecl*)(unsigned long)))
      258    ?mpFNSetEmergencyListCB@CSwiGobiDll@@1P6AKP6AXEPAUemergencyNumberEntry@@@Z@ZA (protected: static unsigned long (__cdecl* CSwiGobiDll::mpFNSetEmergencyListCB)(void (__cdecl*)(unsigned char,struct emergencyNumberEntry *)))
      259    ?mpFNSetEmergencyModeCB@CSwiGobiDll@@1P6AKP6AXPAE@Z@ZA (protected: static unsigned long (__cdecl* CSwiGobiDll::mpFNSetEmergencyModeCB)(void (__cdecl*)(unsigned char *)))
      260    ?mpFNSetInfoRecCB@CSwiGobiDll@@1P6AKP6AXPAEPAUsignalInfo@@PAUcallerIDInfo@@PAD330PAUpeerNumInfo@@44PAUredirectNumInfo@@0000PAUlineCtlInfo@@PAUextDisplayInfo@@@Z@ZA (protected: static unsigned long (__cdecl* CSwiGobiDll::mpFNSetInfoRecCB)(void (__cdecl*)(unsigned char *,struct signalInfo *,struct callerIDInfo *,char *,char *,char *,unsigned char *,struct peerNumInfo *,struct peerNumInfo *,struct peerNumInfo *,struct redirectNumInfo *,unsigned char *,unsigned char *,unsigned char *,unsigned char *,struct lineCtlInfo *,struct extDisplayInfo *)))
      261    ?mpFNSetMobileIPStatusCB@CSwiGobiDll@@1P6AKP6AXK@Z@ZA (protected: static unsigned long (__cdecl* CSwiGobiDll::mpFNSetMobileIPStatusCB)(void (__cdecl*)(unsigned long)))
      262    ?mpFNSetNITZCB@CSwiGobiDll@@1P6AKP6AXGEEEEEEEE@Z@ZA (protected: static unsigned long (__cdecl* CSwiGobiDll::mpFNSetNITZCB)(void (__cdecl*)(unsigned short,unsigned char,unsigned char,unsigned char,unsigned char,unsigned char,unsigned char,unsigned char,unsigned char)))
      263    ?mpFNSetNewSMSCB@CSwiGobiDll@@1P6AKP6AXKK@Z@ZA (protected: static unsigned long (__cdecl* CSwiGobiDll::mpFNSetNewSMSCB)(void (__cdecl*)(unsigned long,unsigned long)))
      264    ?mpFNSetNewSMSCBCB@CSwiGobiDll@@1P6AKP6AXEKEGPAE@Z@ZA (protected: static unsigned long (__cdecl* CSwiGobiDll::mpFNSetNewSMSCBCB)(void (__cdecl*)(unsigned char,unsigned long,unsigned char,unsigned short,unsigned char *)))
      265    ?mpFNSetOMADMNIAlertCB@CSwiGobiDll@@1P6AKP6AXKG@Z@ZA (protected: static unsigned long (__cdecl* CSwiGobiDll::mpFNSetOMADMNIAlertCB)(void (__cdecl*)(unsigned long,unsigned short)))
      266    ?mpFNSetOMADMStateCB@CSwiGobiDll@@1P6AKP6AXKK@Z@ZA (protected: static unsigned long (__cdecl* CSwiGobiDll::mpFNSetOMADMStateCB)(void (__cdecl*)(unsigned long,unsigned long)))
      267    ?mpFNSetOMAEXEventCB@CSwiGobiDll@@1P6AKP6AXPAUFUMOInfo@@PAUOMAInfo@@@Z@ZA (protected: static unsigned long (__cdecl* CSwiGobiDll::mpFNSetOMAEXEventCB)(void (__cdecl*)(struct FUMOInfo *,struct OMAInfo *)))
      268    ?mpFNSetPhonebookRecordReadCB@CSwiGobiDll@@1P6AKP6AXEGPAUarrPBInfo@@@Z@ZA (protected: static unsigned long (__cdecl* CSwiGobiDll::mpFNSetPhonebookRecordReadCB)(void (__cdecl*)(unsigned char,unsigned short,struct arrPBInfo *)))
      269    ?mpFNSetPowerCB@CSwiGobiDll@@1P6AKP6AXK@Z@ZA (protected: static unsigned long (__cdecl* CSwiGobiDll::mpFNSetPowerCB)(void (__cdecl*)(unsigned long)))
      270    ?mpFNSetRFInfoCB@CSwiGobiDll@@1P6AKP6AXKKK@Z@ZA (protected: static unsigned long (__cdecl* CSwiGobiDll::mpFNSetRFInfoCB)(void (__cdecl*)(unsigned long,unsigned long,unsigned long)))
      271    ?mpFNSetRoamingIndicatorCB@CSwiGobiDll@@1P6AKP6AXK@Z@ZA (protected: static unsigned long (__cdecl* CSwiGobiDll::mpFNSetRoamingIndicatorCB)(void (__cdecl*)(unsigned long)))
      272    ?mpFNSetSessionStateCB@CSwiGobiDll@@1P6AKP6AXKK@Z@ZA (protected: static unsigned long (__cdecl* CSwiGobiDll::mpFNSetSessionStateCB)(void (__cdecl*)(unsigned long,unsigned long)))
      273    ?mpFNSetSignalStrengthCB@CSwiGobiDll@@1P6AKP6AXCK@ZEPAC@ZA (protected: static unsigned long (__cdecl* CSwiGobiDll::mpFNSetSignalStrengthCB)(void (__cdecl*)(signed char,unsigned long),unsigned char,signed char *))
      274    ?mpFNSetUSSDInfoCB@CSwiGobiDll@@1P6AKP6AXPAEPAUUSSInfo@@@Z@ZA (protected: static unsigned long (__cdecl* CSwiGobiDll::mpFNSetUSSDInfoCB)(void (__cdecl*)(unsigned char *,struct USSInfo *)))
      275    ?mpFNSetVoiceMsgCB@CSwiGobiDll@@1P6AKP6AXEPAE00@Z@ZA (protected: static unsigned long (__cdecl* CSwiGobiDll::mpFNSetVoiceMsgCB)(void (__cdecl*)(unsigned char,unsigned char *,unsigned char *,unsigned char *)))
      276    SwiATGetCLIP
      277    SwiATGetCLIR
      278    SwiATGetCOLP
      279    SwiATGetCOLR
      280    SwiATGetProvisionStatus
      281    SwiATReleaseCall
      282    SwiATReset
      283    SwiATRtnReset
      284    SwiATSetCLIP
      285    SwiATSetCLIR
      286    SwiATSetCOLP
      287    SwiATSetCOLR
      288    SwiATSetEnum
      289    SwiATSetSideToneGain
      290    SwiActivateAutomatic
      291    SwiActivateProfile
      292    SwiAddPreferredOperatorGobi
      293    SwiAnserCall
      294    SwiApiShutdown
      295    SwiApiStartup
      296    SwiCancelOMADMSession
      297    SwiDeRegisterCallback
      298    SwiDialCall
      299    SwiEndCall
      300    SwiGetActivationStatus
      301    SwiGetActiveNam
      302    SwiGetAirServerInfo
      303    SwiGetAvailAirServers
      304    SwiGetBootVersion
      305    SwiGetByteCounter
      306    SwiGetCDMANetworkParameters
      307    SwiGetCallConnectionState
      308    SwiGetCarrierID
      309    SwiGetCdmaIMSI
      310    SwiGetCdmaSMSMessageStatus
      311    SwiGetChannelNumber
      312    SwiGetCurrentBaseStation
      313    SwiGetECIO
      314    SwiGetEFile
      315    SwiGetEFileInfo
      316    SwiGetESN
      317    SwiGetESNGobi
      318    SwiGetFirmwareVersion
      319    SwiGetGeneralFeatureSupport
      320    SwiGetGsmIMSI
      321    SwiGetGsmProfileBasic
      322    SwiGetGsmProfileSummary
      323    SwiGetGsmSMSCAddr
      324    SwiGetGsmSystemStatus
      325    SwiGetHardwareVersion
      326    SwiGetHdrHybrPref
      327    SwiGetHdrRoamStatus
      328    SwiGetHdrSrvState
      329    SwiGetIOTADisable
      330    SwiGetIPAddress
      331    SwiGetIPConfigurationGobi
      332    SwiGetImagePreference
      333    SwiGetImei
      334    SwiGetMEIDESN
      335    SwiGetMipErrCode
      336    SwiGetMobileIPProfile
      337    SwiGetModelID
      338    SwiGetNDISMode
      339    SwiGetNetworkProviderID
      340    SwiGetOMADMConfig
      341    SwiGetOMADMNIAlert
      342    SwiGetOMADMSessionState
      343    SwiGetPLMNMode
      344    SwiGetPLMNSelection
      345    SwiGetPRLVersion
      346    SwiGetPhoneNumber
      347    SwiGetPhonebookEntry
      348    SwiGetPinStatus
      349    SwiGetPktSessionStatus
      350    SwiGetPktSessionStatusEx
      351    SwiGetPower
      352    SwiGetPreferredOperatorListGobi
      353    SwiGetPriInfo
      354    SwiGetPriVersion
      355    SwiGetProfile
      356    SwiGetProfileSummary
      357    SwiGetRadioPower
      358    SwiGetRoamingStatus
      359    SwiGetRssi
      360    SwiGetRssiEcio
      361    SwiGetSIMRecordStatus
      362    SwiGetSMSMessageStatus
      363    SwiGetServiceIndication
      364    SwiGetServingNetworkGobi
      365    SwiGetSimLock
      366    SwiGetSimLockGobi
      367    SwiGetSimVerifyGobi
      368    SwiGetSystemTime
      369    SwiGetTechBandClass
      370    SwiGetTechHardwareVersion
      371    SwiGetTechNID
      372    SwiGetTechPowersaveMode
      373    SwiGetTechSID
      374    SwiGetTrafficStatistics
      375    SwiHandleResume
      376    SwiHandleSuspend
      377    SwiIsModemReady
      378    SwiManageCalls
      379    SwiModemReset
      380    SwiNotify
      381    SwiOMAEXGetSessionInfo
      382    SwiOMAEXGetSettings
      383    SwiOMAEXInit
      384    SwiOMAEXSelection
      385    SwiOMAEXSessionCancel
      386    SwiOMAEXSessionStart
      387    SwiOMAEXSetSettings
      388    SwiOMAEXShutdown
      389    SwiPowerSaveExit
      390    SwiPriGetActivationMask
      391    SwiPriGetMDNLength
      392    SwiPriGetMaxMosmsLen
      393    SwiPstGetAccolc
      394    SwiPstGetDisplayBannerName
      395    SwiPstGetDsMipActiveProf
      396    SwiPstGetDsMipEnableProf
      397    SwiPstGetDsMipGenUser
      398    SwiPstGetDsMipSsUserProf
      399    SwiPstGetDsQcMip
      400    SwiPstGetHdrPassword
      401    SwiPstGetHdrUserId
      402    SwiPstGetHomeSidNid
      403    SwiPstGetImsi1112
      404    SwiPstGetImsiMcc
      405    SwiPstGetPrefMode
      406    SwiPstGetSci
      407    SwiPstGetSystemPref
      408    SwiPstGetTermHome
      409    SwiPstGetTermNid
      410    SwiPstGetTermSid
      411    SwiPstLock
      412    SwiPstSetAccolc
      413    SwiPstSetCurrentNam
      414    SwiPstSetDsMipActiveProf
      415    SwiPstSetDsMipGenUser
      416    SwiPstSetDsMipSsUserProf
      417    SwiPstSetDsQcMip
      418    SwiPstSetHdrPassword
      419    SwiPstSetHdrUserId
      420    SwiPstSetHomeSidNid
      421    SwiPstSetImsi1112
      422    SwiPstSetImsiMcc
      423    SwiPstSetPrefMode
      424    SwiPstSetSci
      425    SwiPstUnlock
      426    SwiRegisterCallback
      427    SwiRemovePreferredOperatorGobi
      428    SwiResetByteCounter
      429    SwiResetModem
      430    SwiRetrieveCBSMSMessageGobi
      431    SwiRetrieveCdmaSMSMessage
      432    SwiRetrieveSMSMessageGobi
      433    SwiRtnReset
      434    SwiSelectAirServer
      435    SwiSendCdmaSMS
      436    SwiSendGenericSimCommand
      437    SwiSendRestrictedSIMCmd
      438    SwiSendSMS
      439    SwiSetAKey
      440    SwiSetCallDisconnectCmd
      441    SwiSetCallOriginateCmd
      442    SwiSetDormant
      443    SwiSetGsmProfileBasic
      444    SwiSetGsmSMSCAddr
      445    SwiSetHdrHybrPref
      446    SwiSetHostStartup
      447    SwiSetIMSI
      448    SwiSetImagePreference
      449    SwiSetMobileDirNum
      450    SwiSetMobileIPProfile
      451    SwiSetNDISPrefMode
      452    SwiSetNetworkPreferenceGobi
      453    SwiSetOMADMConfig
      454    SwiSetOMADMNIAlertResponse
      455    SwiSetOMAEXEventReport
      456    SwiSetPLMNMode
      457    SwiSetPower
      458    SwiSetPowerDown
      459    SwiSetProfile
      460    SwiSetRadioPower
      461    SwiSetSimLock
      462    SwiSetSimLockGobi
      463    SwiSetSimPassword
      464    SwiSetSimPasswordGobi
      465    SwiSetSimVerifyGobi
      466    SwiSetTempModePref
      467    SwiStartDataSession
      468    SwiStartOMADMSession
      469    SwiStartPLMNSearch
      470    SwiStopDataSession
      471    SwiStopNotify
      472    SwiStoreCdmaSMSMessage
      473    SwiStoreSMSMessageGobi
      474    SwiUpgradeFirmware
